:020000040800F2
:10800000488A002069810008E1EB0008E5DC0008EF
:10801000DDEB00083D9B0008854E010800000000D4
:108020000000000000000000000000002D06010814
:10803000F9BE0008000000005DF700084D110108BE
:10804000E94F0108838100088381000883810008CB
:1080500083810008838100088381000883810008F0
:1080600083810008838100088381000883810008E0
:1080700083810008838100088381000883810008D0
:10808000838100088381000883810008C59B000864
:10809000419B000883810008619B000883810008E0
:1080A00083810008838100088381000883810008A0
:1080B00083810008ED120108838100088381000894
:1080C0008381000883810008838100088381000880
:1080D00083810008F93B0108A13C0108793D0108B2
:1080E000838100088381000883810008000000006C
:1080F0000000000000000000000000000000000080
:108100000000000000000000838100088381000857
:10811000A52B01089D2C010883810008838100089C
:10812000838100088381000883810008838100081F
:10813000838100088381000883810008A99E0008CC
:1081400083810008DD9D0008159E000883810008DA
:10815000DFF810D000F0AEFC00480047E1870108CE
:10816000AFF30080488A0020064880470648004751
:10817000FEE7FEE7FEE7FEE7FEE7FEE7FEE7FEE7D7
:10818000FEE7FEE72112010851810008202A04DBE6
:10819000203A00FA02F1002070479140C2F120031A
:1081A00020FA03F3194390407047202A04DB203A59
:1081B00021FA02F00021704721FA02F3D040C2F107
:1081C0002002914008431946704740EA01039B078B
:1081D00003D009E008C9121F08C0042AFAD203E03C
:1081E00011F8013B00F8013B521EF9D27047D2B2A0
:1081F00001E000F8012B491EFBD270470022F6E790
:1082000010B513460A4604461946FFF7F0FF20460C
:1082100010BD30B505462A460B4612F8010B13F87F
:10822000014B08B1A042F8D01CB1002802D06D1C4F
:10823000F1E7284630BD421C10F8011B0029FBD194
:10824000801A704730B504460020034600E05B1CEE
:10825000934203D2E05CCD5C401BF8D030BDF0B45B
:1082600080EA0102D40F4200B2EB410F02D2024673
:10827000084611464A0042D0C30DDDB2C1F3C752D1
:10828000AD1A202D35DAC1F3160141F4000204B114
:108290005242C5F1200602FA06F12A411044B3EB1E
:1082A000D05F23D0C4B1012DA0EBC35009DCF0BCDA
:1082B0004FF0004202EAC352DBB200F5000000F0CA
:1082C00055BB400000F1807000EBC350A0F18070FE
:1082D00040EAD170490009E0490841EAC071A0EBC9
:1082E000C35000F50000400800EBC350F0BC00F0A4
:1082F00034BB6142012202EB4101001BF6E7F0BCF6
:10830000704781F00041AAE780F00040A7E780EACB
:10831000010210B502F00043400022D04A001FD0F5
:10832000010E01EB1261C0F35600C2F3560240F495
:10833000000042F40002A0FB022000047F39140474
:1083400000D0401C50EA124001D44000491EC2B285
:108350000C0604EBD010401C4008802A02D003E039
:10836000002010BD20F00100002900DA0020184391
:1083700010BD30B480EA010202F0004530F0004246
:1083800021F0004013D090B1C30DD40DC2F31601FB
:10839000C0F31600E41A41F4000140F400027D34F9
:1083A000914201D3641C00E04900002C02DA30BC89
:1083B000002070474FF400000023914201D3891A36
:1083C000034340084FEA4101F7D151B1914202D134
:1083D0004FF0004105E002D24FF0010101E06FF0E3
:1083E000010103EBC450284430BC00F0B6BA2DE9BB
:1083F000FE4F804681EA0300C00F0C46009021F03A
:10840000004123F00045B8EB0200A94105D24046E7
:10841000214690461C460B46024623F0004010437E
:1084200047D0270DC7F30A00C3F30A510290401A40
:10843000019040286BDAC3F3130040F4801B0098CE
:10844000924620B10023D2EB030A63EB0B0B019899
:108450005946C0F140025046FFF798FE06460D46C9
:1084600050465946019A00F066FA10EB0800614147
:10847000002487EA115284EAE7731A4340D0009A35
:1084800062B3019A012A4FEA075215DC001B61EB27
:1084900002014FF0004202EA0752CDE90042001CFF
:1084A00041F5801132462B4600F09DFA03B0BDE83D
:1084B000F08F40462146F9E7001B61EB0201001CEA
:1084C00041F5801300185B412018A2F5001747EB17
:1084D000030140EAD570B6196D4111E06D084FEA0D
:1084E000360645EAC0754FEA0752001B61EB0201F0
:1084F000001C41F5801149084FEA30000019514134
:1085000032462B4603B0BDE8F04F00F05DBA00984C
:10851000012240000023D0EB020263EBE0730098DD
:1085200021464FEAE074B8EB000061EB0401E9E793
:1085300083F000435BE781F0004158E72DE9FE4FEF
:1085400081EA030404F0004421F0004100944FF05C
:10855000000B23F0004350EA01045ED052EA03040A
:108560005BD0C3F30A54C1F30A552C44A4F2F3348C
:108570000194A0FB0254C1F3130141F48011C3F331
:10858000130343F4801301FB024400FB034E840AEF
:10859000970A44EA815447EA8357A4FB0768029587
:1085A0008D0A05FB07854FEA932C04FB0C54270525
:1085B000029D4FEA065847EA1637B5EB08056EEB01
:1085C000070C870E920E47EA811742EA8312A7FB37
:1085D0000201B6EB0B0164EB00042B0D43EA0C33F4
:1085E0005E1844EB1C50DA465146E7FB0201C5F326
:1085F00013044FEA0B3343EA14534FEA0432019C4D
:1086000043EA0603A4F10C040294009CCDE900B4F3
:1086100000F0E9F903B0BDE8F08F00200146F9E76A
:108620002DE9F04D81EA030404F0004B21F00045F0
:1086300014464FF0000A23F0004150EA050220D012
:1086400054EA01021DD0C5F30A570246C5F31303CD
:10865000C1F31300C1F30A5640F4801543F48013AC
:10866000A7EB0608101BD64608F2FD3873EB050091
:1086700002D308F1010801E092185B41B8F1000F44
:1086800003DA00200146BDE8F08D00204FF4801190
:10869000064684460EE0171B73EB050705D3121B35
:1086A00063EB050306434CEA010C49084FEA30002E
:1086B00092185B4150EA0107EDD152EA030012D053
:1086C00082EA040083EA0501084305D0101BAB4190
:1086D00006D20122002306E000224FF0004302E010
:1086E0006FF0010253101AEB06004CEB085110EB2F
:1086F0000A0041EB0B01BDE8F04D00F065B9C10F78
:1087000080EAE0700844CA079623002100F02EB9E1
:1087100096230022114600F029B90EB540F23341EC
:1087200002910021CDE900110A460B4600F05BF9E9
:1087300003B000BD00F0004220F00040C10DC0F3C6
:10874000160040F400007F2901DA002070479629C6
:1087500003DCC1F19601C84001E096398840002A47
:10876000F4D04042704720F00040C10DC0F3160025
:1087700040F400007F2901DA00207047962903DCCD
:10878000C1F19601C8407047963988407047C1F3DF
:108790000A5210B5C1F3130140F2FF3341F48011C6
:1087A0009A4201DA002010BD40F233439A42A2F20D
:1087B000334203DC5242FFF7F8FC10BD904010BD7D
:1087C00000F0004230F000400AD0C10D01F56071A8
:1087D000C0F3160042EA0151C20840071143704736
:1087E000002001467047000030B5041E71F10004FE
:1087F00004DB4FF00044404264EB0101141E73F1AE
:10880000000405DB1C464FF00043524263EB0403B7
:108810008B4208BF824230BD30B5041E71F10004A6
:1088200004DB4FF00044404264EB0101141E73F17D
:10883000000405DB1C464FF00043524263EB040387
:10884000994208BF904230BD01F0004330B421F09E
:10885000004150EA010206D00A0DA2F56072C1F390
:108860001301002A02DC30BC00207047440F44EAA8
:10887000C104C100E01830BC00EBC25000F06DB87C
:10888000002801DBC0F10040002901DBC1F10041FB
:1088900081427047002801DBC0F10040002901DB64
:1088A000C1F100418842704730B50B4601460020B7
:1088B0002022012409E021FA02F59D4205D303FAA2
:1088C00002F5491B04FA02F52844151EA2F1010223
:1088D000F1DC30BD2DE9F05F0546002092469B4655
:1088E00088460646814640241BE0284641464746C6
:1088F0002246FFF75AFC53465A46C01A914110D3FC
:10890000114618462246FFF741FC2D1A67EB010875
:108910004F46224601200021FFF738FC17EB0009E3
:108920004E41201EA4F10104DFDC484631462A46B0
:108930004346BDE8F09F202A06DBCB17203A41FAD8
:1089400002F043EAE07306E041FA02F3D040C2F1DC
:10895000200291400843194670470029A8BF70477C
:10896000401C490008BF20F00100704710B4B0FA65
:1089700080FC00FA0CF050EA010404BF10BC704700
:1089800049B1CCF1200421FA04F411FA0CF118BF1A
:10899000012121430843A3EB0C01CB1D4FEA0061E9
:1089A0004FEA102042BF002010BC704700EBC350BC
:1089B00010440029A4BF10BC7047401C490008BFE8
:1089C00020F0010010BC704710B5141E73F10004B4
:1089D00008DA401C41F1000192185B411A4301D1B1
:1089E00020F0010010BD2DE9F04D92469B4611B1DB
:1089F000B1FA81F202E0B0FA80F220329046FFF73D
:108A0000C5FB04460F4640EA0A0041EA0B01534603
:108A10005A46084313D0114653EA010019D0C8F151
:108A200040025046FFF7C1FB05460E4650465946E8
:108A30004246FFF7ABFB084305D0012004E0204687
:108A40003946BDE8F08D0020054346EAE0762C4328
:108A500037430A986305E40AA0EB08000022FD0AE8
:108A600044EA47540A3002D500200146E9E70105EF
:108A700010196941DDE9084500196941BDE8F04D6B
:108A8000A2E7C1F30A52C1F3130140F2FF3341F4EC
:108A900080119A4202DA00200146704740F23343C7
:108AA0009A42A2F2334202DC5242FFF77EBBFFF74A
:108AB0006DBB0000064C074D06E0E06840F0010386
:108AC00094E8070098471034AC42F6D3FFF744FB14
:108AD000C4C70108E4C7010870B58C1810F8015B21
:108AE00015F0070301D110F8013B2A1106D110F847
:108AF000012B03E010F8016B01F8016B5B1EF9D14B
:108B00002B0705D40023521E0DD401F8013BFAE7D0
:108B100010F8013BCB1A921C03E013F8015B01F83B
:108B2000015B521EF9D5A142D8D3002070BD014689
:108B30000878704710B5214840792049C9788842A3
:108B40000DD01F48007850B9042003F081FD30B9E2
:108B500001201B49087004200CF0F8FF0CE01748B6
:108B600040791649C978884206D11548007801280D
:108B700002D1002012490870104880790F49097904
:108B800088420DD00F48007850B9032003F060FDF3
:108B900030B901200B49087005200CF0D7FF0CE01C
:108BA0000648807905490979884206D10548007848
:108BB000012802D100200349087010BDC4250020FF
:108BC000C4080020C508002010B51B48007830B14B
:108BD000012814D0022820D003282AD123E0032022
:108BE00003F036FD18B103201349087006E0042095
:108BF00003F02EFD10B102200F4908701AE0032087
:108C000003F026FD18B9042003F022FD08B101206D
:108C100000E00020084908700CE002F03FFB012052
:108C20000549087006E002F0FBFA012002490870CD
:108C300000E000BF00BF10BD3509002021B18268EF
:108C400042F00102826003E0826822F00102826049
:108C5000704721B1826842F48072826003E08268CA
:108C600022F4807282607047014600208A6802F018
:108C700004020AB1012000E00020704701460020F4
:108C80008A6802F008020AB1012000E00020704763
:108C900030B502460020002350680F4C20400D796B
:108CA0000C6844EA05242043506090680B4C204037
:108CB000D1E902542C434D7944EA450420439060A5
:108CC000D06A20F470000C7C641EE4B2234340EAB6
:108CD0000350D06230BD0000FFFEF0FFFDF7F1FF52
:108CE000F0B504460D4600200021092D11DDE06895
:108CF000A5F10A0606EB4607072606FA07F18843A0
:108D0000A5F10A0606EB460603FA06F10843E06001
:108D10000CE0206905EB4507072606FA07F18843B2
:108D200005EB450603FA06F108432061072A0FDA2E
:108D3000606B561E06EB86071F2606FA07F188436E
:108D4000561E06EB860605FA06F10843606322E02C
:108D50000D2A0FDA206BD61F06EB86071F2606FAB0
:108D600007F18843D61F06EB860605FA06F108438D
:108D7000206310E0E06AA2F10D0606EB86071F26CD
:108D800006FA07F18843A2F10D0606EB860605FAFE
:108D900006F10843E062F0BD816841F0080181609E
:108DA000704721B1826842F4A002826003E08268C9
:108DB00022F4A00282607047816841F00401816062
:108DC00070470000F8B505460E46002490208DF847
:108DD000000001208DF801008DF802608DF803502D
:108DE0000949086005F094F800BF08E01DF8040088
:108DF00005F0C8F80A2000F029F8601CC4B2042C61
:108E0000F4DB05F0A5F8F8BD9881214208B50121F1
:108E1000082007F025F9C020ADF8000003208DF8E8
:108E2000020010208DF803006946054803F0F0FEAB
:108E30000120044908600449C1F8980108BD0000F8
:108E4000000C01409C8121420080214200BF411E54
:108E500089B2081EFBD1704710B50B48007B10B9D2
:108E60000BF062F920B100200749C874012010BD41
:108E70000548C07C30B901200349C87407F066FA80
:108E8000014988600020F2E74809002000B591B050
:108E90000121084607F0B4F8012140F2112007F043
:108EA000DFF84FF4004007F09FF83920ADF840009C
:108EB00000208DF8430010A9374803F0A9FE0020D8
:108EC0000B900E904FF460200D9001208DF8310032
:108ED00004208DF83C0001208DF830000BA92F48AC
:108EE000FFF7D6FE052301220A212C48FFF7F8FEE2
:108EF000052302220D212948FFF7F2FE0523032254
:108F00000E212648FFF7ECFE052304220F212348FB
:108F1000FFF7E6FE21484C300090801506900020B7
:108F200004901F4801904FF48060079080200590C6
:108F300000200290042003902020089000200A9036
:108F40004FF4805009906946164802F0C7FE01218F
:108F5000144802F0B7FE01211048FFF77AFE012104
:108F60000E48FFF76BFE0D48FFF716FF00BF0B48DA
:108F7000FFF784FE0028FAD10848FFF71DFF00BF65
:108F80000648FFF771FE0028FAD101210348FFF7D8
:108F900008FF11B000BD0000001001400024014096
:108FA00060000020080002402DE9F04104460F4611
:108FB0000C200FF03DFF05463888288078686860EF
:108FC000206830B9012020726560AD602560BDE881
:108FD000F081266800E0B668B06861688842FAD11E
:108FE000B5602068A86000BFF1E7000070B502F02E
:108FF00075FB0E4909780E4A52F8210080470B494B
:1090000009780C4A52F82100804704460748007846
:1090100000EB4000084901EBC00050F824501DB19E
:109020002046A8470149087070BD000004260020B2
:109030006407002084070020A406002000200649C1
:10904000097819B90121044A117003E00021024A8C
:109050001170042070470000A1060020014601F0B5
:109060000F000A0902EB820200EB4200C0B2704717
:1090700010B5012007F004F8002007F001F810BD3A
:1090800010B5A2B0002441F204000C49A1F805007B
:10909000202048800A48007C401C0949087409A027
:1090A0000CF06CF801AA02A9044802F035FE002178
:1090B000094809F015FC22B010BD0000DE1F002099
:1090C0006421002073656E642043686172676520C7
:1090D000646174610A0D0000A005002010B51048FD
:1090E00090F86C00642804D1062003F0CBFA00202D
:1090F00010BD0B4A106F126F1169884720B91C20F0
:1091000003F0C0FA0020F3E7054A106F126F91696F
:10911000884710B903A00CF031F80120E8E70000FF
:10912000D8070020564355BDFBD6B9B3E4B5E70DCB
:109130000A00000010B5A2B0002441F209000A495B
:10914000A1F80500122048800848007C401C07490F
:10915000087407A00CF012F801AA02A9024802F054
:10916000DBFD22B010BD0000DE1F002064210020C6
:1091700053656E64204368617267696E6744617409
:1091800061200A0D0000000000B5A1B00020009091
:1091900041F203000E49A1F805000E4801780C4881
:1091A000817204200A4948800B48007C401C0A490F
:1091B00008740AA00BF0E2FF6A4601A9044802F015
:1091C000ABFD00210A4809F08BFB21B000BD000077
:1091D000DE1F00200C0200206421002073656E64F5
:1091E0002073746174652064617461200A0D00004D
:1091F0009805002010B5242003F00CFA0021034844
:1092000009F06EFB002002F063FA10BD1C2600205E
:1092100010B5A2B0002441F221001549A1F80500C3
:109220001448007DC8711348808A010A10480172F1
:1092300010484069010C0E4841720E484069000E0A
:109240000B498872042048800B48007C401C0A4966
:1092500008740AA00BF092FF01AA02A9044802F0C8
:109260005BFD04210248C01D0EF09EFB22B010BD24
:10927000DE1F0020981B0020642100200A0D736867
:10928000656E676A6979696E676461200A0D00001E
:1092900010B5A2B000244FF481500F49A1F8050089
:1092A0005520C871AA210C48017202200A49488041
:1092B0000A48007C401C0949087409A00BF05EFFB5
:1092C00001AA02A9044802F027FD02210248C01D9C
:1092D0000EF06AFB22B010BDDE1F002064210020CA
:1092E0004F54412041434B200A0D000010B5A2B05D
:1092F000002441F208001E49A1F805001D481EA1E6
:10930000096801601EA10968416019481949096886
:10931000C0F8071017494968C0F80B101548017AC2
:109320001348C17313480089010A11480174114898
:109330008068010C0E4841740E488068000E0C498C
:1093400088740C48017B0A48C1740D200849488084
:109350000D48007C401C0C4908740CA00BF00EFF5B
:1093600001AA02A9024802F0D7FC22B010BD0000F9
:10937000DE1F002096230020533230310000000011
:10938000574C494E470000006421002073656E640D
:1093900020626D732076657273696F6E0A0D00002E
:1093A0000648008A401C054908820846008AC828E9
:1093B00001DBAA2070470020FCE700000426002003
:1093C00010B501214FF0C05006F02AFE012005F033
:1093D00011FD10BDF0B503460C46FF25FF26151202
:1093E000D6B209E013F8010B80EA05010648405C9B
:1093F00080EA06050548465C201EA4F10107BCB2C0
:10940000F0D146EA0520F0BDA8BB0108A8BC0108C0
:1094100070B502460C46FF25FF2309E012F8010B48
:1094200080EA05010648405C80EA03050548435C84
:10943000201EA4F10106B4B2F0D143EA052070BDAC
:10944000A8BB0108A8BC010810B5022101A006F0C4
:1094500040FF10BD4154000010B50A2101A006F0E4
:1094600038FF10BD41542B53544154453D3F00003B
:1094700070B504460E462546288845F6A521884243
:1094800002D128460FF054FD70BD000030B589B000
:109490000446202101A8FEF7B1FE202101A8FEF715
:1094A000ADFE224606A101A80BF078FE01A8FEF74A
:1094B000C2FE0546294601A806F00BFF09B030BDE3
:1094C00041542B4E414D453D2573000010B50921F7
:1094D00001A006F0FEFE10BD41542B4E414D453D0E
:1094E0003F00000010B50D2101A006F0F2FE10BDF6
:1094F00041542B554152545F4346473D3F000000C5
:1095000010B50B2101A006F0E4FE10BD41542B560E
:109510004552494F4E3D3F0010B52548007801287F
:1095200045D124480078062837D2DFE800F0031739
:109530000D36202A072220A12148FEF783FE10B90C
:1095400002201C49087028E00A221EA11C48FEF7D0
:1095500079FE10B90120174908701EE01C4918480F
:10956000FEF757FE10B104201249087015E00B22D7
:1095700018A11348FEF766FE10B905200D490870C2
:109580000BE00F480B4948601548008808811448D3
:1095900001880B48FFF76CFF00BF00BF00200449A3
:1095A00008700F49088080210548FEF727FE10BD8E
:1095B000120200206421002041542B4F4B0D0A0061
:1095C000881C002041542B4F4B0D0A3033303300A0
:1095D0000817002041542B4F4B0D0A30310D0A0063
:1095E0001002002010B516480078072824D2DFE8C2
:1095F00000F0040A07230D1F220000F077FA1CE098
:1096000000F078FA19E000F031FA16E000F05CFAA8
:109610000C4890F8760018B900200949887006E0D7
:10962000084890F87600012801D10549887004E0C7
:1096300000F00AF801E000E000BF00BF10BD00002C
:1096400064210020F816002010B5594890F8A800B1
:10965000012808D15748007C0A2803DB0020544920
:1096600081F8A80010BD4FF47A7053490880514822
:10967000007C14280EDD4E4890F8760018B90020C2
:109680004C49887006E04A4890F87600012801D1DC
:10969000484988704748807807287AD2DFE800F088
:1096A00004070E666782830000F0B0F97DE000F0E9
:1096B0006DF900203E4981F8A80076E03E48018817
:1096C0003E4809F00DF901284FD13D480088401C63
:1096D0003B49088008460088092801DD00200880F1
:1096E0000021364809F0FCF83548008810B900F030
:1096F00021F93AE032480088012802D1FFF7C0FC86
:1097000033E02F480088022802D1FFF73DFD2CE00E
:109710002B480088032828D029480088042802D133
:1097200000F050F821E026480088052802D1FFF714
:10973000DDFD1AE022480088062802D1FFF7FAFC76
:1097400013E01F480088072802D10CF051FB0CE001
:109750001B480088082802D10CF0E4FA05E01848FC
:109760000088092801D10CF00BFB1EE01DE0114818
:10977000417C407C401C0F4A5074142911DD0020AC
:10978000114608700A4890F8760018B900208870D1
:1097900007E009E0064890F87600012801D1054964
:1097A000887002E001E000E000BF00BF00BF59E7A1
:1097B000F816002064210020840500208005002088
:1097C0007C05002010B5A2B000200190002441F2D9
:1097D00007004B49A1F805004A48808B4949C98BCD
:1097E000484342F2107190FBF1F084B24548007F8B
:1097F0004349C8714348808B011241480172414876
:10980000817F3F4841723F48C08B01123C488172C2
:10981000C4723C4890F8291039480173394890F8CF
:10982000281037484173202181735F21C173354867
:10983000C17E33480174334890F826103048417493
:109840003048C08C01122E4881742E48C17E2C48AD
:10985000C1742C48417A2A4801752A48B0F8090099
:109860000112274841752748C17A25488175254846
:10987000B0F80B0001122248C175224841782048F7
:1098800001762048B0F8010001121D4841761D48BC
:1098900041791B4881761B48B0F805000112184831
:1098A000C1761848C179164801771648817C14485A
:1098B00041771448408A010A11488177114890F88D
:1098C0002A100F48C1770F4890F82B100C4880F8E9
:1098D00020100DA00BF052FC1A200949488001AA63
:1098E00002A9074802F018FA0C48007C401C0B49FA
:1098F000087400210A4808F0F3FF22B010BD0000F0
:10990000DE1F0020D80D002073656E6420444344A0
:109910004320646174610A0D00000000642100208E
:10992000B805002070B504460D462946204606F0CD
:10993000C3FC70BD00B5A1B0002000900AA00BF0E0
:109940001DFC3A200E4948806A4601A90C4802F0E5
:10995000E3F90C48007C401C0A49087400210A48BD
:1099600008F0BEFF21B000BD73656E6420686561BC
:109970007274626561742064617461200A0D000074
:10998000DE1F0020642100209005002000B591B06A
:109990000020009040F6B831134808F0A1FF0128DC
:1099A0001FD141F201001149A1F8050010A00BF0F0
:1099B000E5FB0E48C01D1349CA6E0260096F416085
:1099C00011490A6882604968C160102007494880CF
:1099D0006A4601A9054802F09FF90021024808F0F3
:1099E0007FFF11B000BD00008C050020DE1F0020AD
:1099F00073656E64204C6F67696E20646174610DDD
:109A00000A000000F8160020A0BA010800B591B0C5
:109A10000020009041F288310C4808F061FF0128D5
:109A200011D100030A49A1F805000020488009A0CF
:109A30000BF0A4FB6A4601A9054802F06DF900216C
:109A4000024808F04DFF11B000BD0000880500205D
:109A5000DE1F002053656E6420526567697374656C
:109A600072656420646174610A0D000010B54FF4E2
:109A70007A71124808F034FF01281ED1104800788E
:109A800018B901200E49087013E00D48007801282C
:109A900006D10C48FFF7FAFC02200949087008E0DB
:109AA00007480078022804D1FFF710FD0020044980
:109AB00008700021014808F013FF10BD7405002054
:109AC000700500200817002010B540F6B831064890
:109AD00008F006FF012805D1FFF7BEFC002102486F
:109AE00008F0FEFE10BD00007805002010B5FFF75D
:109AF000ABFC10BD10B54FF47A710E4808F0F0FEC3
:109B0000012815D10C48007828B9FFF7F9FC01208D
:109B10000949087008E008480078012804D1FFF7D7
:109B2000E1FC0020044908700021024808F0D8FE3A
:109B300010BD00006C0500206B05002000BFFEE793
:109B400000B585B06A460021044800F0AEFE6946C3
:109B500000200DF0ABF905B000BD0000006400402E
:109B600010B54FF40071154800F05AFC01280DD1D2
:109B70001349124800F018FC012802D100200DF012
:109B800073FA4FF400710D4800F0E2F94FF4806170
:109B90000A4800F045FC01280ED10949891C0748F4
:109BA00000F002FC012802D100200DF083FA4FF4EE
:109BB0008061024800F0CCF910BD00000064004054
:109BC0000200F01010B50021194800F0A7FF04466C
:109BD000022C08D0012C00D100E000200246002118
:109BE00008460DF09FF90121114800F097FF044647
:109BF000022C08D0012C00D100E0002002460121F7
:109C000000200DF08FF90221094800F087FF04467B
:109C1000022C08D0012C00D100E0002002460221D5
:109C200000200DF07FF90121014800F091F910BDED
:109C30000064004000B589B006F0F9FC012109205C
:109C400006F00EFA0121480606F0EAF9012188061D
:109C500006F0E6F90021594800F0D6FD4FF4005017
:109C6000ADF8200003208DF8220018208DF8230085
:109C700008A9534802F0CCFF4FF48050ADF8200003
:109C800048208DF8230008A94D4802F0C1FF0020AC
:109C90008DF81A0001208DF81B0000208DF81C00A3
:109CA0008DF81D008DF81E0001208DF81F0000208A
:109CB0008DF8160001208DF8170008208DF8180087
:109CC00001208DF819000620ADF8140005A93B48C5
:109CD00000F03FFC3B48407BD0B10E208DF80E00D9
:109CE00000208DF80F0001208DF810000020ADF845
:109CF0000400ADF80600ADF80800ADF80A00012038
:109D0000ADF80C008DF8110001A800F0DFF903E0B8
:109D10002D49002000F033FB01221021274800F0DC
:109D20000FFC41208DF8000001208DF8010000207B
:109D30008DF8020001208DF80300684604F064FFEE
:109D4000012211461D4800F0FBFB012251021B4875
:109D500000F0F6FB01229102184800F0F1FB01220D
:109D6000D103164800F0ECFB0121144800F04CFD33
:109D70003F208DF8000001208DF8010000208DF8B3
:109D8000020001208DF80300684604F03DFF4220E8
:109D90008DF8000001208DF8010000208DF80200F0
:109DA00001208DF80300684604F02EFF06F041FC08
:109DB00006A00BF0E3F9002009B000BD00680040E8
:109DC000000C0140480900200C06002063616E2051
:109DD00032206F70656E210A0000000000B585B06A
:109DE000012009498873094806F0B3FC6A4601213D
:109DF000074800F05AFD9DF8090018B9694601208E
:109E00000DF054F805B000BD480900205837002077
:109E10000068004010B54FF400711F4800F000FBCF
:109E2000012810D11D491C4800F0BEFA012805D1B7
:109E30000DF01AF91949184800F06EF84FF4007146
:109E4000154800F085F84FF48061134800F0E8FAF7
:109E5000012820D11149891C0F4800F0A5FA0128DA
:109E600011D10F4948740846007C401C08740D4805
:109E700006F06FFC01200DF01DF90849891C064809
:109E800000F04AF802E00020054908744FF48061B0
:109E9000014800F05DF810BD006800400200F010BD
:109EA000480900206037002010B50021194800F053
:109EB00035FE0446022C08D0012C00D100E0002021
:109EC0000246002101200DF02DF80121114800F07B
:109ED00025FE0446022C08D0012C00D100E0002011
:109EE0000246012108460DF01DF80221094800F044
:109EF00015FE0446022C08D0012C00D100E0002001
:109F00000246022101200DF00DF80121014800F068
:109F10001FF810BD0068004000220C4B994202D18E
:109F20000023836111E0C1F3130201F000730BB150
:109F3000C2600AE001F080630BB1026105E001F04C
:109F400000630BB1826000E0426070477000F03047
:109F5000B1F5007F3AD00FDC202928D006DC01299A
:109F60001CD004291DD0082940D11DE0402921D052
:109F7000B1F5807F3AD126E0B1F5004F31D006DC53
:109F8000B1F5806F25D0B1F5006F2FD124E0B1F588
:109F9000803F12D0B1F5003F28D111E0154A826010
:109FA00025E00822C26022E01022C2601FE00822E1
:109FB00002611CE01022026119E00822426016E0F2
:109FC0001022426013E00422426010E0042242604A
:109FD0000DE0042242600AE0002282610422426015
:109FE00005E0002282610422426000E000BF00BF61
:109FF000704700000101010010B504460B4884427F
:10A0000009D10121480606F01BF800214FF000702D
:10A0100006F016F808E00121880606F011F8002184
:10A020004FF0806006F00CF810BD000000640040A6
:10A030002DE9F04104460D4617461E46ECB10020BE
:10A04000207220606060B5F5006F03D30420207299
:10A05000656002E000202072256006B127B900206B
:10A06000A0720220607208E000206072A672324680
:10A07000394604F10B00FEF7A8F8BDE8F0812DE9A0
:10A08000F04104460D4617461E46ECB100202072F2
:10A0900020606060B5F5006F03D304202072656016
:10A0A00002E000202072256006B127B90020A072CE
:10A0B0000220607208E000206072A67232463946C3
:10A0C00004F10B00FEF781F8BDE8F08110B5002126
:10A0D000837A012202FA03F13D4A126842F001023A
:10A0E0003B4B1A603A4A1C3212688A43384B1C3385
:10A0F0001A60027BCAB9364A0C3212688A43344B62
:10A100000C331A604288C38842EA0343304A403223
:10A11000847A42F834300288838842EA03432C4A26
:10A120004032847A02EBC4025360027B012A19D1C7
:10A13000274A0C3212680A43254B0C331A604288B6
:10A14000038842EA0343224A4032847A42F8343098
:10A15000C288838842EA03431D4A4032847A02EB74
:10A16000C4025360C27A3AB9194A121D12688A436E
:10A17000174B1B1D1A6006E0154A121D12680A4390
:10A18000134B1B1D1A60028932B9114A143212682E
:10A190008A430F4B14331A600289012A06D10C4AF4
:10A1A000143212680A430A4B14331A60427B012AA4
:10A1B00006D1074A1C3212680A43054B1C331A6049
:10A1C000034A126822F00102014B1A6010BD000020
:10A1D000006600402DE9FF4706460F46B9460024B9
:10A1E0004FF00108404600F0D9FB8DF80A800120AD
:10A1F0008DF80B008DF80C00ADF808008DF80D00FF
:10A2000000253EE0204604EBD0714910A4EB41014B
:10A21000491C012902D0022920D10FE056F835004F
:10A22000042101EBC000000CADF8000036F8350049
:10A2300001EBC00080B2ADF802000FE056F8350027
:10A24000042101EBC000000CADF8040036F8350025
:10A2500001EBC00080B2ADF8060000BF00BF641C77
:10A26000204604EBD0714910A4EB410141B9684686
:10A27000FFF72CFF9DF80A00401CC0B28DF80A00C1
:10A280006D1C4D45BEDB204604EBD0714910A4EB9C
:10A29000410111B16846FFF719FFBDE8FF872DE9BD
:10A2A000FF4706460F46B94600244FF001084046D6
:10A2B00000F074FB8DF80A8001208DF80B0000205F
:10A2C0008DF80C000120ADF808008DF80D00002578
:10A2D00047E02046E11704EB91718910A4EB81015E
:10A2E000491C012906D002290DD0032914D00429C4
:10A2F00024D11AE056F835004FF6FF7101EA4010FC
:10A30000ADF800001AE056F835004FF6FF7101EA8B
:10A310004010ADF8020011E056F835004FF6FF711D
:10A3200001EA4010ADF8040008E056F835004FF699
:10A33000FF7101EA4010ADF8060000BF00BF641CC9
:10A34000E11704EB91718910A4EB810141B96846D2
:10A35000FFF7BCFE9DF80A00401CC0B28DF80A0051
:10A360006D1C4D45B5DBE11704EB91718910A4EB31
:10A37000810111B16846FFF7A9FEBDE8FF8770B5FE
:10A3800004460D46112624B931462846FFF787FFBB
:10A3900008E0012C04D131462846FFF71BFF01E0FD
:10A3A000002070BD0120FCE710B50246002001F43A
:10A3B000700343B19369C1F3130423400BB101202F
:10A3C0002DE000202BE001F0807343B15368C1F30E
:10A3D000130423400BB1012021E000201FE001F015
:10A3E000006343B19368C1F3130423400BB1012010
:10A3F00015E0002013E001F0007343B1D368C1F30E
:10A40000130423400BB1012009E0002007E0136989
:10A41000C1F3130423400BB1012000E0002010BD64
:10A4200070B504460D46002660692840002871D0AA
:10A43000B5F5807F5CD010DC082D35D006DC012D11
:10A4400020D0022D24D0042D72D127E0102D31D040
:10A45000202D35D0402D6BD138E0B5F5004F60D0C0
:10A4600009DCB5F5007F49D0B5F5806F4CD0B5F566
:10A47000006F5DD14FE0B5F5803F2DD0B5F5003FC1
:10A4800056D12FE0A0682D4901F080F8064651E032
:10A49000E068032101F07AF806464BE0E068082105
:10A4A00001F074F8064645E0E068102101F06EF80E
:10A4B00006463FE02069032101F068F8064639E0CE
:10A4C0002069082101F062F8064633E02069102176
:10A4D00001F05CF806462DE06068082101F056F8AE
:10A4E000064627E06068102101F050F8064621E09A
:10A4F000A069012101F04AF806461BE0A06902218B
:10A5000001F044F8064615E0A069042101F03EF888
:10A5100006460FE00FE0A069702101F037F806460B
:10A5200008E06068042101F031F8064602E0FFE728
:10A53000002600BF00E00026304670BD010101008A
:10A540001AB143690B43436102E043698B434361A2
:10A55000704730B5024600200023146824F002043E
:10A560001460146844F00104146000E05B1C54683B
:10A5700004F001041CB94FF6FF74A342F6D15468ED
:10A5800004F001040CB900206CE08C79012C04D19A
:10A59000146844F08004146003E0146824F080041C
:10A5A0001460CC79012C04D1146844F04004146088
:10A5B00003E0146824F0400414600C7A012C04D1E8
:10A5C000146844F02004146003E0146824F02004AC
:10A5D00014604C7A012C04D1146844F01004146007
:10A5E00003E0146824F0100414608C7A012C04D168
:10A5F000146844F00804146003E0146824F00804AC
:10A600001460CC7A012C04D1146844F00404146062
:10A6100003E0146824F0040414608C78A407CD7857
:10A6200044EA05640D7944EA05444D7944EA055449
:10A630000D886D1E2C43D461146824F0010414604D
:10A64000002300E05B1C546804F001041CB14FF6C9
:10A65000FF74A342F6D1546804F001040CB1002049
:10A6600000E0012030BD2DE9F04107460C461546BB
:10A67000264616B100212846B047BDE8F08170B5E6
:10A6800006460C461546E9B2E0B20DF011FE70BD6B
:10A6900000B589B00121052005F0E2FC0121480642
:10A6A00005F0BEFC0021524800F0AEF84FF4805097
:10A6B000ADF8200003208DF8220018208DF823002B
:10A6C00008A94C4802F0A4FA4FF40060ADF820004D
:10A6D00048208DF8230008A9464802F099FA002086
:10A6E0008DF81A0001208DF81B0000208DF81C0049
:10A6F0008DF81D008DF81E008DF81F008DF81600D6
:10A700008DF817000C208DF8180001208DF8190025
:10A710000920ADF8140005A93548FFF71AFF0020FD
:10A720008DF80E008DF80F0001208DF8100000202C
:10A73000ADF80400ADF80600ADF80800ADF80A0069
:10A74000ADF80C0001208DF8110001A8FFF7BEFC48
:10A75000012202212648FFF7F3FE14208DF80000A5
:10A7600001208DF8010000208DF8020001208DF8F5
:10A770000300684604F048FA012211461C48FFF71E
:10A78000DFFE012251021A48FFF7DAFE0122910290
:10A790001748FFF7D5FE0122D1031548FFF7D0FE79
:10A7A0000121134800F030F813208DF8000001203B
:10A7B0008DF8010000208DF8020001208DF80300C3
:10A7C000684604F021FA16208DF8000001208DF86B
:10A7D000010000208DF8020001208DF8030068467A
:10A7E00004F012FA04A00AF0C9FC002009B000BD70
:10A7F000006400400008014063616E2031206F70EA
:10A80000656E210A0000000010B502460B460020CC
:10A810004FF6FF71BBB9146824F0020444F0010440
:10A82000146000E0491E546804F00304012C01D0B8
:10A830000029F7D1546804F00304012C01D0002052
:10A8400032E0012030E0012B13D1146824F003041E
:10A85000146000E0491E546804F003040CB10029A0
:10A86000F8D1546804F003040CB100201CE001206E
:10A870001AE0022B17D1146824F0010444F00204FA
:10A88000146000E0491E546804F00304022C01D057
:10A890000029F7D1546804F00304022C01D00020F1
:10A8A00002E0012000E0002010BD10B500F5D873D3
:10A8B00003EB01131B6803F004031372137A53B9FB
:10A8C00000F5D87303EB01131B6840F2FF7404EA30
:10A8D0005353136009E000F5D87303EB01131B68B1
:10A8E0006FF0604404EAD303536000F5D87303EBC0
:10A8F00001131B6803F00203537200F5D87303EBD6
:10A9000001135B6803F00F03937200F5D87303EB38
:10A9100001135B681B0AD37400F5D87303EB0113B2
:10A920009B68D37200F5D87303EB01139B681C0A74
:10A93000147300F5D87303EB01139B681C0C54735C
:10A9400000F5D87303EB01139B681B0E937300F59E
:10A95000D87303EB0113DB68D37300F5D87303EBF3
:10A960000113DB681C0A147400F5D87303EB0113A0
:10A97000DB681C0C547400F5D87303EB0113DB681F
:10A980001B0E937421B9C36843F02003C36003E036
:10A99000036943F02003036110BD00000B490968FF
:10A9A00041F00101094A11601146096843F60E722F
:10A9B0009143064A11601146096841EA002111607D
:10A9C0001146096821F001011160704700660040DE
:10A9D00010B502460020504B9A420CD10B68B3F5DB
:10A9E000457F00D120E00B68B3F57A7F01D10120CB
:10A9F0001AE0022018E0936803F08063B3F1806FDF
:10AA000001D1002010E0936803F00063B3F1006F00
:10AA100001D1012008E0936803F08053B3F1805F17
:10AA200001D1022000E00420042874D002F5C07394
:10AA300003EB00131B6803F0010402F5C07303EB82
:10AA400000131C600B7A7BB94B7A0C8843EA4453A1
:10AA500002F5C07404EB00142468234302F5C074AB
:10AA600004EB0014236010E00B7A4C6843EAC40343
:10AA70004C7A234302F5C07404EB0014246823438A
:10AA800002F5C07404EB001423608B7A03F00F030B
:10AA90008B7202F5C07303EB00135B6823F00F04A5
:10AAA00002F5C07303EB00135C6002F5C07303EBA7
:10AAB00000135B688C7A234302F5C07404EB001426
:10AAC00063608B7B1C064B7B44EA03440B7B44EAAC
:10AAD0000323CC7A234302F5C07404EB0014A36073
:10AAE0008B7C1C064B7C44EA03440B7C44EA032326
:10AAF000CC7B234302F5C07404EB0014E36002F541
:10AB0000C07303EB00131B6843F0010402F5C0732C
:10AB100003EB00131C6010BD0068004010B5024636
:10AB2000002321B1012907D002290FD109E0906843
:10AB30001D4C00EA04030BE090681C4C00EA04037F
:10AB400006E090681A4C00EA040301E0002300BF0D
:10AB500000BF184C181BA34216D007DC83B16FF05E
:10AB60008060184470B1022818D111E0B0F5007F60
:10AB700010D0114C204448B1B0F5003F0ED10BE08D
:10AB800002230DE000230BE0002309E0002307E08F
:10AB9000012305E0012303E0012301E0002300BFBE
:10ABA00000BFD8B210BD000003000004000300087D
:10ABB00000000310000100080001FFF770B51D48F8
:10ABC000858884881C480068E8B11C4800683C21DE
:10ABD000B0FBF1F01949086008460068C000184948
:10ABE000086008460068FDF793FD06461549FDF725
:10ABF000C0FB1549086000200F4908600F49086034
:10AC00000F49086014E0114800683C280AD20B483C
:10AC100000682044094908600C480068401C0B4942
:10AC2000086005E000200949086001200249086029
:10AC300070BD0000600000209800002090000020FF
:10AC40009400002000401C46880D00209C0000203D
:10AC500010B5054890F8210020B9292001F012FD17
:10AC6000002010BD0120FCE7200E002030B5034677
:10AC70000C46002118785D7800EB0520184DA5F8EA
:10AC80001B009878DD7800EB052001B2B1F57A6FF2
:10AC900002DDA1F57A6001E0C1F57A6001B2104DE4
:10ACA000A5F81D100A2906DB2846B0F81D000D4D39
:10ACB000A5F8070003E000200A4DA5F80700187961
:10ACC0005D7900EB0520064DA5F81F002846B0F879
:10ACD0001F00A5F81F00987985F82100012030BDDC
:10ACE000200E00209B0E002010B503461C7807485C
:10ACF00080F827405C7880F828409C7880F82940CC
:10AD0000DC7880F82A40012010BD0000200E0020D1
:10AD100070B505460C461646032C00DD032422467A
:10AD200029460248FDF751FA012070BD200E00208F
:10AD300030B503460C46002118785D7840EA0520BE
:10AD4000144D68829878DD7840EA0520114DA8827C
:10AD500018795D7940EA052001B2B1F57A6F02DD1C
:10AD6000A1F57A6001E0C1F57A6001B2094DE9828E
:10AD70009879DD7940EA052001B2B1F57A6F02DDFC
:10AD8000A1F57A6001E0C1F57A6001B2014D298335
:10AD9000012030BD200E002010B50346082900DD3B
:10ADA000082118780A4CE070587820719C7808487F
:10ADB0004471DC7884711C79C4715879044C207218
:10ADC0009C7903484472DC798472012010BD000034
:10ADD000200E002010B503461878024CA076012002
:10ADE00010BD0000200E002010B503461879074C56
:10ADF00084F834005C79054880F835409C7980F807
:10AE00003640DC7980F83740012010BD200E00204C
:10AE100010B503461C78074880F823405C7880F81A
:10AE200024409C7880F82540DC7880F8264001207A
:10AE300010BD0000200E002030B503460C4615461C
:10AE4000082C00DD08241878FEF708F91449C872A8
:10AE50005878FEF703F9124908739878FEF7FEF860
:10AE60000F494873D878FEF7F9F80D4988731879B7
:10AE7000FEF7F4F80A49C8735879FEF7EFF8084965
:10AE800008749879FEF7EAF80549487405480B31CB
:10AE90000A6802608A88828089798171012030BDC8
:10AEA000200E0020150E002010B5044608A00AF060
:10AEB00065F900F0B5F900BF01200749C8710748DE
:10AEC00003F0BBFD00BF064803F0B7FD012010BD35
:10AED00054310D0A00000000C4250020AC0A0020F7
:10AEE000E80A002010B5044602A00AF047F9022043
:10AEF00010BD00005431300D0A00000010B50446AA
:10AF000002A00AF03BF9062010BD00005431310DBB
:10AF10000A00000010B5044602A00AF02FF906202E
:10AF200010BD00005431320D0A00000010B5044677
:10AF300004A00AF023F903F0F7FE00F097F90020CF
:10AF400010BD00005431330D0A00000010B5044656
:10AF500003A00AF013F900F089F9012010BD0000E8
:10AF60005431340D0A00000010B5044608A00AF060
:10AF700005F900BF012008490872084803F05DFD8B
:10AF800000F068F900BF064803F02CFD072010BD53
:10AF90005431350D0A000000C4250020D40A0020D9
:10AFA000E80A002010B5044608A00AF0E7F800BF40
:10AFB000002008490872084803F014FD00200749E2
:10AFC0000870074908700749087010BD5431360DE4
:10AFD0000A000000C4250020D40A0020AD00002093
:10AFE000AC000020480C002010B5044602A00AF076
:10AFF000C5F8022010BD000054320D0A0000000008
:10B0000010B5044602A00AF0B9F8032010BD0000F4
:10B0100054330D0A0000000010B504460020044916
:10B02000C874088203A00AF0A9F8042010BD00002B
:10B030000426002054340D0A0000000010B5044618
:10B0400002A00AF09BF8052010BD000054350D0A3F
:10B050000000000010B5044602A00AF08FF8062098
:10B0600010BD000054360D0A0000000010B5044663
:10B0700009A00AF083F800200949487109490875B8
:10B0800000F0F4F803F050FE00F0E4F800BF0648CA
:10B0900003F0A8FC002010BD54370D0A000000008A
:10B0A000AC25002004260020E80A002010B5044644
:10B0B00002A00AF063F8022010BD000054380D0A07
:10B0C0000000000010B5044602A00AF057F8022064
:10B0D00010BD000054390D0A0000000010B52520F5
:10B0E00001F098FA0021034807F0FAFB012000F074
:10B0F000EFFA10BD2026002010B52248406A00F06B
:10B10000004018B120A00AF039F834E01D48406A28
:10B1100000F0804018B120A00AF030F82BE0194868
:10B12000406A00F0005018B120A00AF027F822E091
:10B130001448406A00F0805018B121A00AF01EF8AF
:10B1400019E01048406A00F0006018B11FA00AF032
:10B1500015F810E00B48406A00F0806018B11FA09D
:10B160000AF00CF807E00748406A00F0007010B1E0
:10B170001DA00AF003F80348406A40F080700149BE
:10B18000486210BD00100240B5CDB9A6BAC4B8B42B
:10B19000CEBB0D0A00000000B4B0BFDABFB4C3C517
:10B1A000B9B7B8B4CEBB0D0A00000000B6C0C1A24A
:10B1B000BFB4C3C5B9B7B8B4CEBB0D0A0000000018
:10B1C000C8EDBCFEB8B4CEBB0D0A0000C9CFB5E7D0
:10B1D0002FB5F4B5E7B8B4CEBB0D0A00D2FDBDC59E
:10B1E000B8B4CEBB0D0A0000424F52B8B4CEBB0D6E
:10B1F0000A00000010B5084803F0F4FB012000F03D
:10B200007CFE064803F019FC4FF4FA7000F075FE5E
:10B21000024803F0E7FB10BD880B00209C0B0020C8
:10B2200010B503F00DFB642000F067FE03F020FB77
:10B2300001200349487103A009F0A0FF10BD0000E0
:10B24000C4250020434C4F53455F41435265616C18
:10B25000790D0A0010B500200249C871024803F0B8
:10B26000C1FB10BDC4250020AC0A002010B5002091
:10B270000449887104A009F081FF074803F0B2FB7C
:10B2800010BD0000C4250020434C4F53455F44438C
:10B290005265616C790D0A00840A002010B5002007
:10B2A0000449887104A009F069FF074803F09AFB7C
:10B2B00010BD0000C4250020434C4F53455F44435C
:10B2C0005265616C790D0A00840A002010B50020D7
:10B2D0000449887104A009F051FF074803F082FB7C
:10B2E00010BD0000C4250020434C4F53455F44432C
:10B2F0005265616C790D0A00840A0020F0B504469D
:10B300000D462946204600F009F80746615D681C95
:10B31000205C41EA002686EA0700F0BD70B50246CF
:10B320004FF6FF7048F2050517E0491E12F8014B71
:10B3300080EA042000230EE000F400462EB14FF610
:10B34000FF7606EA4000684003E04FF6FF7606EA23
:10B3500040005E1CF3B2082BEEDB0029E5D170BD86
:10B3600000BF00BF0C4A126F128802EB820252002B
:10B37000094BB3F8463092FBF3F0074AB2F8482085
:10B38000A2F57A6200EB8003A2EB430211B2024AFB
:10B39000126F518070470000D80700200020012064
:10B3A0007047000010B50E48007D18B101200D490E
:10B3B000087002E000200B490870062001F048F9EF
:10B3C00040B907480078062807D100BF064803F0B7
:10B3D0001EFB10B90220034908700248007810BD16
:10B3E000042600209C060020380B002001460A8815
:10B3F000322A01DC012070470020FCE710B500BFB5
:10B400000648C08F0649898A884204DA282001F05C
:10B4100039F9002010BD0120FCE70000D80700200A
:10B42000200E002010B52048007920B1012807D057
:10B4300002280DD108E011211C4801F04BFB07E068
:10B440001A4801F079FB03E0112001F085FB00BFF1
:10B4500000BF3221164807F043FA012805D10AF04F
:10B460004FFE0021124807F03BFA124890F83800CE
:10B4700000F01000B0B101200F4908750D48806B35
:10B4800020F010000B498863FA210948083007F0C2
:10B4900027FA012806D10BF083F90021044808306F
:10B4A00007F01EFA10BD0000AC2500200D63010856
:10B4B000E8250020200E00200426002010B52C488E
:10B4C0000088401C80B22A4908800A2803DB00203B
:10B4D000088001F029FF274880880012264981F85A
:10B4E000E80024480179244880F8E910214880794F
:10B4F000214981F8F8001F48C1791F4880F8F910E8
:10B500001E480088401C80B21C49088064281DDB4E
:10B51000002008801A4800781A4991F828108842BB
:10B5200014D0184890F828001549087008211448CC
:10B53000FFF7F4FE84B212490C72211210484172D6
:10B5400000230A220146104800F088FF0D48407889
:10B5500001280CD10B488078012808D10020094926
:10B560004870887002F0B4FB01200649487110BD94
:10B570008C0C0020883800208C3700208A0C00209A
:10B58000BE47002068470020C84700200246002030
:10B5900002EA01030BB1012000E000207047000027
:10B5A000002003490978C1F3800101B101207047EF
:10B5B00088380020002003490978C1F3400101B117
:10B5C000012070478838002010B5034600202AB1BA
:10B5D0008B4201D0012006E0002004E08B4201D123
:10B5E000012000E0002010BD00200249097A01B1CD
:10B5F000012070478838002001460020012901D031
:10B60000032900D10120704701460020012905D0FF
:10B61000022903D0042901D00A2900D10120704752
:10B620000146002001F0800202B901207047024665
:10B6300000208A4200D1012070470020012070477D
:10B6400070B500201649086016490870002512E000
:10B6500005EBC501144800EB410410212046FCF71E
:10B66000CDFD10212046FFF759FE86B22674311217
:10B670006174681CC5B2122DEADB4FF4A2720A494C
:10B680000A48FCF7A2FD00234FF4A27206490848BD
:10B6900000F0E4FE00F00EF800F010F870BD0000BD
:10B6A000740C00207C0C0020A8380020EC3900200D
:10B6B0005148002010B508F021FD10BD00200249BE
:10B6C00008800249088070477E0C0020800C002012
:10B6D000012201490A5470472426002001207047A6
:10B6E00010B5044908698047022801D1012010BD26
:10B6F0000020FCE76C00002070B50521AB4805F088
:10B7000015F828B10020AA490873A84805F021F8C7
:10B710000521A648083005F009F830B10020A449F9
:10B720008873A248083005F014F805219F481030AE
:10B7300004F0FCFF30B100209D4908749B48103094
:10B7400005F007F89B49C86880470646FDF738F8BA
:10B7500004460022984BFDF747F807D22A2000F054
:10B7600077FF18B92A2000F08DFF0EE09149C868D4
:10B77000804704469149FDF78DF806D22A2000F053
:10B7800067FF10B12A2000F045FF8A49C86880474A
:10B790000646FDF715F804460022894BFDF73CF8F4
:10B7A00007D2322000F054FF18B9322000F06AFFAF
:10B7B0000FE08049C868804704464FF08341FDF799
:10B7C0005FF806D2322000F043FF10B1322000F0C3
:10B7D00021FF7C4890F84C00C0F30100032802D1FF
:10B7E0002E2000F04FFF7748406CC0F381600328A3
:10B7F00002D10B2000F046FF7248406CC0F301708C
:10B80000032802D12B2000F03DFF6E48406C800FD2
:10B81000032802D12C2000F035FF6A48406CC0F3A9
:10B820000140032802D12D2000F02CFF6548406C18
:10B83000C0F38150032802D10C2000F023FF61489F
:10B8400090F84400C0F30000012802D10D2000F060
:10B8500019FF5C48B0F84400C0F38130032802D1DE
:10B860000E2000F00FFF574890F84400C0F380000E
:10B87000012802D10F2000F005FF524890F8440043
:10B88000C0F3C000012802D1102000F0FBFE4D489B
:10B8900090F84400C0F30010012802D1112000F0FC
:10B8A000F1FE484890F84400C0F34010012802D14E
:10B8B000122000F0E7FE434890F84400C0F38110E6
:10B8C000032802D1132000F0DDFE3E48006CC0F3D7
:10B8D0008060012802D1142000F0D4FE3948006CA9
:10B8E000C0F30060012802D1152000F0CBFE3548DE
:10B8F000006CC0F34060012802D1162000F0C2FEA7
:10B900003048006CC0F30070012802D1172000F00D
:10B91000B9FE2C48006CC00F012802D1182000F09D
:10B92000B1FE2848006CC0F34040012802D1192024
:10B9300000F0A8FE2348006CC0F30150032802D198
:10B940001A2000F09FFE1F48B0F84000C0F3C0204E
:10B95000012802D11B2000F095FE1A4890F85C00E7
:10B96000C0F38000012802D11D2000F08BFE154895
:10B9700090F85C00C0F3C000012802D11E2000F046
:10B9800081FE104890F85C00C0F34010012802D1FD
:10B990001F2000F077FE0B4890F85C00C0F3C01049
:10B9A000012802D1202000F06DFE70BD503700202C
:10B9B000480900206C0000200000214000001041D8
:10B9C000008030403025002070B51F491F4800F02E
:10B9D0009FFF04461E491D480C3000F099FF0546A4
:10B9E0001B481D38B0F81D00002806DD012C04D1CD
:10B9F000012000F047FE002070BD15481D38B0F84A
:10BA00001D00B0F5A07F0EDD032D0CD103211148E0
:10BA100004F08CFE38B1052000F034FE0D4804F02F
:10BA200098FE0020E8E70B4804F093FE032000F0A6
:10BA30000FFE08B10020DFE7312000F009FE08B159
:10BA40000020D9E70120D7E7940D002040260020F0
:10BA50003D0E00204037002010B52A2000F0F8FDF0
:10BA600000B110BD33494868804755280BDB3420AE
:10BA700000F008FE2F4948688047642813DB302017
:10BA800000F000FE0FE02B49486880475A280ADC86
:10BA9000302000F0BFFD274948688047502802DC6D
:10BAA000342000F0B7FD244890F9000055280BDB46
:10BAB000332000F0E7FD204890F90000692813DBEF
:10BAC000312000F0DFFD0FE01B4890F900005F28F7
:10BAD0000ADC312000F09EFD174890F90000502844
:10BAE00002DC332000F096FD1348007A88B111493A
:10BAF00008681249FCF7C4FE0BD20221104804F07A
:10BB000015FE30B1352000F0BDFD0D4804F021FEDA
:10BB10000EE00948007A58B1064908680749FCF761
:10BB2000B9FE05D2352000F075FD054804F011FE80
:10BB300000BF96E76C000020C425002000002041D3
:10BB40006837002010B5002415480078002805DB70
:10BB500013480078042801DC012408E0104800782C
:10BB6000052803D00E480078072800D102240320BE
:10BB700000F06EFD88B9042000F06AFD68B930203D
:10BB800000F066FD48B9312000F062FD28B9054893
:10BB9000407810B90348807800B10324204610BDD6
:10BBA00004260020C425002010B541F288310F483A
:10BBB00006F096FE012807D1252000F063FD012044
:10BBC00005F0E4F8002010BD41F288310748001F5D
:10BBD00006F086FE012807D1242000F053FD002046
:10BBE00005F0D4F80020EEE70120ECE72026002045
:10BBF00001460878704700002DE9FC4701A9294853
:10BC000000F014FCDFF8A090002420E0274931F870
:10BC1000140001F0E5FA0546FF2D16D0244830F84F
:10BC2000150000EB0908234830F81460224830F86A
:10BC300014000199471831463846FFF75FFB20B9D9
:10BC4000324639464046FCF7C0FA601CC4B2092CA3
:10BC5000DCDB08F0C3FC694612480A3800F0E6FB5A
:10BC600008210098FFF74AFB98B90098007813491B
:10BC7000087008460078124981F82800084690F8B4
:10BC8000280003280CDB0A2081F829000120C87055
:10BC900006E000200A4981F82900C87081F82800D0
:10BCA000BDE8FC87D24700208C3700207CC001080B
:10BCB000E4BF01086AC0010858C00108BE4700205F
:10BCC0006847002021B1026842F00102026004E0EE
:10BCD00002684FF6FE731A400260704710B50022EA
:10BCE000026847F6F0739A430C6A8B6823430C6929
:10BCF00023434C6923438C692343CC6923434C6A17
:10BD000023438C6A23431A430260CB6843600B6869
:10BD100083604B68C36010BD2DE9F04706460C46B2
:10BD200092460025A946A84606B114B90020BDE8F0
:10BD3000F087708819301FFA80F8A5222846691C00
:10BD4000CDB222545A222846691CCDB2225428462C
:10BD5000691CCDB204F800804FEA18222846691CFD
:10BD6000CDB2225420222846691CCDB2225460193B
:10BD700010221849FCF729FA05F11000C5B27279B2
:10BD80002846691CCDB22254B6F80500020A28469E
:10BD9000691CCDB222547088022807DB72886019B2
:10BDA000F11DFCF712FAB0782844C5B229462046A6
:10BDB000FDF72EFB07462846691CCDB227543A0AE8
:10BDC0002846691CCDB2225429462046FDF7AAFD1B
:10BDD0000120ACE7F816002010B51948007820B112
:10BDE00001280BD0022827D117E01648407B08B164
:10BDF000012000E00020124908701EE000201149D7
:10BE000088740846407B08B1012000E002200C49FC
:10BE100008700D4804F09DFC0FE003210A4804F06F
:10BE200085FC40B10020064908700120054988744E
:10BE3000054804F08EFC00E000BF00BF10BD00000C
:10BE400034090020480900207037002038B56946C1
:10BE5000224800F0EBFA1225002432E0A91E04EB80
:10BE6000C402009B03EB4200FFF748FAC8B904EB99
:10BE7000C402009B03EB420104EBC403184A02EB2B
:10BE800043002A46FCF7A1F904EBC402009B03EB34
:10BE9000420104EBC402134B03EB42002A46FCF7B9
:10BEA00094F904EBC4010E4810F81100092806D1DA
:10BEB0000D4800680121A14008430B490860601C3F
:10BEC000C4B2122CCADB4FF0FF3008490860084AA0
:10BED0000849034805F090F838BD0000514800209B
:10BEE000A8380020EC390020740C0020780C0020C9
:10BEF0007C0C0020303B0020704710B5044606E063
:10BF0000142009F087F802F08BF9601E84B2002C2F
:10BF1000F6DC10BD2DE9F84F83464FF0000A0020F3
:10BF20000090584601F070F98046B8F1FF0F29D013
:10BF3000584601F055F90546FF2D23D01248445DBF
:10BF4000DFF84890124830F8150000EB090621464A
:10BF50003046FFF7E3F987B23755641C3812305585
:10BF6000641C0C4830F818100B4801EB000ABAF1B9
:10BF7000000F05D0002322463146504600F06EFAED
:10BF800008F02CFBBDE8F88F0AC001088C370020B0
:10BF9000E4BF010858C00108D247002070B506462A
:10BFA000DDE90445012070BD70B505460C46104E14
:10BFB00005EBC5010F4800EB4103122D00DB70BDFE
:10BFC0001878A04211D0092C0FD1184605F006F8B8
:10BFD000587820B93078401C307030785870587BD1
:10BFE000FF2802D0587B401C58731C7000BFE6E746
:10BFF0007C0C0020A8380020416170470161704727
:10C00000533530385F444355323430312DE9FC4FDD
:10C0100082460F4615461C464FF00008012001904D
:10C0200000200090DFF878B059212278501C207051
:10C03000A9542178481C207005F801A06A46594689
:10C04000384604F0D9FF00BF23E03BF818004FEA60
:10C050002029144850F82960C6F307412278501C63
:10C060002070A954C6F307212278501C2070A954CF
:10C070002278501C2070AE5409EBC90007EB400039
:10C0800041782278501C2070A95408F1010000F07A
:10C09000FF089DF800008045D7DB0020BDE8FC8F3D
:10C0A000303B002074BF01082DE9FF4781469046D0
:10C0B0001F46DDE90C5400264FF0010A5921227871
:10C0C000501C2070A9542178481C207005F801905C
:10C0D00000BF4AE0019820F07F40274951F8261020
:10C0E000884240D19DF806102278501C2070A95437
:10C0F0009DF805102278501C2070A9549DF804105A
:10C100002278501C2070A95406EBC60017F81010B6
:10C110002278501C2070A954B8F1010F03D0B8F157
:10C12000FF0F00D023E04FF0000A06EBC60007EB3C
:10C130004000407B00B91AE001212278501C207099
:10C14000A95408212278501C2070A95406EBC6027D
:10C1500007EB4202911C2278501904F0B9FE2178B5
:10C160000844207003E0701CC6B2122EB2DB00BF80
:10C17000504604B0BDE8F08774BF010800B5A6487A
:10C180000078C0F3001038B1A448006820F0200007
:10C190002030A249086005E0A048006820F0200097
:10C1A0009E4908609C480078C0F3401038B19B4815
:10C1B000006820F0400040309849086005E097484A
:10C1C000006820F040009549086093480078C0F36B
:10C1D000801038B19148006820F0800080308F498D
:10C1E000086005E08D48006820F080008B490860F9
:10C1F00089480078C00940B18848006820F4807000
:10C2000000F580708549086005E08448006820F4E6
:10C210008070824908608048407800F0010040B199
:10C220007E48006820F4007000F500707B490860CB
:10C2300005E07A48006820F4007078490860764884
:10C240004078C0F3400040B17448006820F480603A
:10C2500000F580607149086005E07048006820F4CE
:10C2600080606E4908606C484078C0F3800040B13F
:10C270006A48006820F4006000F5006067490860C3
:10C2800005E06648006820F4006064490860624880
:10C290004078C0F3C00040B16048006820F480508E
:10C2A00000F580505D49086005E05C48006820F4B6
:10C2B00080505A49086058484078C0F3001040B197
:10C2C0005648006820F4005000F5005053490860BB
:10C2D00005E05248006820F40050504908604E487C
:10C2E0004078C0F3401040B14C48006820F48040D2
:10C2F00000F580404949086005E04848006820F49E
:10C3000080404649086044484078C0F3801040B1FE
:10C310004248006820F4004000F500403F490860B2
:10C3200005E03E48006820F400403C4908603A4877
:10C330004078C00940B13948006820F4803000F5E9
:10C3400080303649086005E03448006820F48030C9
:10C35000324908603048807800F0010040B12F4831
:10C36000006820F4003000F500302C49086005E03A
:10C370002A48006820F4003028490860FFF734F9A3
:10C3800058B12548007A08280DDB2448006820F0C1
:10C39000100010302149086005E02048006820F0B6
:10C3A00010001E490860FFF71FF940B9FFF7F8F8C1
:10C3B00028B9FFF7FFF810B91948407B28B10020D1
:10C3C000184908801849088000BD16480088401C9C
:10C3D00080B214490880C82809DD1048006820F0A0
:10C3E0000100401C0D49086000200E4908800E48DD
:10C3F0000088401C80B20C490880B0F5967F09DDAA
:10C400000648006820F00200801C044908600020F3
:10C410000549088000BFD7E788380020740C002049
:10C42000480900207E0C0020800C002002460A48AB
:10C43000904201D108600DE007487F38904201D159
:10C44000086007E004488938904201D1086001E0A3
:10C45000002070470120FCE7514800202DE9F04101
:10C4600004460D4616461F463B46324629462046A0
:10C470000EF066FF0120BDE8F081000010B502A0BB
:10C4800008F07CFE10BD00004556454E545F410D3E
:10C490000A00000010B513A008F070FE00241AE096
:10C4A0001348407910B9FEF7BBFE01E002F03CFCF6
:10C4B0000F48407910B9FEF7B3FE01E002F034FCFA
:10C4C00000BF0C4802F0A3FA09494979884200D11B
:10C4D00010BD601CC4B2052CE2DB042000F0D2F8D1
:10C4E00000BFF5E74556454E545F41430D0A000035
:10C4F000C4250020240B002010B502A008F03EFE49
:10C5000010BD00004556454E545F420D0A00000024
:10C5100010B502A008F032FE10BD00004556454E91
:10C52000545F430D0A00000010B517A008F026FE66
:10C53000002422E017488079012802D1FEF7C6FEC8
:10C5400001E002F00BFC6420FFF7D7FC1148807972
:10C55000012802D1FEF7BAFE01E002F0FFFB6420E1
:10C56000FFF7CBFC00BF0C4802F051FA094989796A
:10C57000884200D110BD601CC4B2052CDADB032058
:10C5800000F080F800BFF5E74556454E545F444340
:10C590000D0A0000C4250020380B002010B5102122
:10C5A0000648FBF72BFE064800210160416001812F
:10C5B0000020044908600449086010BDC42600201A
:10C5C000D42600203C0900204009002010B510E0CE
:10C5D0000A480B4A1268815C0AA008F0CFFD08489F
:10C5E0000068401C0A2190FBF1F201FB1200044993
:10C5F00008600CF087F80028EAD010BDD42600208F
:10C600003C090020457272204E554D20697320254B
:10C61000640D0A0070B50546284600F0E1F9284689
:10C6200000F016F878B1284600F0ACFD0446284624
:10C6300000F09EFD06460548005D0021B14008401F
:10C640000249085500BF012070BD0000C42600202B
:10C650002DE9F0410446204600F094FD05462046B1
:10C6600000F086FD06460648405D0121B14000EA23
:10C67000010717B10120BDE8F0810020FBE70000B1
:10C68000C426002070B505462846FFF7E1FF90B9A3
:10C69000284609F047FA284600F074FD044628466B
:10C6A00000F066FD06460548005D0121B1400843E3
:10C6B0000249085500BF012070BD0000C4260020BB
:10C6C0000149C860704700000020024030B50446B0
:10C6D00004250F4800F0AAF80546042D16D10D4890
:10C6E000006940F002000B49086108464461006996
:10C6F00040F040000861064800F098F805460548FB
:10C70000006941F6FD71084002490861284630BDC4
:10C71000FFFF0F000020024004200B49C96801F010
:10C72000010109B101200EE00749C96801F00401C7
:10C7300009B1022007E00449C96801F0100109B1FC
:10C74000032000E0042070470020024003480069F5
:10C7500040F080000149086170470000002002405D
:10C7600070B504460D4604264FF6FF7000F05EF8E3
:10C770000646042E12D10A48006940F0010008491B
:10C78000086125804FF6FF7000F050F80646044817
:10C79000006941F6FE71084001490861304670BDEC
:10C7A0000020024078B506460C4604250020009083
:10C7B0004FF6FF7000F03AF80546042D26D11448D4
:10C7C000006940F001001249086134804FF6FF70A3
:10C7D00000F02CF80546042D11D1B01C0090200C5F
:10C7E000009908804FF6FF7000F020F805460848D1
:10C7F000006941F6FE7108400549086106E00448F9
:10C80000006941F6FE71084001490861284678BD7B
:10C8100000200240024803494860034848607047CE
:10C820002301674500200240AB89EFCD00B50246E9
:10C830000423FFF771FF034603E0FFF76DFF034694
:10C84000521E012B01D1002AF7D102B90523184647
:10C8500000BD000010B50A2900DD10BD028801EB03
:10C8600041030E4C24F82320827801EB410304EBB2
:10C8700083039A70C27801EB410304EB8303DA70FF
:10C88000027901EB410304EB83031A7101EB4103CD
:10C8900004EB830382689A6000BFDEE7282600204D
:10C8A00000B501211148FFF7D5FF02211048FFF71D
:10C8B000D1FF03210F48FFF7CDFF04210E48FFF7FA
:10C8C000C9FF05210D48FFF7C5FF06210C48FFF7FA
:10C8D000C1FF07210B48FFF7BDFF08210A48FFF7FA
:10C8E000B9FF09210948FFF7B5FF00BDC8080020BE
:10C8F000D4080020E0080020EC080020F808002000
:10C9000004090020100900201C090020280900202B
:10C9100070B504460E463046A16888470546207922
:10C92000A84203D00020A07025710EE0E078A84254
:10C9300002D10020A07008E0A078401CA070A07870
:10C940002188884201DB2079E070E07870BD00002A
:10C950002DE9F041074620480088401E86B2002598
:10C9600000241E4800EBC60041683846FBF788FFEC
:10C9700007D31A4800EBC50041683846FBF78AFF29
:10C9800003D240F6FF70BDE8F0811EE0A81900EB6D
:10C99000D071C1F34F04114800EBC4004168384620
:10C9A000FBF778FF02D2601E86B20EE00B4800EB68
:10C9B000C40041683846FBF763FF02D2601C85B2B1
:10C9C00003E0064830F93400DDE7B542DEDD034818
:10C9D00030F93500D7E700006A00002024B50108CF
:10C9E00010B50246002018E00E49095C914212D1B0
:10C9F000014605E00B4C4B1CE35C63544B1CD9B265
:10CA0000C0F10A0303448B42F4DC07490968491E5C
:10CA1000054B196010BD411CC8B20A28E4DB00BFF9
:10CA2000F8E70000D42600204009002010B524219A
:10CA30001948FBF7E3FB1222174918480AF0A6F938
:10CA400010221549123116480AF0A0F91248007850
:10CA5000FF2802D01048007850B90A20FFF74DFA9D
:10CA600010A008F08BFB12220B490C480AF08EF93B
:10CA70000948807CFF2802D00748807C58B90A20EA
:10CA8000FFF73BFA0DA008F079FB102202491231A2
:10CA900003480AF07BF910BDA026002000F0010831
:10CAA00000F801086273705F5265616443707546F7
:10CAB0006C61736820310D0A000000006273705FC2
:10CAC00052656164437075466C61736820320D0A6B
:10CAD0000000000070B504460D466421124805F0C0
:10CAE000FFFE012808D1A04700201049C872486005
:10CAF00000210D4805F0F4FE0C48C07A112811D130
:10CB00000A48407CA8420DD1084840686FF30F00E6
:10CB10000749884206D100200449C87248600120B4
:10CB20000449087170BD0000D8250020B00E002017
:10CB30000000EC1CAC25002010B504460220A047E4
:10CB40000220034908710021024805F0C9FE10BD0A
:10CB5000AC250020DC25002010B504461148C07A21
:10CB6000132812D10F48407CA0420ED10D484068D6
:10CB70006FF30F000C49884207D100200949C872A1
:10CB800048600A4908710A4988633221094805F05A
:10CB9000A7FE012804D100200449087104498863D4
:10CBA00010BD0000B00E00200000EC1CAC250020E1
:10CBB000200E0020DC25002010B50F4948680FA189
:10CBC000FBF727FB38B10C4A127E921ED1B20A4AFB
:10CBD000906803F031FD084948680BA1FBF719FB89
:10CBE00048B1054A127E032303EB8202D1B2024A06
:10CBF000906803F035FD10BD482100204F72646538
:10CC0000725F436F646500005365745F534E0000AC
:10CC10002DE9F041024600250026002000230024D3
:10CC2000002791F803C00CF00F0591F803C00CF039
:10CC3000100CBCF1000F03D091F802C04CEA0505BE
:10CC400091F800C0BCF1000F31D0146800202BE037
:10CC50004FF0010C0CFA00F3B1F800C00CEA030627
:10CC60009E4220D183004FF00F0C0CFA03F7BC4317
:10CC700005FA03FC4CEA040491F803C0BCF1280F48
:10CC800006D14FF0010C0CFA00FCC2F814C00AE007
:10CC900091F803C0BCF1480F05D14FF0010C0CFA1C
:10CCA00000FCC2F810C0401C0828D1D31460B1F8B1
:10CCB00000C0BCF1FF0F34DD546800202EE000F10D
:10CCC000080C4FF0010808FA0CF3B1F800C00CEAA8
:10CCD00003069E4221D183004FF00F0C0CFA03F79C
:10CCE000BC4305FA03FC4CEA040491F803C0BCF110
:10CCF000280F05D100F1080C08FA0CF8C2F81480CE
:10CD000091F803C0BCF1480F07D100F1080C4FF0B7
:10CD1000010808FA0CF8C2F81080401C0828CED38D
:10CD20005460BDE8F0810000F0B50A4600230024FD
:10CD30000021002500F00046B6F1004F02D11D4E43
:10CD4000F16901E01B4E7168C0F3034583B200F442
:10CD50004016B6F5401F08D121F07061154E766877
:10CD600026F07066134F7E6012E000F48016B6F570
:10CD7000801F06D1032606FA05F4A14341F0706135
:10CD800006E0460D360103FA06F6B14341F0706144
:10CD900022B1460D360103FA06F6314300F0004693
:10CDA000B6F1004F02D1034EF16101E0014E716016
:10CDB000F0BD0000000001400246002093680B40D7
:10CDC0000BB1012000E00020704701460878704751
:10CDD00010B50E490869804702280ED103210C487E
:10CDE00003F0A4FC48B10A4803F0B3FC0749886883
:10CDF000804740B20749087007E004490869804746
:10CE0000022802D000200349087010BD6C000020E9
:10CE100048370020C42500202DE9F05F1048B0F805
:10CE200002A0104A0121504608F064F80D4800683D
:10CE3000FBF7C6FC804642460B460B480B49FBF706
:10CE4000EFFB064600220A4BFBF772FB0446FBF79A
:10CE5000FBFC8346FFF77CFD06494881BDE8F09F57
:10CE600060000020B80000209A9999999999134080
:10CE70000000F03F880D00203CB504460B46002121
:10CE80000020019035A000680090012C32D100BF35
:10CE900007E0585C1DF80150684001AD6854481C1B
:10CEA000C1B20429F5DB9DF8050000F0F0009DF803
:10CEB000045005F00F0540EA051010709DF80500BC
:10CEC0000007000E9DF8065040EA151050709DF8BE
:10CED000060000F0F0009DF8075040EA1510907031
:10CEE0009DF8070000F00F059DF8040065F31F1082
:10CEF000D07030E0002107E0585C1DF80150684018
:10CF000001AD6854481CC1B20429F5DB9DF804004A
:10CF100000F00F059DF8050065F31F1010709DF8D7
:10CF2000050000099DF8065005F00F0540EA0510C0
:10CF300050709DF8070000F0F0009DF8065040EAA0
:10CF4000151090709DF8070000F00F009DF8045038
:10CF500040EA1510D07000203CBD00009023B021A5
:10CF600070B5054607F0A2F84443601C10B9AA202A
:10CF7000444303E014B907F099F804442C70200CE2
:10CF80006870200AA870EC70002070BD2DE9FF4386
:10CF900004460F461546002003903E4695F8019042
:10CFA0000B2E77D2DFE806F0900607555D9077905C
:10CFB0009090080000BF00BF4B46324603A92046B0
:10CFC00000F036F9A8B90020039059219DF80C20F3
:10CFD000501CC0B20390A1549DF80C10481CC0B264
:10CFE0000390665409219DF80C20501CC0B2039098
:10CFF000A154012E2CD10020039059219DF80C2022
:10D00000501CC0B20390A1549DF80C10481CC0B233
:10D010000390665409219DF80C20501CC0B2039067
:10D02000A15400219DF80C20501CC0B20390A154C3
:10D030002948C17A9DF80C20501CC0B20390A1541D
:10D040002548817A9DF80C20501CC0B20390A15451
:10D050003BE003AB224620490C313046FEF7D6FFB9
:10D0600033E068788DF80A00A8788DF80900E87830
:10D070008DF8080095F8048003A8174B0C3342463E
:10D08000CDE9004030460299FFF70EF808B10020C4
:10D0900003901AE018E068788DF80A00A8788DF8F7
:10D0A0000900E8788DF8080095F8048003A80A4B79
:10D0B0000C334246CDE9004030460299FEF76EFF40
:10D0C00008B10020039000E000BF00BF9DF80C00F5
:10D0D00004B0BDE8F08300009C3800202DE9F04743
:10D0E0000646002400271D4890F82C001B4991F8A3
:10D0F0002B1000EB012087B262222146641C72547F
:10D100003A0A2146641C72542146641C7754DFF8A5
:10D110005090002507E0134830F81500B84200D1C0
:10D1200003E0681CC5B2132DF5DB00BF132D00D141
:10D130000224022C0ED00C4810F805800B4A32F85D
:10D14000152002EB090130194246FBF73EF804EBCB
:10D15000080084B22046BDE8F08700006847002040
:10D160008C3700201EC001080AC00108E4BF010876
:10D1700001460A46C81701EB5070C010A1EBC00071
:10D18000C0B2704701460A46C81701EB5070C0F3A1
:10D19000C700704700B5FEF703FA38B10F480068C2
:10D1A00020F0080008300D49086005E00B480068D1
:10D1B00020F0080009490860FEF7FCF938B107487B
:10D1C000006820F00400001D0449086005E00348E1
:10D1D000006820F004000149086000BD740C0020C4
:10D1E0000246FF20002108E0064B33F8113093423D
:10D1F00001D1084603E04B1CD9B21329F4D300BF78
:10D20000704700001EC001080246FF20002108E010
:10D21000064B33F81130934201D1084603E04B1C12
:10D22000D9B20929F4D300BF704700007CC00108BF
:10D230002DE9F04104460E4615460020002100224B
:10D240000027DFF8D8C0ACF80A704FF059089446B0
:10D25000521C04F80C809446521C04F80C504FF0F9
:10D2600009089446521C04F80C8000BF50E001EB02
:10D27000C10C2A4F0C3717F81C701F404FB901EB37
:10D28000C10C264F0C3717F81C709F4201D00A2D95
:10D290003CD1234F3F68CF4007F00107B7B30120CF
:10D2A0001E4F7F897F1CDFF874C0ACF80A701D4FD9
:10D2B00057F82170C7F30748174602F1010C0CF02C
:10D2C000FF0204F80780174F37F82170C7F30728CB
:10D2D000174602F1010C0CF0FF0204F80780114F11
:10D2E00017F82180174602F1010C0CF0FF0204F838
:10D2F000078001EBC10C094F0C3717F81C8017464B
:10D3000002F1010C0CF0FF0204F807804F1CF9B287
:10D310001229ACDB3270BDE8F08100009C3800209F
:10D32000780C002074BF01082DE9F8433A480088C2
:10D33000002806DD38480088401E37490880BDE8CF
:10D34000F883FFF727FFFEF719FF344890F827000E
:10D3500000B1F4E7324800680090002514E000981E
:10D36000E84000F0010010B14FF0090806E005EBBD
:10D37000C5012C4810F8110020F00108414628464C
:10D38000FEF712FE681CC5B2122DE8DB12262648F5
:10D39000007800EBC001234800EB410420782249CB
:10D3A000097801EBC101214A12F81110884219D005
:10D3B000B11E2046FDF7B2FF87B22774391261749F
:10D3C00020781949097801EBC101184A02F81100C7
:10D3D0001749154A127806FB0210002332462146EF
:10D3E000FFF73CF810480078401C0F4908700846C9
:10D3F0000078122801DB002008700E480078401CDD
:10D40000C0B20C4908700A2803DB0020087007F03E
:10D4100007F900BF93E700006E0C0020684700206A
:10D42000740C0020A8380020880C0020EC39002063
:10D4300051480020890C00200246002112E001EB37
:10D44000410000EBC1000E4B03EB0010007890424E
:10D4500006D101EB410000EBC10003EB0010704767
:10D46000481CC1B2022909D201EB410000EBC10006
:10D47000034B03EB00100078FF28E0D10020EEE71B
:10D48000141500202DE9F0478246BAF1010F34D17E
:10D49000EB2182200BF066F9644908800846008879
:10D4A000B0F5004F0CDB08460088B0F5803F07DA86
:10D4B000084600884FF6FF71081A5C49088008E0AA
:10D4C0005A4800884FF6FF71884202DB0020574916
:10D4D000088056480088FBF720F98046544A554B8F
:10D4E000FBF72CF806460022534BFBF799F804464D
:10D4F000FBF7AAF95149086094E0BAF1020F59D13B
:10D50000E321B2200BF02EF9484908800846008834
:10D51000B0F5004F0ADB01204949088043480088E4
:10D520004FF6FF71081A4149088002E00020444983
:10D5300008803E480088FBF7F0F880463C4A3D4BA7
:10D54000FAF7FCFF064600223B4BFBF769F804465E
:10D55000FBF77AF93949086008460068FBF730F9AB
:10D5600006464FF03332374BFAF7E8FF0446364AA7
:10D57000364BFBF755F88046FBF766F92F490860F4
:10D580002F48008801284DD14FF4FA61304805F04A
:10D59000A7F9012806D12FA007F0F0FD00212C48A3
:10D5A00005F09EF9254801680020FAF7AAFE2349F4
:10D5B000086037E0BAF1030F34D1E321B4200BF057
:10D5C000D1F81A49088008460088B0F5004F0CDBF6
:10D5D00008460088B0F5803F07DA084600884FF615
:10D5E000FF71081A1149088008E0104800884FF6BA
:10D5F000FF71884202DB00200C4908800B4800883C
:10D60000FBF78BF806460A4A1B4BFAF797FF0446CE
:10D610000022094BFBF704F88046FBF715F9074990
:10D62000086000BF05480068BDE8F087CA00002018
:10D63000FCA9F1D24D622040E0FFEF40CC00002079
:10D64000D0000020F308CA40F6285C8FC2F51340D2
:10D65000E40000204E6567617469766520766F6C22
:10D66000746167652073616D706C65206661756CAF
:10D6700074210D0A000000004D6210400146087A36
:10D6800070470146087970470146C879032801D1DF
:10D6900001207047C879042801D10020F9E7002053
:10D6A000F7E701468879012800D17047887908B9E1
:10D6B0000020FAE70020F8E70148B0F90A007047B7
:10D6C000880D00200148406870470000880D002048
:10D6D000F8B5044600200090574A106F126F116B86
:10D6E000884705465548007830B1012840D00228C7
:10D6F00052D003286FD16FE051492046FBF7C0F8A4
:10D700000FD22046FBF75CF806464E4A4E4BFBF71D
:10D7100083F806D24D48C07B022802DA012000902F
:10D7200025E04FF07F512046FBF7AAF80BD248497D
:10D730002046FBF7AFF806D24448C07B022802DB44
:10D740000320009013E04FF081412046FBF7A2F840
:10D7500007D240492046FBF793F802D202200090FE
:10D7600005E015B100203949C8730020009059E048
:10D7700033492046FBF784F80BD22046FBF720F80C
:10D780000646354A354BFBF747F802D20120009098
:10D7900001E00020009045E04FF07F512046FBF76C
:10D7A0006FF807D22E492046FBF774F802D2032007
:10D7B00000900FE04FF081412046FBF76BF807D255
:10D7C00024492046FBF75CF802D20220009001E0D9
:10D7D0000020009026E022E04FF07F512046FBF72A
:10D7E0004FF80BD22046FAF7EBFF06461A4A1B4BBE
:10D7F000FBF712F802D2032000900FE04FF08141B6
:10D800002046FBF747F807D216492046FBF738F8C1
:10D8100002D20220009001E00020009002E00020EF
:10D82000009000BF00BF69460F48FFF771F8034939
:10D83000087008460078F8BDD8070020480C002082
:10D84000333373409A9999999999B93F04260020E6
:10D850003333333F0000C0407B14AE47E17A843F4E
:10D860000AD7233C0000E040342600202DE9FC4785
:10D870001848046801681848FAF743FD0546154939
:10D8800008681649FAF743FD06462946FAF771FD7E
:10D8900004462046FAF794FF07460022104BFAF799
:10D8A0004AFE05460E462046FAF78AFF0746002242
:10D8B0000B4BFAF743FE81462A463346FAF7B0FE91
:10D8C000CDE90001FAF7C0FF04460648046020468F
:10D8D000BDE8FC87880D00200000A0403333A34042
:10D8E000000024406C0000200148B0F90800704797
:10D8F000880D002001464879012800D170474879F9
:10D9000008B90020FAE70020F8E700000148007895
:10D9100070470000AD00002010B56A480088401C28
:10D9200080B2684908800A287EDB002008806648AB
:10D93000B0F84000B0F5FA7F33DA6348B0F8400041
:10D94000401C6149A1F840000846B0F84000B0F51D
:10D95000FA7F26D1002008720846407F032803D0B2
:10D960000846407F02281CD1002057490877012033
:10D970004877002081F8220088714874A1F840009F
:10D9800081F8240081F8250081F82700C8734F48EA
:10D990000079012803D100204C498861087100F00A
:10D9A0003DFC494890F8240058B14948007820F0DF
:10D9B0000100474908700846007820F0020008700E
:10D9C0000CE04348007820F00100401C40490870FA
:10D9D0000846007820F00200801C08703A4890F851
:10D9E000250058B13A48007820F004003849087002
:10D9F0000846007820F0080008700CE034480078F1
:10DA000020F00400001D324908700846007820F01C
:10DA10000800083008702C48B0F8540070B12A484B
:10DA2000B0F85400401E00E049E02749A1F8540036
:10DA30000846B0F8540008B90020C873254800888B
:10DA4000401C80B223490880642800DA10BD002001
:10DA5000204908801C4890F82900D8B11A4890F84D
:10DA60002900401E184981F82900084690F829002D
:10DA700080B90846C07801280CD10020C87008463B
:10DA800090F82800002805DD084690F82800401E80
:10DA900081F828000C48007A30B10D48007820F059
:10DAA00010000B4908700AE00948007820F01000C7
:10DAB0001030074908700020487700F0AFFB00BF26
:10DAC000C4E700003E0D00206847002030470020DA
:10DAD000500C00203C0D0020014601F00F010929E7
:10DAE00003DD01F13700C0B2704701F13000C0B270
:10DAF000FAE701460911092903DD01F13700C0B237
:10DB0000704701F13000C0B2FAE77047704700007B
:10DB100070B505460E4608480670002404E0285DEE
:10DB200006490855601CC4B2034800788442F6DBFD
:10DB300003F02EFD70BD0000490D0020400D0020B7
:10DB40000146002004E0054A125C0A54421CD0B28F
:10DB5000034A12789042F6DB70470000400D002027
:10DB6000490D002070B504460D4603F01DFE064623
:10DB700032462946204605F0A5FF70BD70B5054622
:10DB80000E4608480670002404E0285D0649085542
:10DB9000601CC4B2034800788442F6DB03F07CFDCD
:10DBA00070BD0000490D0020400D002010B503F0AD
:10DBB0008DFE10BD10B5044606F018F8002001498E
:10DBC000087010BD480D0020014800787047000023
:10DBD000490D00207FB505460E48006800900E48AC
:10DBE00000788DF80400002405E0295D0DF10500A2
:10DBF0000155601CC4B2084800788442F5DB01205E
:10DC00008DF80D00054948709DE80F0004F050FFA5
:10DC10007FBD00004C0D00204A0D00206847002009
:10DC200001490870704700004A0D002020B940F2F9
:10DC3000B471044A116003E040F2B471014A11600A
:10DC4000704700004C0D0020704700002DE9F041A6
:10DC500005460E4603F0A8FD04460A48007878B948
:10DC60007F2020706570A67003270020FFF7DEFF7D
:10DC700004F094F9384603F0F7FD012001490870DB
:10DC8000BDE8F081480D00202DE9F04105460E4623
:10DC900003F08AFD80460D480078A8B9A5B100249C
:10DCA00004E0305D08F80400601C84B2AC42F8DB8C
:10DCB0002F460020FFF7BAFF04F070F9384603F052
:10DCC000D3FD012001490870BDE8F081480D002016
:10DCD00010B503F0FFFB10BD014608787047014600
:10DCE0000878704700BFFEE770B50446002500BF06
:10DCF00000259120005D06281ED2DFE800F0031EFB
:10DD00004C4D5C7094F85400032815DB04F170004E
:10DD10000DF0C4F980B904F1940104F170000DF024
:10DD2000DDF940B1012191200155002084F89000D7
:10DD30000021AC200155012567E094F89930942228
:10DD40001159207804F19A02A668B04784F8980027
:10DD500094F89000401C84F8900094F89800FF28F4
:10DD60000ED00221912001550021AC200155012542
:10DD700094F8540081280DD1032084F8540009E060
:10DD800094F8901094F84400814203DB0421912020
:10DD90000155012539E038E094F8901094F84400DA
:10DDA000814203DB04219120015502E001219120F1
:10DDB0000155012529E0002191200155D4F8A80042
:10DDC00020B10121D4E92902904706E0206D20B15D
:10DDD0000121226DD4F8A4009047012515E000210F
:10DDE00091200155D4F8A80028B10220D4E92921B6
:10DDF00009F0A0FA07E0206D28B10220D4F8A42091
:10DE0000216D09F097FA012500BF00BF012D04D153
:10DE10009120005D04287FF46BAF25B122780421A6
:10DE2000012009F087FA70BD10B504469120005D0D
:10DE3000022811D194F8901094F84400814203DB39
:10DE400004219120015502E00321912001552278FF
:10DE50000421012009F06EFA10BD70B504460D468C
:10DE60009120005D022803D09120005D03280DD190
:10DE700094F89800A84209D105219120015594F801
:10DE80005400032802DB2046FFF72EFF70BD000080
:10DE900070B50024002515E001201B49086005200D
:10DEA000FAF7D4FF6006040E1848D0F81C0108B138
:10DEB00044F001040020144908600520FAF7C6FF69
:10DEC000681CC5B2082DE7DB00200F49086005205B
:10DED000FAF7BCFF00200D49C1F89C010520FAF7B4
:10DEE000B5FF0120084908600520FAF7AFFF0020C0
:10DEF0000649C1F898010520FAF7A8FF0120024958
:10DF0000091D0860204670BD988121420080214291
:10DF100010B501200C4908600520FAF797FF012091
:10DF20000A49C1F898010520FAF790FF0020064938
:10DF300008600520FAF78AFF00200449C1F898011B
:10DF40000520FAF783FF10BD9C8121420080214209
:10DF500010B50020094908600520FAF777FF012075
:10DF60000749C1F898010520FAF770FF012003491D
:10DF700008600520FAF76AFF10BD00009C8121426D
:10DF80000080214270B50446002018490860002531
:10DF90001CE004F0800020B101201449091D086034
:10DFA00003E000201149091D086001200F490860A5
:10DFB0000520FAF74BFF00200D49C1F89801052014
:10DFC000FAF744FF6006040E681CC5B2082DE0DBBA
:10DFD00001200649091D08600549C1F8980105207E
:10DFE000FAF734FF00200149086070BD9881214292
:10DFF0000080214210B54FF400600B4908600AF020
:10E0000062FA4FF480600849091F08600AF05BFA61
:10E010004FF48060044908600AF055FA4FF400603C
:10E020000149091F086010BD140C014010B54FF4E0
:10E030000060094908600AF046FA4FF4806006491A
:10E0400008600AF040FA4FF480600349091D086037
:10E050000AF039FA10BD0000100C014070B50546F9
:10E060000024002618E06006040E4FF480600F497B
:10E0700008600AF028FA0D480838006800F40060CB
:10E0800008B1601CC4B24FF480600849091D0860E3
:10E090000AF019FA701CC6B2082EE4DB15B9FFF7B6
:10E0A000C5FF01E0FFF7A6FF204670BD100C014040
:10E0B00070B50446002524E004F0800020B14FF440
:10E0C00000601149086004E04FF400600E49091D2A
:10E0D00008600AF0F8F94FF480600B4908600AF014
:10E0E000F2F94FF480600849091D0860072D02D13C
:10E0F0004000091F08606006040E0AF0E4F9681C7D
:10E10000C5B2082DD8DB70BD100C014010B54FF41E
:10E1100000600A490860401008600AF0D4F94FF422
:10E1200000600649091D08600AF0CDF94FF48060CF
:10E130000249091D08600AF0C6F910BD100C014023
:10E1400010B54FF40060074908604010091F0860CF
:10E150000AF0B9F94FF400600249091F08600AF09B
:10E16000B2F910BD140C014010B54FF400600E4917
:10E1700008600AF0A8F94FF480600B4908600AF0C3
:10E18000A2F909480838006800F4006008B10124C9
:10E1900000E000244FF480600349091D08600AF084
:10E1A00092F9204610BD0000100C014001460A887B
:10E1B000002000BF064BB3F83530934206DB00BFAA
:10E1C000034BB3F843301433934200DC0320704711
:10E1D000D80700202DE9F04104462568002600BF3D
:10E1E0000D48B0F839008046FAF792FA07462946FA
:10E1F000FAF746FB01D201260BE000BF0648C08FAC
:10E200008046FAF785FA07462946FAF743FB00D21B
:10E2100002263046BDE8F081D80700207047000094
:10E220007F20034908600020024908707047000001
:10E23000002C0040E901002010B51748C06940F4E7
:10E2400000601549C86140F2FF30144908607F2022
:10E25000091F08600846006840F080000860002040
:10E260000146002807DA0A07140E0D4A00F00F03D2
:10E270001B1FD45403E00A07130E0A4A135400BFAD
:10E280000020012181404209920002F1E022C2F8FF
:10E29000001100BF10BD000000100240042C00401F
:10E2A00018ED00E000E400E00EB541F28730ADF873
:10E2B00000006748019069466648FAF775FE42F229
:10E2C0000F70ADF800006448019069466148FAF7A4
:10E2D0006BFE40F6C310ADF800005F480190694640
:10E2E0005C48FAF761FE40F6C310ADF800005B48E9
:10E2F000019069465748FAF757FE41F28730ADF86A
:10E3000000005348019069465248FAF74DFE42F228
:10E310002730ADF800005048019069464D48FAF7A3
:10E3200043FE40F2E730ADF800004D4801906946E9
:10E330004848FAF739FE41F28730ADF80000464808
:10E34000019069464348FAF72FFE40F6C310ADF836
:10E3500000003F48019069463E48FAF725FE40F626
:10E36000C310ADF800003D48019069463948FAF7FE
:10E370001BFE42F20F70ADF800003748019069466D
:10E380003448FAF711FE41F28730ADF80000324808
:10E39000019069462F48FAF707FE41F28730ADF841
:10E3A00000002B48019069462A48FAF7FDFD40F627
:10E3B000C310ADF800002848019069462548FAF7D7
:10E3C000F3FD41F64B50ADF800002448019069463A
:10E3D0002048FAF7E9FD41F28730ADF800001E4809
:10E3E000019069461B48FAF7DFFD40F69F70ADF8D3
:10E3F00000001748019069461648FAF7D5FD40F22B
:10E40000E730ADF800001648019069461148FAF768
:10E41000CBFD41F64B50ADF800000F480190694626
:10E420000C48FAF7C1FD40F6C310ADF800000B48E8
:10E43000019069460748FAF7B7FD41F28730ADF819
:10E4400000000548019069460248FAF7ADFD0EBD8F
:10E4500059F6000880370020F5F10008A9F30008FC
:10E46000010D010810B5002414E004EB440101EB98
:10E47000C4010F4A02EB0110B021F9F7BFFEFF20E3
:10E4800004EB440101EBC401094A02EB01110870DD
:10E49000601CC4B2022CE8D302F0F6FD054901204D
:10E4A00008F062FF0449022008F05EFF10BD000082
:10E4B000141500207FA6000867A6000810B54821A3
:10E4C0000E48F9F79BFE28210D48F9F797FE0D48F5
:10E4D00001F0E4FF044624B1142221460848F9F76C
:10E4E00074FE0848203001F0D9FF04462CB11422F4
:10E4F000214603481430F9F768FE10BD441100208E
:10E500001C11002054BA010810B5204800F0FCF995
:10E510001F4800F0F9F91F4800F0F6F91E4800F016
:10E52000F3F91E4800F0F0F91D4800F0EDF91D4820
:10E5300000F0EAF91C4800F0E7F91C4800F0E4F9A3
:10E540001B4800F0E1F91B4800F0DEF91A4800F022
:10E55000DBF91A4800F0D8F9194800F0D5F9194844
:10E5600000F0D2F9184800F0CFF9184800F0CCF9C3
:10E57000174800F0C9F9174800F0C6F9164800F02E
:10E58000C3F9164800F0C0F910BD0000840A00204D
:10E59000980A0020AC0A0020140C0020C00A0020B9
:10E5A000D40A0020E80A0020FC0A0020100B0020FA
:10E5B000240B0020380B00204C0B0020600B0020A7
:10E5C000740B0020880B00209C0B0020B00B002057
:10E5D000C40B0020D80B0020EC0B0020000C002006
:10E5E00010B528480078052848D2DFE800F0030C71
:10E5F000391B2A002448C07B08B1032000E0012019
:10E60000204908703BE021480078072804D02049C1
:10E6100008698047022801D1022000E00120194941
:10E6200008702CE019480078072804D018490869B8
:10E630008047022801D1032000E00420114908701E
:10E640001DE012480078072804D011490869804766
:10E65000022801D1022000E004200A4908700EE0DF
:10E66000002009494860487301F070FE064988603F
:10E670000020044908700749087000E000BF00BF8F
:10E6800010BD00005C09002048090020042600207D
:10E690006C000020440900202DE9F04180460D4621
:10E6A000164600244046FEF7C7FE04460CB105B1ED
:10E6B00016B90020BDE8F081287818B194F854000C
:10E6C000012801D00020F5E795F8200000F00100B6
:10E6D00018B1A86A08B90020ECE795F8251084F86D
:10E6E000451094F8450010B9322184F8451094F88B
:10E6F000451001EB4101C80006F092FDC4F88C0002
:10E70000D4F88C0048B194F84530182204F1700018
:10E71000D4F88C100CF0D4FC01E00020CAE795F886
:10E72000200000F00100D8B994F84510080106F067
:10E7300077FDC4F88800D4F8880048B194F84530D3
:10E74000102204F15800D4F888100CF0B9FC07E04E
:10E75000D4F88C0006F036FD0020C4F88C00A9E740
:10E76000296A216404F1200720213846F9F746FD83
:10E770001F2229463846F9F728FDE86AF862A86A98
:10E78000B86295F8240087F82400286B386308489D
:10E7900030610848F0600848B06008487060084878
:10E7A000306008487061022084F85400012081E73D
:10E7B000D98C0108058B0108858B01089F8B010806
:10E7C000298C0108218A010838B5054601213C2021
:10E7D00001F046FC0121084601F042FC01211348EA
:10E7E000FEF7A2FAAC681CB911A006F0C7FC38BD50
:10E7F0002088ADF8000010208DF8030002208DF86D
:10E80000020069466068FEF703FA207A012804D105
:10E8100021886068FDF7F2FB05E0207A18B92188AD
:10E820006068FDF7E9FB00BFE1E70000000230008F
:10E830004F5053206973204E554C4C0D0A00000078
:10E8400010B5034800F0CEF8024800F0F6F810BD0D
:10E85000880B00209C0B002010B5034800F0C2F884
:10E86000024800F0EAF810BD9C0B0020880B002045
:10E8700010B5034800F0B6F8024800F0B3F810BD38
:10E88000880B00209C0B002010B5054800F0AAF86A
:10E89000044800F0A7F804A006F070FC10BD0000CA
:10E8A000880B00209C0B0020414320C8ABB5CD0055
:10E8B00010B5054800F0C1F8044800F0BEF804A007
:10E8C00006F05CFC10BD0000880B00209C0B0020B3
:10E8D000414320C8ABB8DF0038B505460121102000
:10E8E00001F0BEFBAC6804B938BD2088ADF800006B
:10E8F00004208DF8030003208DF80200694660684B
:10E90000FEF786F900BFEFE770B505462C68206872
:10E9100000B970BD20462168884700BFF9E70000B4
:10E9200038B5054601213C2001F09AFBAC681CB9C2
:10E9300010A006F023FC38BD2088ADF800001020A0
:10E940008DF8030002208DF8020069466068FEF72A
:10E950005FF9207A012804D121886068FDF74EFB19
:10E9600005E0207A18B921886068FDF745FB00BFF3
:10E97000E1E700004F5053206973204E554C4C0D79
:10E980000A00000038B505460121042001F068FBAB
:10E99000AC6804B938BD2088ADF8000010208DF8AF
:10E9A000030003208DF8020069466068FEF730F925
:10E9B000207A012804D121886068FDF71FFB05E05B
:10E9C000207A18B921886068FDF716FB00BFE1E7DF
:10E9D00010B5044621886068FDF70EFB0020207208
:10E9E000012010BD70B5044620684568686808B904
:10E9F000002070BD22689068696888470120F8E7A8
:10EA000010B5044621886068FEF7D6F910BD70B5D0
:10EA1000044620684568A86808B9032070BD2268CC
:10EA20009068A9688847F9E710B5044621886068AE
:10EA3000FDF7E4FA0120207210BD70B5044620688D
:10EA40004568286808B9002070BD22689068296868
:10EA500088470120F8E738B505460121102001F06C
:10EA6000FFFAAC6804B938BD2088ADF80000482032
:10EA70008DF8030003208DF8020069466068FEF7F8
:10EA8000C7F800BFEFE7000070B50A48C4880A4A1B
:10EA90000221204606F02EFA084907480068F9F7D7
:10EAA00036FC05464FF07A51F9F7D9FB0449486026
:10EAB00070BD000060000020B40000200000304164
:10EAC000880D002070B50446002000BF14F8016BCB
:10EAD0008E4204D1012A00D108E0551EEAB203B9E2
:10EAE00004E0451CA8B25D1EABB2EFE700BF70BDED
:10EAF00010B517480078072804D0164908698047E0
:10EB0000022801D1642001E04FF47A7012490860B4
:10EB100008460168114803F0E3FE012816D11048A9
:10EB200001780068401C0E4A106001F0010020B11D
:10EB300000BF0C48FFF756FF04E000BF0948FFF78D
:10EB40007CFF00BF0021054803F0CAFE10BD000095
:10EB5000042600206C000020080000200000002097
:10EB600004000020100B00201048807A08B9002013
:10EB700070470E480B300E490978405C30B10B48A5
:10EB80000B300B490978405C0A4908800848007836
:10EB9000401C074908700548807A0978884202DCE1
:10EBA00000200349087003480078E1E7500C00207A
:10EBB0009D0600209E0600207047000003A006F07E
:10EBC000DDFA06F005FA00F0CBFD0000476F207477
:10EBD0006F20536C6565700D0A00000000BFFEE7F2
:10EBE000704710B54FF4A06000F046F810BD00006B
:10EBF00000F01F0201219140024A430942F823100C
:10EC00007047000080E100E070B5002100230F2272
:10EC1000C47804B3154C246804F4E064C4F5E064DB
:10EC2000210AC1F10403CA40447804FA03F184784C
:10EC30001440214309010E4C0678A155047804F0D4
:10EC40001F050124AC4005786D11AD0005F1E025EC
:10EC5000C5F8004109E0047804F01F050124AC4028
:10EC6000044D0678761145F8264070BD0CED00E0A5
:10EC700000E400E080E100E002490143024A116043
:10EC8000704700000000FA050CED00E0024A0A405F
:10EC90000243024B1A60704780FFFF1F08ED00E03F
:10ECA0000648006800F4E06005490843001D034978
:10ECB0000860BFF34F8F00BFFEE700000CED00E0DF
:10ECC0000000FA050648006800F4E06005490843C2
:10ECD000001D03490860BFF34F8F00BFFEE700002F
:10ECE0000CED00E00000FA0510B54FF400720021B1
:10ECF000014805F0C7F910BDC847002010B5084805
:10ED0000FFF79BFE0120FDF7F8F80648FFF795FE98
:10ED10004FF4FA70FDF7F1F80248FFF763FE10BDFB
:10ED2000880B00209C0B002010B5FFF795FD642098
:10ED3000FDF7E3F8FFF79CFD00200349487103A0AD
:10ED400006F01CFA10BD0000C42500204F50454EAF
:10ED50005F41435265616C790D0A000010B50120D6
:10ED60000449887104A006F009FA0748FFF765FE18
:10ED700010BD0000C42500204F50454E5F44435253
:10ED800065616C790D0A0000840A002010B50B48FB
:10ED9000008848B901200949088000200849887383
:10EDA00008A006F0EBF908E00020044908800120E3
:10EDB0000349887307A006F0E1F910BD5205002051
:10EDC000AC250020B4F2BFAAC0CFBBAFC4A3CABD5C
:10EDD0000D0A0000B9D8B1D5C0CFBBAFC4A3CABD1E
:10EDE0000D0A000001460A780AB901207047002088
:10EDF000FCE70000014908627047000000000E4275
:10EE00000349096841EA8001014A11607047000026
:10EE10000070004010B5044604F10B0318460CF0D6
:10EE2000C7F91868C0F3093081B20F4881871868A4
:10EE3000C0F309300A2190FBF1F00B4981F86C0016
:10EE40005868800C81B20848C1875868800C064910
:10EE5000A1F8460018791968890D60F38D210248E0
:10EE6000A0F84810012010BDD807002070B5054655
:10EE700005F10B0420460CF09BF96268C2F3C262F4
:10EE8000D0B20A4A126F516A88472268C2F30262FE
:10EE9000D0B2064A126FD16A88472068C0F340702A
:10EEA000C1B2024880F85910012070BDD807002077
:10EEB00010B5044604F10B0318460CF079F9988854
:10EEC00080B20A2190FBF1F081B20F48A0F86610E1
:10EED0005868000C0A2190FBF1F081B20A48A0F8B2
:10EEE00068105868000C0A2190FBF1F080B240F4E1
:10EEF00080510548A0F84A101868000C024981F8B2
:10EF00004F00012010BD0000D807002010B50446B6
:10EF100004F10B0318460CF04BF99888000A0A30EC
:10EF2000C1B20F4880F86A105868000E0A30C1B2AA
:10EF30000B4880F86B109888010A094880F8501037
:10EF40005868010E064880F852105868010C0448B1
:10EF500080F85110197980F85310012010BD00007D
:10EF6000D807002070B50546FAF744F905F10B04FF
:10EF700020460CF01DF96068C0F3892000EB80008A
:10EF80004FF6FF7101EA40000549A1F841006068B1
:10EF9000000D81B20248A0F84310012070BD0000AE
:10EFA000D807002070B50546FAF724F905F10B04DF
:10EFB00020460CF0FDF82088C0F305202168C1F33D
:10EFC0000441C1EB011100EB810081B20248A0F8BD
:10EFD0004D10012070BD0000D807002010B5044678
:10EFE00004F10B0318460CF0E3F8044918680863B1
:10EFF000024859684163012010BD000030250020FF
:10F0000010B5044604F10B0318460CF0D1F804497E
:10F010001868886302485968C163012010BD000068
:10F020003025002010B5044604F10B0318460CF0FF
:10F03000BFF804491868086402485968416401200F
:10F0400010BD00003025002070B5054605F10B0409
:10F0500020460CF0ADF82068C0F34040C1B21A4819
:10F0600080F845106068000C0A2190FBF1F0164909
:10F07000A1F83300A088C0F38D00088021781248E1
:10F0800041712088010A104880F83B10A088C0F325
:10F090008D0081B20C48A0F839102268C2F30042FA
:10F0A000D0B2094A126FD16888472068C0F3004087
:10F0B000C1B2054880F85A102068800C81B202481D
:10F0C0000181012070BD0000D807002010B5044662
:10F0D00004F10B0318460CF06BF89888C0F38D0010
:10F0E00081B20648C1805868000DC0F57A6081B2CF
:10F0F0000248A0F83510012010BD0000D8070020FC
:10F1000010B5044604F10B0318460CF051F81868CA
:10F11000C0F3893081B20548A0F837100449186857
:10F12000886503485968C165012010BDD8070020D3
:10F13000302500202DE9F041274805880126274881
:10F1400027494860002008702B463246202123487A
:10F15000FFF7B8FC044622494C70AC4202D10120B2
:10F16000BDE8F081701CC6B231E01C48005D20286B
:10F1700002D1601C84B22AE02746184801191848B9
:10F180000278083040F822102B46324620211348DE
:10F19000FFF798FC0446E01BC1B211480278183012
:10F1A000815418380378083050F823200838017843
:10F1B0000CA005F0E3FF0A480078401C08490870DD
:10F1C00008460078042800DB03E0701CC6B2AC429D
:10F1D000CBD100BF0120C3E71E0200204E1E00203D
:10F1E00048210020256420706172616D3A25730A00
:10F1F000000000007CB5002000900190009001907C
:10F200004FF44570624908604860002008724872F7
:10F21000082088726C4601F0D1FA054601F0E4FA44
:10F220000646D4E9000165F31961C4E90001D4E997
:10F23000000165F39B61C4E90001D4E9000166F3B4
:10F240001D71C4E90001D4E9000166F39F71C4E9AE
:10F2500000015048007A08B9012000E00020D4E9FC
:10F26000001260F31142C4E900124A48C07908B99B
:10F27000012000E00020D4E9001260F39342C4E9C9
:10F280000012FCF75FFC0246D4E9000162F38B2018
:10F29000C4E90001FCF786F80146D4E9000261F3F5
:10F2A0001552C4E900023C4908698047022814D17C
:10F2B0003A49898989B20A2291FBF2F188B2C828B9
:10F2C00001DA002101E0A0F1C80188B2D4E90021EF
:10F2D00060F35D52C4E9002106E00022D4E9001089
:10F2E00062F35D51C4E900102D48006FB0F90200CF
:10F2F0000A2190FBF1F000F5FA70D4E9001260F3F6
:10F300001431C4E90012FCF7EBF90146D4E90020FE
:10F3100061F3DF72C4E900202420FDF799F9D4E9F4
:10F32000001260F39E71C4E900121E48807C58B13F
:10F330001C48007B40B11748427AD4E9000162F3CF
:10F340004F31C4E9000106E00022D4E9000162F374
:10F350004F31C4E900010F48407810B90D4880785A
:10F3600008B1012000E00020D4E9002160F3D7516A
:10F37000C4E9002120460BF022FF05480B3000991C
:10F380000160019941600B3808F02CF97CBD000048
:10F3900098250020C42500206C000020880D002046
:10F3A000D8070020480900207CB50020009001907B
:10F3B000009001904FF47A704E4908604860002038
:10F3C00008724872082088726C462820FDF740F9C0
:10F3D00058B92620FDF73CF938B91C20FDF738F95B
:10F3E00018B92120FDF734F908B1012000E0002010
:10F3F000D4E9001260F38E32C4E900123E4800786E
:10F4000004280DDB3C480078062809DC3A48C07C1B
:10F4100030B10122D4E9001062F3CF30C4E900100A
:10F42000FBF7C0FF022803D0FBF7BCFF032806D17F
:10F430000022D4E9000162F3CF31C4E900012F4971
:10F44000486880472830D4E9001260F31F62C4E99D
:10F4500000122B4800782830D4E9001260F31742DC
:10F46000C4E90012254908682649F8F750FF064606
:10F47000F9F779F9054642F210718D4201D90A4631
:10F4800000E02A46D4E9000162F30D01C4E900015D
:10F490001D48807C98B11C48007B80B11B48827A53
:10F4A000D4E9001062F30B21C4E90010FFF75CFB04
:10F4B000D4E9002160F30702C4E900210CE0002236
:10F4C000D4E9001062F30B21C4E90010D4E9001064
:10F4D00062F30701C4E9001020460BF070FE0548F6
:10F4E0000B3000990160019941600B3808F07AF8FF
:10F4F0007CBD000098250020042600206C00002020
:10F50000C425002000007A4448090020500C002047
:10F510001CB50020009001900090019040F23F4007
:10F520001C490860486000200872487208208872F0
:10F530006C4619480078401C174908700846007846
:10F54000102801DB002008700122D4E9000162F3D9
:10F55000CF30C4E9000110480278D4E9001062F30A
:10F560000B21C4E900100C480078401CD4E90012BB
:10F5700060F30701C4E9001220460BF020FE0548A5
:10F580000B3000990160019941600B3808F02AF8AE
:10F590001CBD000098250020A00600201FB50120FA
:10F5A000134908720020A1F840000098A0F23470BE
:10F5B00010B1AB2818D10BE040F234700C49A1F81F
:10F5C0004E009DF804100DF10500FEF7D7FA0CE08F
:10F5D00040F2DF700649A1F84E009DF804100DF1CD
:10F5E0000500FEF795FA00E000BF00BF1FBD000058
:10F5F0006847002010B5044604F10B0318460BF0D1
:10F60000D7FD06491868086104485968416158687F
:10F61000000C0349096F0880012010BD302500202F
:10F62000D807002070B5054605F10B0420460BF005
:10F63000BFFD2268C2F30362D0B2064A126FD169DD
:10F6400088476268920FD0B2024A126F51698847A8
:10F65000012070BDD80700207CB500250020009057
:10F6600001900090019040F22350394908604860B1
:10F67000002008724872082088726C46354802786B
:10F68000D4E9001062F30701C4E900100022D4E9B4
:10F69000001062F39031C4E900102E48006860B198
:10F6A0002C480068042808D200BF0122D4E90001D8
:10F6B00062F30D20C4E9000119E02648006804281F
:10F6C0000ED9F9F7BBFC0546002D01DD022000E054
:10F6D0000120D4E9001260F30D21C4E9001206E014
:10F6E0000022D4E9000162F30D20C4E900011A48A8
:10F6F000425DD4E9001062F31D51C4E90010681C9A
:10F700001549085CD4E9001260F39F71800860F32A
:10F710000702C4E90012A81C0F490A5CD4E90010D2
:10F7200062F31120C4E90010E81C0B490A5CD4E91B
:10F73000001062F39B40C4E9001005480B300099AB
:10F740000160019941600B3807F04CFF7CBD00005F
:10F750009825002040090020D42600207047000092
:10F760004FF0E020006920F002004FF0E021086136
:10F770000220FFF73DFA0320FFF73AFA0420FFF7D3
:10F7800037FA0520FFF734FA0620FFF731FA072091
:10F79000FFF72EFA0820FFF72BFA0920FFF728FAC7
:10F7A0000A20FFF725FA0B20FFF722FA0C20FFF7BB
:10F7B0001FFA0D20FFF71CFA0E20FFF719FA0F2091
:10F7C000FFF716FA1020FFF713FA1120FFF710FACF
:10F7D0001320FFF70DFA1420FFF70AFA1520FFF7A0
:10F7E00007FA1620FFF704FA1720FFF701FA18208E
:10F7F000FFF7FEF91920FFF7FBF91A20FFF7F8F9D8
:10F800001B20FFF7F5F91C20FFF7F2F91D20FFF789
:10F81000EFF91E20FFF7ECF91F20FFF7E9F9202090
:10F82000FFF7E6F92120FFF7E3F92220FFF7E0F9DF
:10F830002320FFF7DDF92420FFF7DAF92520FFF771
:10F84000D7F92620FFF7D4F92720FFF7D1F9FEF7E3
:10F85000E7FC2820FFF7CCF92920FFF7C9F92A2077
:10F86000FFF7C6F93220FFF7C3F93320FFF7C0F9DD
:10F870003420FFF7BDF93520FFF7BAF93620FFF73E
:10F88000B7F93720FFF7B4F93820FFF7B1F939207D
:10F89000FFF7AEF93A20FFF7ABF93B20FFF7A8F9E5
:10F8A0003C20FFF7A5F93D20FFF7A2F93E20FFF726
:10F8B0009FF93F20FFF79CF94020FFF799F941207D
:10F8C000FFF796F94220FFF793F94320FFF790F9ED
:10F8D00000BF002005E04FF0FF32134941F820201F
:10F8E000401C0828F7DB00BF0120FFF789FAFEF76C
:10F8F00097FC00BF0D48FFF775F84FF4FA70FCF75E
:10F90000FCFA0B48FFF799F80A48C07B18B10A487F
:10F91000FFF793F802E00848FFF764F841F28830F7
:10F92000FCF7EBFAFFF7CEF980E100E0140C0020C1
:10F93000000C002048090020EC0B002070B56F4837
:10F940000068401C6D490860084600680521B0FB4E
:10F95000F1F201FB1200052873D2DFE800F0033951
:10F960005188A30066A005F009FC7048007A08B130
:10F970006FA005E0714908698047714951F820007E
:10F98000044621466FA005F0F9FB754A106F126F0F
:10F99000116A8847734951F82040214672A005F04A
:10F9A000EDFB6F4890F86C2075480078754B53F864
:10F9B000201075A005F0E2FB694890F8450008B1F9
:10F9C00079A000E07CA001467FA005F0D7FB93E082
:10F9D0006348B0F84320B0F8411081A005F0CEFB99
:10F9E0008A48B0F81D20B0F81B1089A005F0C6FBAE
:10F9F0005B48006FB0F9021090A005F0BFFB7BE000
:10FA00004E498868804704464C4948688047054607
:10FA1000224629468FA005F0B1FB00BF9548FEF7AE
:10FA2000F6FF08B194A000E096A004469748FEF7C0
:10FA3000EEFF08B193A000E08FA0054622462946BC
:10FA400000E058E092A005F099FB3848007A08B130
:10FA500097A000E097A002463448C07908B196A06C
:10FA600000E096A0014696A005F088FB44E09C4982
:10FA70004868F8F7A5FE044622460B4699A005F013
:10FA80007DFB9748B0F90C109BA005F077FB2B4944
:10FA90000868F8F795FE044622460B469CA005F040
:10FAA0006DFB29E02E4A106F126F116B88479E493B
:10FAB00051F8204021469DA005F060FB1B4880784E
:10FAC00008B1A0A000E0A1A002461848407808B103
:10FAD0009CA000E09DA001469EA005F04FFBF9F719
:10FAE000BBF928B9A14802684168A1A005F046FB0E
:10FAF00000F054F900E000BF00BF70BDC008002056
:10FB00000D0AA1AAA1AAA1AAA1AAA1AAA1AAA1AAD1
:10FB1000A1AAA1AAA1AAA1AAA1AAA1AAA1AAA1AA8D
:10FB2000A1AAA1AAA1AAA1AA0D0A0000C425002089
:10FB300041435F4368617267696E67006C00002033
:10FB40004C0800200D0A4443555F576F726B696E75
:10FB5000674D6F6465203C25733E0D0A0000000070
:10FB6000D8070020900800205643555F576F726BEE
:10FB7000696E674D6F6465203C25733E0D0A000079
:10FB800004260020580800204368617267696E6788
:10FB90005F5374616765203C25733E09534F4320D2
:10FBA0003C25643E0D0A0000436F6E7374616E74F1
:10FBB000566F6C7461676500436F6E7374616E7429
:10FBC00043757272656E74004368617267696E672F
:10FBD0005F4D6F646520203C25733E0D0A000000D8
:10FBE00044656D616E645F766F6C74616765203C1F
:10FBF00025643E0944656D616E645F63757272656C
:10FC00006E74203C25643E0D0A000000200E00208A
:10FC10004F75747075745F766F6C74616765203CA6
:10FC200025643E094F75747075745F6375727265F3
:10FC30006E74203C25643E0D0A000000436861722A
:10FC400067696E6743757272656E74203C25643E09
:10FC50000D0A000054656D7031202020203C256481
:10FC60003E092047554E5F54454D50203C25643E8B
:10FC70000D0A0000240B0020446973636F6E6E65EB
:10FC8000637400004F70656E00000000380B0020A8
:10FC900044435F52656C6179203C25733E202041CE
:10FCA000435F52656C6179203C25733E0D0A00006C
:10FCB00043430000434332004343310043500000BC
:10FCC00043502D4343312020203C25733E092043DF
:10FCD000432D4343322020203C25733E0D0A000073
:10FCE000880D00204B4C33305F566F6C74203C25E0
:10FCF000663E0D0A0000000053616D706C5F766F08
:10FD00006C74616765202020203C25643E0D0A004C
:10FD100043435F5220697320202020202020202090
:10FD2000203C25663E0D0A00780800204F42435FC4
:10FD300047756E436F6E6E6563742020203C25739B
:10FD40003E0D0A004E4F5F4C6F636B004C6F636B50
:10FD5000000000004856494C203C25733E20485680
:10FD6000494C5F32203C25733E0D0A0048090020B3
:10FD7000456E7465722046616C7365536C65657081
:10FD80002049646C6520636F756E74202564204D76
:10FD900041582069732025640D0A000070B50024C5
:10FDA0001FE01148005D002819DDFCF70FFC372625
:10FDB000002511E00D4810F835000B49095D884217
:10FDC00008D10948025D094800EBC500416808A058
:10FDD00005F0D4F9681CC5B2B542EBDB00BF601C6E
:10FDE000C4B20A2CDDDB70BDD4260020ACBD0108F6
:10FDF0004572726F7220436F646520496E466F20B2
:10FE000069732025732D25640D0A000010B52C4858
:10FE1000007830B101280BD0022820D0032848D127
:10FE200045E0F9F719F880F001002549087044E031
:10FE30000BF090F904461CB90120214908700DE02F
:10FE4000012C03D100201E49087007E0022C05D1C7
:10FE500001201C4948730220194908702DE01A48F6
:10FE60000068401C184908601648807B012809D0AA
:10FE700008460068052805D30020086003201049C3
:10FE8000087005E010480068012801D1F9F7D2FE9A
:10FE9000FEF7A6FB0B48007B10B904F045F928B12A
:10FEA00000200849486048730549087005E0FEF7DE
:10FEB00085FE06A005F062F900BF00BF10BD00007E
:10FEC00044090020480900206009002045525220C2
:10FED000536C6565700D0A0030B53D4C647A04EBD7
:10FEE00084046300B3F5AF7F00DA30BD1A46394CA5
:10FEF0002178394C04EBC1046488944226DA084620
:10FF00000DE0354C34F83040944206DA324C04EBC4
:10FF1000C0046488944200DD03E0441CE0B205287C
:10FF2000EFDB00BF052800DB042000242B4D2C70E4
:10FF30002B4C247844B90124294D2C70264C04EB19
:10FF4000C104E488274D2C8001462DE0224C34F872
:10FF50003140944223DD08460DE01F4C34F8304018
:10FF6000944206DA1C4C04EBC0046488944200DD21
:10FF700003E0441EE0B20028EFDC00BF0024184D6F
:10FF80002C70164C247844B90124144D2C70124C5A
:10FF900004EBC104E488134D2C80014604E00024E6
:10FFA0000E4D2C700E4D2C700E4C24882CB10D4C27
:10FFB0002488641E0B4D2C8007E0064C24788C426C
:10FFC00003D0322A01DD034C217000BF8DE7000011
:10FFD00088380020D80C0020BCBF0108E20C0020AB
:10FFE000E10C0020E40C002001460020034A506888
:10FFF00020F4404008435060704700000010024069
:020000040801F1
:1000000029B1064A52690243044B5A6104E0034A8B
:1000100052698243014B5A61704700000010024050
:1000200029B1064AD2690243044BDA6104E0034A6B
:10003000D2698243014BDA61704700000010024030
:1000400029B1064A12690243044B1A6104E0034ACB
:1000500012698243014B1A61704700000010024090
:1000600029B1064A92690243044B9A6104E0034AAB
:1000700092698243014B9A61704700000010024070
:100080000149086070470000400442422DE9F041F8
:1000900000210022002500230026002400278C4692
:1000A000DFF86081D8F8048008F00C0121B1042940
:1000B00007D0082959D109E0DFF84C81C0F8008049
:1000C00058E0DFF84481C0F8008053E0DFF8348165
:1000D000D8F8048008F47012DFF82881D8F804807A
:1000E00008F48035920C0D2A01D0921C00E0062203
:1000F00035B9DFF8188102FB08F8C0F8008033E05A
:10010000DFF80081D8F82C8008F48036DFF8F4801E
:10011000D8F82C8008F00F0808F1010446B9DFF880
:10012000E880B8FBF4F808FB02F8C0F800801BE098
:10013000DFF8D080D8F82C80C8F3031808F1010745
:10014000DFF8C080D8F82C80C8F3032808F1020C2F
:10015000DFF8B480B8FBF7F808FB0CF8B8FBF4F84C
:1001600008FB02F8C0F8008004E0DFF89C80C0F8CB
:10017000008000BF00BFDFF88C80D8F8048008F052
:10018000F0010909DFF8888018F80130D0F8008004
:1001900028FA03F8C0F80480DFF86880D8F80480F3
:1001A00008F4E061090ADFF8688018F80130D0F837
:1001B000048028FA03F8C0F80880DFF84880D8F8EF
:1001C000048008F46051C90ADFF8448018F801304F
:1001D000D0F8048028FA03F8C0F80C80DFF82480F7
:1001E000D8F8048008F44041890BDFF8288018F81B
:1001F0000130D0F80C80B8FBF3F8C0F81080BDE8EF
:10020000F08100000010024000127A0000093D0059
:10021000F10500200106002010B501460022002350
:1002200000204A11012A02D1094C236806E0022A63
:1002300002D1074C236A01E0054C636A01F01F02FA
:10024000012494401C400CB1012000E0002010BDAE
:1002500000100240014908607047000080044242DB
:1002600001490860704700003C0442420249096AA3
:100270000143014A116270470010024010B50D4859
:10028000008F00F4804058B90A4890F8380000F018
:10029000200028B9074890F8380000F0400030B13D
:1002A0002F20FCF7EFF900200249886310BD0120E0
:1002B000FCE70000200E002070B505460E46002425
:1002C00000BF03E0285D03F0DBFC641CB442F9DBF3
:1002D00070BD70B505460E46002400BF03E0285DE2
:1002E00003F0CEFC641CB442F9DB0D2003F0C8FC23
:1002F0000A2003F0C5FC002403E0285D02F042FC64
:10030000641CB442F9DB70BD70B505460E4600248E
:1003100000BF03E0285D02F035FC641CB442F9DB49
:1003200070BD00000348008840F0100001490880BB
:100330007047000004280040034800884FF6EF7122
:100340000840014908807047042800400021034804
:100350000188001F008841EA004070471C280040C7
:1003600010B501214FF0C050FFF75AFE4FF4007056
:10037000FFF77CFF0120FFF773FF0120FEF73AFD36
:10038000F8F776FE0120FFF765FF00BF6120FFF759
:1003900043FF0028FAD04FF40070FFF767FF0120F9
:1003A000FFF75EFF00F024F800F018F849F63F4030
:1003B00000F004F800F012F810BD000000B502468D
:1003C000FFF7B0FFC2F3034003490880091D0A800C
:1003D000FFF7B2FF00BD00000828004000BF03483F
:1003E000008800F020000028F9D070470428004061
:1003F000074800884FF6F77108400549088000BF9C
:100400000348008800F008000028F9D07047000079
:100410000428004010B5012013490860FDF778FD5D
:100420009020FDF7AFFD0020FDF7ACFDFDF790FD3E
:10043000FDF76EFD9120FDF7A5FDFDF729FD0B49A8
:100440000880FDF725FD09494880FDF781FD074833
:1004500040880649098840EA012000B20349088023
:100460000846008880B210BD98812142C400002057
:1004700010B505A004F082FE12210648FFF744FFE4
:1004800005A004F07BFE10BD4F726465725F436F80
:1004900064652000A02600200D0A000070B5054606
:1004A0001DB1686808B1A86808B9002070BD0024B3
:1004B0000EE004EB440000EBC4001B4901EB00100C
:1004C00000782978884201D10020EFE7601CC4B28F
:1004D000022CEED3002422E004EB440000EBC40025
:1004E000114901EB00100078FF2816D104EB4401FC
:1004F00001EBC4010C4A02EB011020222946F7F758
:1005000064FE012004EB440101EBC401064A02EB46
:10051000011181F854000548C8E7601CC4B2022CE0
:10052000DAD30020C2E700001415002044010020A7
:1005300000200149088070471E02002030B50023CA
:10054000002000210022354CA47A1CB90024344D2F
:100550006C7230BD0024334D2C704FE02F4C0B34A7
:10056000304D2D78645D002C43D02C4C0B342D4D38
:100570002D78645D2C4D2C802C462488102C01D1C4
:10058000012036E0284C2488012C0FD0264C2488EA
:10059000022C0BD0244C2488052C07D0224C248814
:1005A000082C03D0204C2488092C01D1022120E002
:1005B0001D4C2488032C1BD01B4C2488042C17D0E2
:1005C000194C2488062C13D0174C24880A2C0FD0E1
:1005D000154C24880B2C0BD0134C24880C2C07D0E2
:1005E000114C24880E2C03D00F4C2488112C00D1E0
:1005F00003220C4C2478641C0A4D2C70074CA47AFE
:10060000084D2D78AC42A9DC00B1034601B10B4680
:1006100002B11346024C637200BF9AE7500C0020EF
:10062000C42500203609002038090020704772B622
:10063000704762B67047000070B505460C46122C34
:1006400000D070BD224629460448F7F7BEFD0120C0
:10065000024981F8220000BFF3E70000A026002035
:10066000F0B502460B4600210020132B00D0F0BD50
:10067000002110E0545C202C0BD0565C0446C517BA
:1006800000EB15752D11A0EB0517074DEE55441C19
:10069000E0B24C1CE1B29942ECDB0124024D123D68
:1006A00085F8234000BFE2E7B226002070B5FDF7D1
:1006B000DDF80646FDF70CF804460025012C01D1B3
:1006C000012506E0022C01D0032C01D1022500E017
:1006D000002512480078854205D0002010490860A6
:1006E0000E48057019E00F480078854203D10020BC
:1006F0000B49086011E00A480068401C084908607E
:1007000008460068022808D30448007805490870A4
:100710000548047000200249086070BDAC0000204C
:10072000C0000020AD000020AE00002070B50446DF
:100730000D46FFF70BFE0646206818B926602068B4
:10074000284460606068B04201D8012070BD00207C
:10075000FCE7014600200860486001207047000067
:1007600010B502241348B0F8410018B11148B0F890
:100770004300A0B93C211048FFF7D8FFC0B10E4894
:10078000FFF7E7FF0B48B0F8410018B90920FBF765
:1007900079FF02E00A20FBF775FF012408E0054815
:1007A000B0F8410020B10348B0F8430000B1002484
:1007B000204610BDD80700203837002010B503248C
:1007C0000848C078012801D1012403E00548C07819
:1007D00000B900240420FBF73BFF00B102242046AF
:1007E00010BD0000C425002010B50324084800797E
:1007F000012801D1002403E00548007900B9012453
:100800000320FBF725FF00B10224204610BD0000A5
:10081000C42500202DE9F04104460D46002700269E
:100820006078217800EB012086B24948008AB04206
:1008300016D14848007AA84210D1474890F82200C3
:1008400050B1FAF7FAFE28B12A46A11C4348F7F73F
:10085000BCFC76E0222774E0332772E0132770E0B7
:100860003B48408AB04217D13A48407AA84211D159
:10087000394890F8220058B1FAF7DFFE30B12A4625
:10088000A11C36481330F7F7A0FC5AE0222758E0A5
:10089000332756E0132754E02D48C08BB04217D1C0
:1008A0002C48C07BA84211D12B4890F8220058B1A7
:1008B000FAF7C3FE30B12A46A11C28487730F7F773
:1008C00084FC3EE022273CE033273AE0132738E05F
:1008D0001F48008CB04217D11E48007CA84211D19D
:1008E0001D4890F8220058B1FAF7A7FE30B12A4609
:1008F000A11C1A487B30F7F768FC22E0222720E091
:1009000033271EE013271CE01148408CB04217D15A
:100910001048407CA84211D10F4890F8220058B1ED
:10092000FAF78BFE30B12A46A11C0C487F30F7F74E
:100930004CFC06E0222704E0332702E0132700E006
:10094000312717B93046FBF7E5FA3846BDE8F081A4
:100950001EC001080AC001086847002001380020B5
:100960002DE9F04F8DB0044692469B464FF00008AB
:10097000C1460025002600278D48B0F84200042813
:1009800003DA13200DB0BDE8F08F94F80090A07842
:10099000617840EA012571223046711C8EB20DF853
:1009A000002022783046711C8EB20DF8002062784B
:1009B0003046711C8EB20DF80020A2783146701CB2
:1009C00086B20DF80120B9F1010F7BD1A0786178D2
:1009D00040EA01257649B1F842000421FAF727FEE2
:1009E00018B140F20320854215D07149B1F8420098
:1009F0000421FAF71CFE10B1B5F5017F0BD06C494C
:100A0000B1F842000521FAF712FE002849D040F261
:100A10000720854245D1664890F8220000283DD045
:100A2000FAF70BFE80B3A5F20320E8B1012802D04B
:100A3000042827D109E0002702205E494877304684
:100A4000711C8EB20DF800701DE0E078012804DC06
:100A50000027E0785749887000E001273046711C74
:100A60008EB20DF800700EE001205149C8734FF4AA
:100A7000FA70A1F8540000273046711C8EB20DF8B0
:100A8000007000E000BF02E0FFE74FF02208B8F17D
:100A9000000F02D10120484908707CE04FF0330874
:100AA00079E040F20320854205D0B5F5017F02D000
:100AB000001D854203D14FF013086CE002E04FF0B7
:100AC000310868E0B9F1030F30D1A078617840EACD
:100AD00001253749B1F842000421FAF7A8FDE0B139
:100AE000B5F5017F19D1324890F8220090B1FAF79C
:100AF000A4FD60B1B5F5017F07D12E48477F304690
:100B0000711C8EB20DF8007000E000BF43E04FF0A2
:100B1000220840E04FF033083DE0B5F5017F02D1F7
:100B20004FF0130837E04FF0310834E0B9F1020F0D
:100B300028D11F49B1F842000421FAF778FDC0B16D
:100B4000B5F5017F15D11A4890F8220070B1B5F5BE
:100B5000017F09D100270020164948773046711CD3
:100B60008EB20DF8007000E000BF14E04FF03308C3
:100B700011E0B5F5017F02D14FF013080BE04FF003
:100B8000310808E00A480079012804D1002008490A
:100B900008714FF01208ABF80060B8F1000F04D1F3
:100BA000324669465046F7F710FB4046EAE6000039
:100BB00068470020500C00208E0C00204BF65C2073
:100BC000034908804AF65520091D08807047000037
:100BD000B06C004010B500F001F810BD0CB500205D
:100BE000019000904048006840F480303E49086021
:100BF00000BF3D48006800F4003000900198401CA0
:100C00000190009820B94FF6FF7101988842F0D109
:100C10003548006800F4003010B10120009001E078
:100C200000200090009801285CD13048006840F016
:100C300010002E4908600846006820F00300086094
:100C40000846006840F002000860274840682649CE
:100C500048600846406848600846406840F4806044
:100C600048600846C06A224908401F49C8620846D1
:100C7000C06A204908431C49C8620846006840F021
:100C80008060086000BF1848006800F0006000281D
:100C9000F9D01548406820F47C1013494860084694
:100CA000406840F4E81048600846006840F08070F2
:100CB000086000BF0C48006800F000700028F9D000
:100CC0000948406820F0030007494860084640682A
:100CD00040F00200486000BF0348406800F00C008C
:100CE0000828F9D10CBD000000100240002002408D
:100CF00000F0FEFF1408010010B5FFF75FFF10BD04
:100D000010B50A480078072804D0094908698047C7
:100D1000022808D10748416880680A30814200D320
:100D200010BDFEF7F5FB00BFFAE700000426002027
:100D30006C00002048090020014602480172012091
:100D400070470000A40700200146024801710120FD
:100D500070470000A40700200146032903D004299E
:100D600001D0002070470248C1710120FAE700005D
:100D7000A40700200146012902D009B100207047D4
:100D8000014881710120FAE7A407002000220149EF
:100D90000A54704724260020014602484171012070
:100DA00070470000A407002010B5FEF7C3F908B98A
:100DB000002010BDFBF700FF0020134908801DE054
:100DC000114A128802EB4202104B03EB8202516877
:100DD0000F4A5068F7F71DFA58B10B48008800EB2E
:100DE00040000A4901EB8000846804B1A04701205B
:100DF000DFE705480088401C034908800248008856
:100E00001528DDD30020D4E728020020ACBA010861
:100E1000482100201FB500BF2748FDF7F8FD08B1A5
:100E2000012000E00020039000BF2448FDF7EFFD03
:100E300008B1012000E00020029000BF2048FDF72B
:100E4000E6FD08B1012000E00020019000BF1D4830
:100E5000FDF7DDFD08B1012000E00020009003A9AE
:100E60001948FBF755FD08B1012000E000201749A3
:100E7000C87002A914480C38FBF74AFD08B10120DC
:100E800000E000201149087101A90F480C30FBF760
:100E90003FFD08B1012000E000200C494870694680
:100EA00009481830FBF734FD08B1012000E00020AC
:100EB000064988701FBD0000240B0020380B00205D
:100EC000C40B0020D80B002064260020C42500207D
:100ED00070B502460B4600204FF44F410E120546F6
:100EE000401C56550546401C51551E780546401C71
:100EF0005655491C0E120546401C56550546401CC9
:100F000051555E780546401C56559E780546401C56
:100F10005655491C0E120446451CE8B216550446A7
:100F2000451CE8B21155DE780446451CE8B216555A
:100F30001E790446451CE8B21655491C0E1204469B
:100F4000451CE8B216550446451CE8B211555E79B9
:100F50000446451CE8B21655491C0E120446451CB1
:100F6000E8B216550446451CE8B211559E79044670
:100F7000451CE8B21655491C0E120446451CE8B241
:100F800016550446451CE8B21155DE790446451C49
:100F9000E8B21655491C0E120446451CE8B2165517
:100FA0000446451CE8B211551E7A0446451CE8B2B9
:100FB00016555E7A0446451CE8B21655491C0E12B9
:100FC0000446451CE8B216550446451CE8B21155C6
:100FD0009E7A0446451CE8B2165570BD05490A685C
:100FE000C0F802204A68C0F806200A894281897A3E
:100FF00001737047913800202DE9F0410446002329
:10100000002000250027177000BF15E003EBC30781
:1010100004EB47077F786FB103EBC30704EB470787
:101020007F7847EA032C92F8008008F101071770D7
:1010300021F818C05F1CFBB2122BE7DB177807B34F
:1010400000251AE0002011E011F810C0471C11F82B
:101050001770BC4508DD471C31F8176031F810C027
:1010600021F817C021F81060471CF8B217787F1BD1
:101070007F1E8742E8DC6F1CFDB217787F1EAF42EF
:10108000E0DCBDE8F081000010B50948006820B937
:10109000084806F0E1F9064908600548006806F0CE
:1010A0006EFA20B90A210248006806F05BFA10BD0A
:1010B000580100204DB4010810B5F8F70FF820B919
:1010C0000FA004F05BF8002010BDFAF76DFD08B921
:1010D0000020F9E7FAF778FC08B90020F4E7134894
:1010E00090F8380000F0100038B1F9F7B1FD20B9E0
:1010F0000FA004F043F80020E6E70120E4E7000039
:10110000424D5320546865204368617267696E6779
:101110002050686173652053746F70732041626E54
:101120006F726D616C6C790A0D000000200E00205A
:10113000434353204E6F204368617267696E672096
:10114000416C6C6F7765646E0D0000000F4800689D
:10115000401C0E4908600E480068401C0C4908609D
:101160000A4800684FF47A71B0FBF1F201FB1200FB
:10117000012804D107480068401C06490860064859
:10118000007810B90120044908707047F40100206C
:10119000EC010020F8010020F001002030B51648D5
:1011A00000684FF47A72B0FBF2F1B1F1807F01D3A5
:1011B00001201DE021F07F40401E4FF0E0225061F1
:1011C00050170F22002807DA13071D0E0B4B00F0F3
:1011D0000F04241F1D5503E013071C0E084B1C545D
:1011E00000BF00204FF0E022906107201061002036
:1011F00008B100BFFEE730BD0C00002018ED00E094
:1012000000E400E010B5FDF70BF84FF41772024947
:10121000024805F0D3FD10BDF816002000F00108CB
:1012200010B51648006840F00100144908600846EF
:101230004068134908401149486008460068114950
:1012400008400E4908600846006820F480200860C5
:101250000846406820F4FE0048600846006820F018
:10126000A05008604FF47F0088600020C862FFF73C
:10127000B1FC4FF000600449086010BD001002404E
:101280000000FFF0FFFFF6FE08ED00E02DE9F05F43
:101290001048B0F800A0104A0021504603F02AFE82
:1012A0000D480068F7F78CFA804642460B460B481B
:1012B0000B49F7F7B5F9064600220A4BF7F738F95C
:1012C0000446F7F7C1FA8346FBF742FB064908815B
:1012D000BDE8F09F60000020B00000209A99999925
:1012E000999913400000F03F880D002010B50121AE
:1012F000054800F04AF828B101F012FB012102482C
:1013000000F034F810BD0000000400407FB5054631
:101310000C4601210220FEF783FEADF80850ADF81F
:1013200004400020ADF80A00ADF8060001A90E48FF
:1013300000F048F8012211460B4800F037F81D2054
:101340008DF8000001208DF8010003208DF80200C7
:1013500001208DF803006846FDF756FC0121024884
:1013600000F007F87FBD000000040040CA4302827D
:10137000704721B1028842F00102028004E0028835
:101380004FF6FE731A400280704730B502460020C7
:1013900000230024158A05EA0103958905EA010462
:1013A00013B10CB1012000E0002030BD1AB18389D7
:1013B0000B43838102E083898B438381704781855E
:1013C00070470000002202881D4B98420ED01D4B32
:1013D00098420BD0B0F1804F08D01B4B984205D0FB
:1013E0001A4B984202D01A4B984204D14FF68F7391
:1013F0001A404B881A43174B984207D0164B984215
:1014000004D04FF6FF431A40CB881A4302808B88E2
:1014100083850B8803850A4B98420BD0094B984271
:1014200008D00E4B984205D00D4B984202D00D4B80
:10143000984201D10B7A0386012383827047000012
:10144000002C01400034014000040040000800402E
:10145000000C00400010004000140040004001401B
:10146000004401400048014010B51248008888B986
:10147000002011490870114908701149087011497C
:101480000870114908700846017810480088FCF778
:1014900069FB0DE00720094908700D480078401CE1
:1014A0000B49087008460078102801D10020087008
:1014B00010BD0000AC0C0020C80C0020B60C0020B1
:1014C0009F0C0020C40C0020BD0C0020A40C0020A8
:1014D000A20C002010B501202149087000202149EC
:1014E000087021480078012805D12048007810288C
:1014F00001D1FCF70AFB1C480078012803D11B48E6
:101500000078102805D01A48007858B1194800789A
:1015100040B9962018490880012018490870022017
:101520001749087016480078012802D1154800783C
:1015300048B10E48007830B10B480078042804D137
:101540001148008808B900F0FDFC10480078012817
:1015500005D105480078062801D100F0F3FC10BD44
:10156000C00C0020C50C0020B60C00209A0C0020F6
:10157000920C0020910C0020B20C0020C70C00201F
:10158000900C0020930C0020980C00209F0C002051
:1015900070B536480078012866D0354800790128B2
:1015A00004D134480078012800D170BDFCF70CFB51
:1015B000314908803148FCF7C3FA3048007800F020
:1015C000F0002F49087000202E4908802E4800881E
:1015D0002749A1F84200002008712848007800F04F
:1015E0000F0522480078022803D115B901201F49B0
:1015F000087020480078012801D100F0A3FC2048A1
:10160000007820BB1D48007800F00F001E490880BC
:1016100001240CE01948005D1C491A4A12888854BC
:1016200018480088401C17490880601CC4B216483E
:1016300000888442EEDD00F03DFA48B909201449E3
:1016400008700846017810480088FCF78BFA0BE018
:1016500001201049087000200D49087008460178E3
:1016600009480088FCF77EFA00BF9EE7900C002036
:10167000684700209F0C0020AA0C0020CA0C002004
:10168000A60C0020A80C0020A40C0020543B002035
:10169000BD0C0020BF0C002010B51F4800780128A9
:1016A00024D001201D490870FCF78EFA1C490880DF
:1016B0001C48FCF745FA1B48007800F00F04164858
:1016C0000078022803D114B9012013490870164884
:1016D0000078012801D100F035FC00201349087082
:1016E0000120134908701349087114E00F4800786D
:1016F000401CC0B20D49087002280CDB02F086F9CC
:1017000000F064F8002009490870034908700A498C
:1017100008700A49087010BD900C0020C10C002010
:10172000AA0C0020CA0C00209F0C0020D30C002023
:10173000D20C002068470020B60C0020480D002085
:1017400010B51148007838B1104840781049087039
:1017500000F0EAFB0F4908700D4800780E49087048
:101760000C4800780D49087000200D49087000F001
:1017700029FC0B48007818B904200A49087002E0D7
:1017800003200849087010BDC90C0020CA0C0020B5
:10179000920C0020930C0020910C0020940C00204F
:1017A000960C0020B60C002000487047543B0020E7
:1017B00010B505480078012804D1002002490870BE
:1017C00000F050F910BD0000C10C002000200D49B0
:1017D00008700D4908700D4908700D4908700D49D1
:1017E00008700D4908700D4908700D4908700D49C1
:1017F00008700D4908700D4908700D4908700D49B1
:1018000008707047B60C0020900C00209F0C002040
:10181000C30C0020C40C0020C00C0020C10C002010
:10182000C50C0020C60C0020C70C0020C80C0020EE
:10183000BC0C0020C20C002010B507480078FCF753
:10184000EFF90648FCF7C6F9462005490880012053
:101850000449087010BD00009E0C0020CA0C002036
:10186000AE0C0020C50C002010B5044611480480C1
:101870000088072803DC00200F49087002E01020D0
:101880000D49087001200D49087000200C4908809E
:101890000C480078012802D100F054FC09E00C202B
:1018A0000949087008460078FCF784F900200349CC
:1018B000087010BD980C00209A0C0020900C00209D
:1018C0009C0C0020C30C0020BD0C002010B500F0C3
:1018D0003DFE00F037FB10BD10B50A48007820B17E
:1018E000012805D0022809D105E000F091FA06E0B0
:1018F00000F0AAFA03E000F0DDFA00E000BF00BF4C
:1019000010BD0000A30C002010B52E4840782D49D2
:10191000097801F00F0140EA01202B4908800846B0
:1019200000882A4908802848008840F60201884239
:1019300013DD0D20264908700846017822480088EA
:10194000FCF710F902202349087000F083FB002007
:10195000204908702049087032E01B480088082898
:101960002EDB00F0A7F848B909201949087008468D
:10197000017815480088FCF7F5F821E0022411E011
:101980001048005D1549164A128888540F4800888F
:10199000401E0E49088012480088401C10490880EB
:1019A000601CC4B2072CEBDD01200E49087006480C
:1019B0000088FCF7ABF801200B49087000F04AFBE7
:1019C00010BD0000CA0C0020A40C0020AC0C0020AC
:1019D000BD0C0020BC0C0020B60C0020543B0020A5
:1019E000A80C0020A20C00209F0C002010B5184865
:1019F000007800F00F001749088001240CE014481B
:101A0000005D1549154A1288885414480088401C06
:101A100012490880601CC4B20E4800888442EEDD82
:101A200000F048F848B909200D49087008460178C7
:101A300008480088FCF796F808E00020084908707C
:101A40000846017803480088FCF78CF810BD0000B8
:101A5000CA0C0020A40C0020543B0020A80C00203D
:101A6000BD0C002010B50E48007800F0F0000D49C4
:101A7000087000200C4908800C490870094800785B
:101A80000B49C8760748007810B9FFF7AFFF05E0AB
:101A900004480078102801D1FFF736FF10BD000080
:101AA000CA0C0020A60C0020A80C0020BF0C0020AF
:101AB0006847002000202149097831B1102912D04F
:101AC000202918D0302935D12CE01D49098849B189
:101AD0001C490A881A490988491C8A4201DA0020EF
:101AE00000E0012027E017490988082901DA0020D1
:101AF00000E001201FE014490988072907DB11498C
:101B00000988082901DA00200BE0012009E00D49CD
:101B10000A880D490988491C8A4201DA002000E040
:101B2000012008E007490988032901DA002000E0C4
:101B3000012000E000BF00BF70470000A60C00209D
:101B4000A40C0020AA0C0020AC0C00202C49098811
:101B5000072933DA01212B4A1180012016E02A4996
:101B6000095C2A4A2A4B1B88D15429490988491CF7
:101B7000274A118027490988491E264A1180214990
:101B80000988491C1F4A1180411CC8B21C49098898
:101B90008842E4DD1F49098819B901211E4A82F8EB
:101BA000211001211D4A117008211D4A11700121C7
:101BB0001C4A11700021164A118020E01049098842
:101BC00007291CDB012011E00F49095C0F4A104B6B
:101BD0001B88D1540E490988491C0D4A11800D49B2
:101BE0000988491E0B4A1180411CC8B20728EBDD49
:101BF0000849098819B90121074A82F8211070475C
:101C0000B80C0020BA0C0020CA0C0020543B002065
:101C1000A80C0020AC0C002068470020A30C00207A
:101C2000B60C0020C40C002010B52D48008838B92F
:101C300003202C4908700846007800F0D1F84EE0E7
:101C40002948007801284AD10020274908702749EF
:101C500008702748007800F0F00026490870084610
:101C6000007818B108460078102809D106201D49CF
:101C700008700846007800F0B3F8FFF7F3FE2EE096
:101C80001C48007820282AD1FFF714FF38B9092012
:101C9000144908700846007800F0A2F81FE01448C4
:101CA000007800F00F0014490978884210D1002014
:101CB00012490870FFF710FE96200949088001209C
:101CC0000A4908700D48007848B9FFF7CDFB06E0D7
:101CD0000420044908700846007800F081F810BD1F
:101CE000B40C0020BD0C0020C10C0020C80C00204A
:101CF000CA0C0020A60C0020A20C0020A30C00207F
:101D000010B52D4A12882D4B1B889A4220DB2B4A96
:101D10001178012011E02A4A125C2A4B2A4C2488AF
:101D20001A55294A1288521C274B1A80234A1288B6
:101D3000521E224B1A80421CD0B28842EBDD1F4A51
:101D40001288002A36D10122204B83F8212031E06D
:101D5000194A1288194B1B889A422BDA01221C4B14
:101D60001A80012016E0164A125C164B164C248885
:101D70001A55154A1288521C134B1A800F4A1288A2
:101D8000521E0E4B1A80124A1288521C104B1A8097
:101D9000421CD0B2084A12889042E4DD02220D4B68
:101DA0001A7008220C4B1A7001220C4B1A70002278
:101DB000054B1A8010BD0000B80C0020AC0C0020B0
:101DC000CA0C0020543B0020A80C002068470020CB
:101DD000BA0C0020A30C0020B60C0020C40C00207C
:101DE00010B50446214606480088FBF7BBFE0020DC
:101DF00004490870044908700449087010BD0000C7
:101E0000A40C0020B60C00209F0C0020C40C002065
:101E100010B50A48008840F60201081A08490880EF
:101E200008480088072802DBFFF790FE05E0054818
:101E30000088072801DAFFF763FF10BDA80C002017
:101E4000B80C0020AC0C00201248007808BB16E04B
:101E5000114812490988405C1149124A1288885475
:101E600010480088401C0F4908800F480088401E19
:101E70000D49088009480088401C08490880074827
:101E800000880728E4DD0020084908700720084979
:101E900008707047C40C0020CA0C0020BA0C002047
:101EA000543B0020A80C0020AC0C0020A30C002008
:101EB000B60C00201449097821BB1449087816E0B3
:101EC0001349144A1288895C134A144B1B88D15455
:101ED00012490988491C114A11800C490988491E78
:101EE0000A4A11800B490988491C0A4A118009498C
:101EF0000A88411C8A42E3DD0021094A117007214A
:101F0000084A117070470000C40C0020AC0C00207F
:101F1000CA0C0020BA0C0020543B0020A80C002062
:101F2000A30C0020B60C0020054A917831B17F291E
:101F300000DD7F21C8B2421CD0B200E00120704712
:101F4000CA0C002010B514480078092821D2DFE817
:101F500000F005080B0E1114171A1D00FFF728FCDE
:101F600018E000F06BFC15E000F0D6FB12E000F08A
:101F70001BF80FE000F030FB0CE000F099FC09E0EA
:101F800000F02EFC06E0FFF74FFE03E000F098FBA8
:101F900000E000BF00BF10BDB60C002001200149C9
:101FA00008707047C30C002010B500F00BF8034810
:101FB000007810B904200249087010BD960C00206A
:101FC000B60C002010B50A48007820B1012805D0D1
:101FD000022809D105E000F0CBF906E000F0EEF9A7
:101FE00003E000F02DFA00E000BF00BF10BD0000CC
:101FF000960C002012490988C1F3032141F0100119
:10200000104A11700E4909785170022011E00E49F2
:102010000E4A1288895C0B4A11540C490988491CE4
:102020000A4A118006490988491E054A1180411C47
:10203000C8B20728EBDD0821054A1170704700007F
:10204000980C0020CA0C0020543B00209C0C00205F
:102050009E0C002010B51848007840F03000174959
:1020600008700020487014208870002014490880EF
:10207000032014490870032404E0CC200F490855BC
:10208000601CC4B2072CF8DD08200E49087000203F
:10209000FBF7CCFD0B480078FBF7C2FD0748FBF7C8
:1020A00099FD06200849087046200849088001204B
:1020B0000749087010BD0000BC0C0020CA0C0020AD
:1020C000A00C00209E0C0020B60C0020B00C0020BC
:1020D000C60C0020164A1278164B1A7001200121F6
:1020E0000EE0154A154B1B88D25C124B5A54134A0A
:1020F0001288521C114B1A80421CD0B24A1CD1B219
:102100000B4A12889142ECDD094A1278521C0C4BA2
:102110001A7007280ADC04E0CC22064B1A54421C31
:10212000D0B20728F8DD0822054B1A70704700006E
:10213000980C0020CA0C0020543B00209C0C00206E
:102140009E0C002010B51048007810B9FFF7C2FFB0
:1021500005E00D480078102801D1FFF74BFF012062
:102160000A4908700A480078FBF75AFD0948FBF74E
:1021700031FD0120084908704620084908800120E7
:102180000749087010BD00009A0C0020950C002033
:102190009E0C0020CA0C0020B60C0020AE0C0020C3
:1021A000C50C002010B52A48008807282BDA01202A
:1021B00028490880012416E0274828490988405CFE
:1021C0002749085525480088401C2449088025488F
:1021D0000088401E234908801E480088401C1D4975
:1021E0000880601CC4B21A4800888442E4DD0120E3
:1021F0001D49087000201D490870FBF725FD0020CF
:102200001649088023E01248008807281FDB0124B4
:1022100011E0114811490988405C114908550F48DF
:102220000088401C0D4908800E480088401E0D495A
:102230000880601CC4B2072CEBDD08200C49087034
:10224000FFF7FAFA04200B49087000F065F910BD99
:10225000B80C0020BA0C0020543B00209C0C00203D
:10226000CA0C0020980C0020960C0020C30C002003
:102270009E0C0020B60C002070B53348008833490E
:10228000098888422DDB012530480678012413E0B7
:102290002F4830490988405C2F4908552D4800884F
:1022A000401C2C49088029480088401E2749088086
:1022B000681CC5B2601CC4B2B442E9DD2748067090
:1022C00004E0CC2024494855681CC5B2072DF8DD30
:1022D000082022490870FFF7AFFA0420204908704F
:1022E00030E0194800881949098888422ADA012013
:1022F0001C490880012416E0154816490988405CED
:102300001549085513480088401C124908800F4899
:102310000088401E0D49088012480088401C114961
:102320000880601CC4B2084800888442E4DD0220B2
:102330000D49087000200D490870FBF785FC00204E
:102340000449088070BD0000B80C0020980C0020E3
:10235000543B00209C0C0020CA0C00209E0C002046
:10236000B60C0020BA0C0020960C0020C30C0020F4
:1023700010B50D48007840F020000C4908700C485A
:10238000008840F60201081A0A4908800A480088B5
:10239000072802DBFFF706FF05E00748008807284B
:1023A00001DAFFF769FF10BD950C0020CA0C002070
:1023B0009C0C0020B80C0020980C002010B5174889
:1023C0000078012828D116E0154816490988405C94
:1023D0001549164A1288885412480088401C114931
:1023E000088013480088401E114908800F48008863
:1023F000401C0E4908800D4800880728E4DD0820AD
:102400000C490870FFF718FA00200B4908700420E7
:102410000A49087000F080F810BD0000C30C0020CD
:10242000543B00209C0C0020CA0C0020BA0C002059
:10243000980C00209E0C0020960C0020B60C00206A
:1024400010B52048007801283AD11F480478007858
:102450001E49097808441E49087018E01D481E49A5
:102460000988405C1D49184A128888541A48008817
:10247000401C1949088015480088401E13490880EF
:10248000601CC4B210480088401C0F4908800E48E8
:1024900000880F4909788842E0DB04E0CC200F492E
:1024A0000855601CC4B2072CF8DD082008490870E4
:1024B000FFF7C2F900200A49087004200949087092
:1024C00010BD0000C30C0020BA0C0020980C0020A6
:1024D0009E0C0020543B00209C0C0020CA0C0020C5
:1024E000960C0020B60C002010B504462046FBF7E1
:1024F00061FB002004490870044908700449087011
:102500000449087010BD0000B60C0020900C00209B
:10251000C30C0020C00C002009480078401C08496A
:10252000087008460078102801D10020087005487E
:10253000007820B104480078401E034908707047B5
:10254000950C0020920C0020910C00201A48007875
:10255000012808D119480088002804DD17480088A0
:10256000401E1649088016480078012808D11548F1
:102570000088002804DD13480088401E11490880A7
:1025800011480078012808D110480088002804DD8F
:102590000E480088401E0D4908800D48007801282B
:1025A00008D10C480088002804DD0A480088401E35
:1025B0000849088070470000C50C0020AE0C0020C0
:1025C000C60C0020B00C0020C70C0020B20C00206C
:1025D000C80C0020B40C002010B52C48008838B975
:1025E00001202B49087008460078FFF77DFF4CE07A
:1025F00028480078012803D027480078012844D1D2
:10260000002026490870234908702548008838B9F9
:1026100000201F49087008460078FFF765FF34E086
:102620002048007848B12048007830B900201F4980
:10263000087002201E49087027E01E48007818B173
:102640001C48007801280CD1FFF7BCFC1A48007820
:1026500018B900201049087017E001200E490870D1
:1026600013E014480078022803D1032010490870B1
:102670000BE010480078022807DD10480078401E63
:102680000E49087005200A49087010BDAE0C0020E4
:10269000BD0C0020C00C0020C20C0020C50C002086
:1026A000980C0020920C0020910C0020C90C0020F6
:1026B000B60C0020930C0020960C0020940C0020F7
:1026C00010B51148008838B9032010490870084631
:1026D0000078FFF785FB15E00D48007801280AD146
:1026E00000200B4908700B20084908700846007844
:1026F000FFF776FB06E0FFF7EFF80648007808B929
:10270000FEF7B2FE10BD0000B40C0020BD0C00208E
:10271000C10C0020A30C002010B52B48008838B94C
:1027200002202A49087008460078FFF7DDFE49E0DC
:1027300027480078012845D1002025490870254800
:10274000007800F0F000244908700846007830282E
:1027500038D10020214908701E48007800F00F048D
:10276000FFF7A8F938B90920184908700846007819
:10277000FFF7BAFE26E0032C07DB0520134908709B
:1027800008460078FFF7B0FE1CE0022C07D10820B5
:102790000E49087008460078FFF7A6FE12E0012CEB
:1027A0000DD107200949087008460078FFF79CFE04
:1027B00095200549088001200849087002E00CB9FD
:1027C000FEF7BEFF10BD0000B20C0020BD0C0020C3
:1027D000C10C0020CA0C0020A60C0020C70C002051
:1027E00010B50F48007801280ED100200C49087060
:1027F0000C49087007200C49087096200B49088086
:1028000001200B49087009E00A48008830B901200E
:102810000949087008460078FFF7E2FA10BD000089
:10282000C00C0020C60C0020B60C0020B40C002008
:10283000C80C0020B00C0020BD0C002010B51548BD
:10284000008838B901201449087008460078FFF75D
:102850004BFE1DE011480078012819D100200F49D6
:1028600008700F4908700F48007838B900200A49ED
:10287000087008460078FFF737FE09E0094800783D
:10288000102805D101200849087002200749087066
:1028900010BD0000AE0C0020BD0C0020C00C0020BC
:1028A000C50C00209A0C0020C90C0020B60C00209A
:1028B00008480078401E074908700846007801283B
:1028C00006DC0320044908700448007801490870B8
:1028D00070470000940C0020B60C0020930C0020E0
:1028E0000246002321B90D4800681060012070479E
:1028F0000A4803681068984205D81068181A884278
:1029000009D30120F3E71068C0F1FF301844884272
:1029100001D30120EBE70020E9E70000F4010020EB
:1029200010B50E48407B012816D03220F9F790FEF2
:1029300090B92A20F9F78CFE70B90948006801881F
:102940000848FEF73CFD0649096848688047044886
:10295000006880680249086010BD00004809002036
:1029600080370020000400404F48007801280AD139
:102970004E48C068401C4D49C860012008700020C6
:102980004949087000E070474848C0680521B0FB1D
:10299000F1F201FB120030B94448C06818B10120BF
:1029A0004249487000E0EEE74048C0680A21B0FBA9
:1029B000F1F201FB120028B93C48C06810B10120B7
:1029C0003A4988703948C0681421B0FBF1F201FB24
:1029D000120028B93548C06810B101203349C870C9
:1029E0003248C0683221B0FBF1F201FB120028B975
:1029F0002E48C06810B101202C4908712B48C068CE
:102A00006421B0FBF1F201FB120028B92748C0682D
:102A100010B10120254948712448C0684FF4FA716B
:102A2000B0FBF1F201FB120028B92048C06810B1D8
:102A300001201E4988711D48C0684FF47A71B0FBAF
:102A4000F1F201FB120028B91848C06810B101204A
:102A50001649C8711548C06840F2DC51B0FBF1F26C
:102A600001FB120028B91148C06810B101200F49BC
:102A700008720E48C0684FF4FA61B0FBF1F201FB36
:102A8000120028B90948C06810B1012007494872EE
:102A90000648C06841F27071884202D300200349A1
:102AA000C86000BF6FE70000F0010020E8160020BA
:102AB0000FB5184800880A2802DB00201549088055
:102AC00014480288001D00EB0210009901609DF877
:102AD000041010480288001D00EB021001719DF8DF
:102AE0000D100C480288001D00EB021041730948CC
:102AF0000188001D00EB0110DDF8051040F8051FEE
:102B0000DDF80910416003480088401C0149088035
:102B10000FBD00005843002010B51748006800B1F1
:102B200010BDF8F73BFC00B9FAE71BE013484088FA
:102B30000A2802DB00201149488010484188001D06
:102B400000EB011494E80F0001F017FB01200C4981
:102B50008870002081F82A0008484088401C0749F6
:102B6000488005E005480088044949888842DDD14D
:102B700000BF00BFD4E700004C0C002058430020E9
:102B80006847002010B504462146054801F059FA6F
:102B900000BF0348008800F080000028F9D010BD75
:102BA000004C004010B540F22551394801F089F938
:102BB000F8B1374801F040FAC4B236480088C82856
:102BC00008DA344801880088401C324A10803248B4
:102BD000445402E000202F4908800A2C04D1FEF75B
:102BE000E3F8FDF7A5FC10BD40F22551284801F09F
:102BF00040F940F22441264801F063F948B1FDF75D
:102C000097FC234801F018FA40F22441204801F0D3
:102C100030F940F227711E4801F053F920B140F21B
:102C200027711B4801F025F940F22661184801F090
:102C300048F920B140F22661154801F01AF908213F
:102C4000134801F031F9012806D10821104801F09C
:102C500007F90F4801F0F0F904210D4801F024F9BB
:102C6000012806D104210A4801F0FAF8084801F0C9
:102C7000E3F90221064801F017F9012806D10221E3
:102C8000034801F0EDF8024801F0D6F900BFAAE7C9
:102C9000004C00401E0200204E1E002010B540F2E5
:102CA0002551334801F00DF9E8B1314801F0C4F97C
:102CB000C4B230480088C82808DA2E480188008845
:102CC000401C2C4A10802C48445402E00020294922
:102CD00008800020294908802949087040F22551C0
:102CE000234801F0C6F840F22441214801F0E9F8F8
:102CF00050B11F4801F0A0F901202149087040F2AD
:102D000024411B4801F0B5F840F22661184801F053
:102D1000D8F820B140F22661154801F0AAF8082140
:102D2000134801F0C1F8012806D10821104801F02C
:102D300097F80F4801F080F904210D4801F0B4F82C
:102D4000012806D104210A4801F08AF8084801F058
:102D500073F90221064801F0A7F8012806D10221E3
:102D6000034801F07DF8024801F066F910BD00004B
:102D70000050004024020020161F002020020020E6
:102D80002202002010B50948007F70B10748C07FBB
:102D900010280AD10549887F00F0AAFA00200349CB
:102DA0000877FF210248F5F729FA10BD684700208F
:102DB000543B002010B50748007F50B10548C07F44
:102DC000112806D103482B3000F03EFB00200149BA
:102DD000087710BD6847002010B50A48007F78B119
:102DE0000848C07F14280BD1032106482B3000F07F
:102DF00087FB002003490877FF210348F5F7FEF918
:102E000010BD000068470020543B002010B5064864
:102E1000007F40B10448C07F192804D100F014F9A4
:102E200000200149087710BD6847002010B506480A
:102E3000007F40B10448C07F222804D100F0AAF9E5
:102E400000200149087710BD6847002010B51548DB
:102E5000007F28B31348C07F272821D1114890F85C
:102E60002B00022809D0104A0E492B31012000F016
:102E70008BFB00200B49087712E00A4890F82B00E2
:102E800002280DD1084A07492B3100F07DFB0020B4
:102E90000449087781F8210003480021016041605E
:102EA00010BD000068470020000D002010B50A4842
:102EB000007F78B10848C07F28280BD1022106483E
:102EC0002B3000F079FC002003490877FF210348EC
:102ED000F5F794F910BD000068470020543B00202E
:102EE00010B50A48007F78B10848C07F2E280BD162
:102EF00007480088401E81B2064800F07FF9002094
:102F0000024981F82100087710BD000068470020C1
:102F1000A80C0020553B002010B50A48007F78B16E
:102F20000848C07F31280BD1032106482B3000F020
:102F3000CDFC002003490877FF210348F5F75EF92F
:102F400010BD000068470020543B002010B5074822
:102F5000007F50B10548C07F3E2806D103482B3082
:102F600000F08CF900200149087710BD6847002067
:102F700010B50A48007F78B10848C07F85280BD17A
:102F8000012106482B3000F0DBFC002003490877C4
:102F9000FF210348F5F732F910BD00006847002013
:102FA000543B00208178064A1170C1785170114657
:102FB0000978491C117011464978891C5170704775
:102FC000000D002010B50948007801280DD10748F0
:102FD00040780C2806DA05484078054951F8204029
:102FE000A04702E000200149087010BD080D002034
:102FF0000C0D002010B501200249087000F006FDFC
:1030000010BD0000080D002010B500200249087016
:1030100000F0FCFC10BD0000080D0020704700000F
:10302000012008494877002081F8220088714874FF
:10303000A1F8400081F8240081F8250081F82700DC
:10304000704700006847002070B500240025002666
:103050004D484078012870DD19204B490870002048
:1030600048704A48B0F84200022878DB474890F898
:103070002B0000F07F060B2E67D2DFE806F0660615
:103080000745256626666666460000BF3046F8F7A7
:10309000BBFAB8B13D49B1F842000321F8F7C7FACD
:1030A00070B13A4A2B3231463948F9F76FFF04467E
:1030B00024B137492046FAF7E7FD04E0312502E064
:1030C000132500E0122549E000BF3046F8F79CFACE
:1030D000C0B12E49B1F842000621F8F7A8FA78B13C
:1030E0002A4A2B3231462A48F9F750FF0446032C6E
:1030F00004DD27492046FAF7C7FD04E0312502E048
:10310000132500E0122529E000BF3046F8F77CFACD
:10311000C8B11E49B1F842000221F8F788FA80B11F
:103120001A4A2B3231461A48F9F730FF044634B1B7
:1031300017492046FAF7A8FD06E023E00FE0312505
:1031400002E0132500E0122508E01048B0F8420024
:10315000022801DA132500E0122500BF00E0132544
:10316000122D01D0312D04D108480079012800D05A
:1031700000251DB129461920FAF768FD0A200349E8
:10318000A1F8460070BD0000500D002068470020E7
:10319000C849002070B50024002515484078012852
:1031A00024DD1449B1F842000321F8F740FA98B140
:1031B0001148F9F793FF0546032D04DB0E49284615
:1031C000FAF762FD09E00B480079012805D10020DB
:1031D00008490871312400E013241CB12146222043
:1031E000FAF734FD1E200349A1F8460070BD000027
:1031F000500D002068470020C84900202DE9F0410B
:1032000004460D46002600271948407801282CDD89
:1032100018480079012828D11649487F0022032147
:10322000F8F7D2F9B8B1032D01DA132714E0A81E7C
:1032300081B22046FDF7EEFA064656B96E200E49D9
:10324000087020784870607888700320FAF71CFDB9
:1032500002E0374600E07F271FB139462E20FAF7FB
:10326000F5FC28200349A1F84600BDE8F0810000E4
:10327000500D002068470020C849002070B5044662
:10328000002500261748407801282ADD1649B1F8A4
:1032900042000221F8F7CBF9C8B1207800F07F0690
:1032A00066B92078F8F7BCF990B17E200F49087014
:1032B000207848700220FAF7E7FC09E00A48007914
:1032C000012805D1002008490871122500E01325C6
:1032D0001DB129463E20FAF7B9FC0A200249A1F89F
:1032E000460070BD500D002068470020C8490020EE
:1032F0002DE9F04105460227002600244F4840787A
:1033000001287CDD10204D490870002048704C4990
:10331000B1F842000221F8F78AF900287ED005F0C2
:103320007F04012C03D0022C01D0032C6DD1444822
:10333000407F03281AD1022C18D141480079012876
:103340006DD1F8F77AF978B13D48C07B60B13C485F
:103350004477FDF7D1FC0120394908730870C82073
:1033600081F8200078265AE0222658E03448407F31
:10337000012801D1022C05D03148407F022807D115
:10338000032C05D12E480079012848D17E2646E03D
:10339000032C03D0012C01D1FAF740FF012C02D1FC
:1033A00000202749C8732648447700202449A1F803
:1033B000400081F82200887148740846407F032845
:1033C00001D1032C07D000201D4981F8240081F889
:1033D000250081F827002846F8F722F9F8B1502097
:1033E0001849087008464570002088703220C8705F
:1033F00001200871F42048710627384602E01BE0DE
:103400000CE002E0FAF740FC09E00D4800790128E1
:1034100005D100200A490871122600E013261EB1CA
:1034200031461020FAF712FC0A2004498880084629
:1034300080880349A1F84600BDE8F081500D0020C6
:1034400068470020C849002070B5044600250026C2
:103450002748407801284ADD1120254908700020BE
:1034600048701E2088802349B1F842000221F8F7F5
:10347000DEF8002831D0207800F07F063046F8F7DB
:10348000BBF808B3F8F7D9F8E0B12078F8F7C8F836
:1034900038B1512018490870207848700220FAF796
:1034A000F3FB16480079012805D100201349087163
:1034B00011490870487001200E490870C82081F831
:1034C00020000BE0222509E00A480079012805D1F7
:1034D000002008490871122500E013251DB1294676
:1034E0001120FAF7B3FB0A200249A1F8460070BD8B
:1034F000500D002068470020C849002030470020B8
:103500002DE9F04104460F4600251C48407801286B
:1035100032DD1420194908701E20888020780004AC
:10352000617800EB0120A17846181549B1F84200F6
:103530000421F8F77CF8A8B16FF07F40864208D1EB
:10354000F8F77EF854200F4908700120FAF79CFB29
:1035500009E00B480079012805D1002008490871CD
:10356000312500E013251DB129461420FAF76EFB22
:103570000A200349A1F84600BDE8F081500D002063
:1035800068470020C84900202DE9F04180460C46DC
:1035900015460026FF2782484078012872DD8148C1
:1035A000007901286ED17F49487F01221146F8F742
:1035B0000BF8002867D02078012842D100207A49F2
:1035C00008707849B1F842000221F8F730F8A8B342
:1035D0007448C078012801D13726D4E067207349A8
:1035E0000870207848706F4890F82200012808D1B0
:1035F0006C488079012804D108460021C0F80210E7
:103600000DE06848407C50B96948F9F7A9FC0120F1
:1036100064494874654866490968C0F80210012089
:10362000614908705F49887167205D490870002012
:1036300048705E490620FAF727FBA4E0FFE713264F
:10364000A1E0207802287BD1002056494874B1F8C7
:1036500042000621F7F7EBFF002872D0514890F89E
:103660002800032802DC5048007868B94D4890F8DB
:103670002800032800DB36264B4800780028ACD110
:10368000242680E08AE07DE047480078012802D1C6
:1036900000204549087045480021016081800422CE
:1036A0004349F4F7CFFD00285BD02178491EC8B20A
:1036B000404A3F49F9F7E0FB0746002F4FD16078B9
:1036C0002870A0786870E078A8702079E8700422EB
:1036D00038492846F4F7B6FDF8B90020314981F899
:1036E0002800672031490870207848702078022827
:1036F00001D1012000E002202A4981F8230067203F
:1037000027490870002048700120264981F82200CE
:1037100026490220FAF7B8FA24E0224890F8280057
:10372000FF2806DA1F4890F82800401C1D4981F840
:1037300028001C4890F82800022803DC352611E0F8
:1037400017E014E0174890F8280003280AD136261D
:103750000A20144981F829000120C87002E01226CD
:1037600000E0242612480021016081800BE013262E
:1037700009E00C48B0F84200022801DA132602E002
:10378000122600E07F261EB131462720FAF75EFAA6
:103790001E20034988800349A1F84600BDE8F08156
:1037A000500D0020684700205E0D0020C849002011
:1037B000560D00205A0D00202DE9F04104468846A0
:1037C00000270025002668203D4908703D484078C4
:1037D000012873DD28203B4908701E2088803A4963
:1037E000487F01221146F7F7EFFE002855D03649F1
:1037F000B1F842000321F7F71AFF00284BD0F7F782
:103800001CFF002845D0207800F07F0566780DB1B8
:10381000032D35D1012E01D0032E28D16DB9012EF3
:1038200004D10020284981F8240015E00020264911
:1038300081F8240081F825000EE0032D0CD1012E23
:1038400004D10120204981F8240005E001201E490F
:1038500081F8240081F825002078F7F7E1FE20B3F5
:103860002078174948700220FAF70EFA1DE0164832
:103870000079012819D1002013490871312714E07B
:1038800011480079012810D100200F490871122732
:103890000BE0222709E0132707E00B4800790128F5
:1038A00003D10020084908717F271FB1394628201D
:1038B000FAF7CCF90A200449A1F84600BDE8F081E6
:1038C000C8490020500D002068470020F8B5054683
:1038D0000E4600240020009016484078012827DD7D
:1038E0003120144908701E2088801348007901286F
:1038F0001ED11149487F01221146F7F765FE38B104
:103900006B460E4A31462846FDF72AF8044600E089
:103910007F2424B121463120FAF798F904E00749C1
:10392000BDF80000FAF7B0F90A200349A1F84600F3
:10393000F8BD0000500D002068470020C849002055
:103940002DE9F04104460F46002600252C4840781A
:10395000012853DD85202A4908701E2088802949C6
:10396000487F01221146F7F72FFE002835D0254960
:10397000B1F842000221F7F75AFE60B3F7F75DFE97
:1039800008B9222631E0207800F07F05012D01D012
:10399000022D17D1012D04D100201A4981F82700EA
:1039A00003E00120174981F827002078F7F738FE57
:1039B000D8B1C52014490870207848700220FAF761
:1039C00063F912E00F48007901280ED100200D495B
:1039D0000871122609E0132607E00A480079012839
:1039E00003D10020074908717F261EB1314685208A
:1039F000FAF72CF90A200349A1F84600BDE8F08146
:103A0000500D002068470020C849002000200449CC
:103A1000087002204870012088700020888070475C
:103A2000500D002010B50848007F58B10649C87FE6
:103A300000F014F8002004490877C877FF210348F4
:103A4000F4F7DCFB10BD000068470020543B002069
:103A500010B50446FFF7D8FA10BD000070B5054652
:103A600000240B484078012810DD0A48007901281D
:103A700003D100200749087111241CB121462846B2
:103A8000FAF7E4F80A200349A1F8460070BD0000E7
:103A9000500D0020684700201E2001498880704793
:103AA000500D002070B505460C46054800782728C3
:103AB00005D16078012802D12046FFF773FA70BD66
:103AC000500D00202DE9F04107460E4614464EBB2E
:103AD0003F484078012825D13D4800784030217882
:103AE000884207D121463846FFF7DCFF02203849DB
:103AF00048706BE020787F2868D13548007861787D
:103B0000884263D1A078782805D1FFF7C5FF04204B
:103B10002F4948705AE0A078FFF79AFF03202C49FC
:103B2000487053E0002E44D129484078022840D103
:103B30002078102805D10220254948706078254951
:103B4000887720782349C877002518E02248405D0F
:103B50002049C97F884210D11E48C07F342803D035
:103B60001C48C07F362805D11C48008820B91C4855
:103B7000457001E01A48457003E0681CC5B20C2D81
:103B8000E4DB00BF0C2D02D10B2015494870142135
:103B900010482B30F4F732FB1422611C0D482B30F7
:103BA000F4F713FB01200B4908770846A0F8427090
:103BB0000CE0092E0AD10B480078012806D100201C
:103BC00008490870FF210848F4F718FBBDE8F081A8
:103BD000500D0020684700208EC00108AC0C00206A
:103BE000080D0020D20C0020543B00200120014988
:103BF00048707047500D002010B540F225511D4807
:103C000000F05FF910B31B4800F016FAC4B21A486E
:103C1000008800F40040C8B91748008800F48040CC
:103C200060B10A2C03D000201349088020E012481C
:103C3000008840F400401049088019E00D2C06D19E
:103C40000D48008840F480400B49088010E00A4885
:103C50000088C0F30D0009490C5407480088401C37
:103C60000549088008460088C72801DD0020088033
:103C700010BD0000003801400E020020C01B0020D3
:103C800010B504462146054800F0DBF900BF0348A3
:103C9000008800F080000028F9D010BD00440040EA
:103CA00010B540F22551304800F00BF9C0B12E4854
:103CB00000F0C2F9C4B22D480088FE2808DA2B486B
:103CC00001880088401C294A10802948445402E099
:103CD00000202649088040F22551234800F0C9F809
:103CE00040F22441204800F0ECF850B11E4800F0AA
:103CF000A3F901201F49087040F224411A4800F03E
:103D0000B8F840F22661184800F0DBF820B140F224
:103D10002661154800F0ADF80821134800F0C4F8FA
:103D2000012806D10821104800F09AF80E4800F04A
:103D300083F904210C4800F0B7F8012806D10421CA
:103D4000094800F08DF8084800F076F9022106488D
:103D500000F0AAF8012806D10221034800F080F8FB
:103D6000014800F069F910BD004400401002002035
:103D7000881C00201202002010B540F22551334863
:103D800000F09FF8E8B1314800F056F9C4B230486D
:103D90000088C82808DA2E4801880088401C2C4A70
:103DA00010802C48445402E000202949088000205B
:103DB000294908802949087040F22551234800F01C
:103DC00058F840F22441214800F07BF850B11F48D8
:103DD00000F032F901202149087040F224411B48CB
:103DE00000F047F840F22661184800F06AF820B168
:103DF00040F22661154800F03CF80821134800F015
:103E000053F8012806D10821104800F029F80F487E
:103E100000F012F904210D4800F046F8012806D1FF
:103E200004210A4800F01CF8084800F005F90221B6
:103E3000064800F039F8012806D10221034800F0B5
:103E40000FF8024800F0F8F810BD000000480040EC
:103E500018020020861D00201402002016020020F7
:103E600001F40072B2F5007F00D100BFCA430280A6
:103E7000704710B50022002340F66A14A14200D119
:103E800000BF0A1201249440A3B2DC43048010BD99
:103E900021B1828942F40052828104E082894DF688
:103EA000FF731A408281704702460020B1F5007FFF
:103EB00000D100BF13880B400BB1012000E00020AF
:103EC000704770B50246002400230025002040F60C
:103ED0006A16B14200D100BFC1F3421501F01F03C1
:103EE000012606FA03F3012D02D19689334006E03C
:103EF000022D02D1168A334001E0968A33400C121B
:103F0000012606FA04F41688344013B10CB10120DE
:103F100000E0002070BDF0B5034600240026002517
:103F2000002040F66A17B94200D100BF1846C1F31D
:103F3000421401F01F06012707FA06F5012C01D1F2
:103F40000C3004E0022C01D1103000E014301AB122
:103F500007682F43076002E00768AF430760F0BDC2
:103F60002DE9F04786B005460E460024A24600BF64
:103F7000A1460027B08900B100BF2F462C8A4CF61D
:103F8000FF700440F08804432C82AC894EF6F31095
:103F90000440B08831890843718908430443AC81E7
:103FA000AC8A4FF6FF400440B0890443AC8201A8BC
:103FB000FCF76CF81F48874202D1DDF810A001E041
:103FC000DDF80CA0A88900F4004040B10AEBCA005B
:103FD00000EB0A1031684900B0FBF1F807E00AEB8A
:103FE000CA0000EB0A1031688900B0FBF1F86420C8
:103FF000B8FBF0F004012009642101FB1089A889B5
:1040000000F4004040B1322000EBC900B0FBF1F0F9
:1040100000F00700044308E0322000EB091064219F
:10402000B0FBF1F000F00F0004432C8106B0BDE8B6
:10403000F08700000038014001468888C0F308007E
:104040007047C1F308028280704710B500F072F922
:10405000FBF742FF10BD10B500F01AFB10BD0000C9
:1040600006480088064908600448001F008809883F
:1040700040EA01400249086070470000BC6C004003
:10408000D40C002070B504460D461646324629462B
:10409000204603F0B5FC70BD70B504460D461646CB
:1040A00032462946204603F0EEFC70BD11490968EE
:1040B00051B94FF0E02189690E4A11601146096833
:1040C0000D4A51430B4A11604FF0E0218969094ABA
:1040D000126888180749096843F285621144054A45
:1040E000116080B21146098801EB810140EA01406C
:1040F00070470000DC0C00200DE37A0570470000DB
:1041000000200349097801F0010101B10120704745
:10411000500C0020002003490978C1F3400101B18F
:1041200001207047500C0020002003490978C1F39A
:10413000001101B901207047500C002001460020F9
:1041400040F2B472914200D1012070470FB41FB504
:10415000069800909DF822008DF804009DF8042038
:104160000DF123010DF10500F4F72FF89DE80F0084
:1041700000F0F8FA1FBC5DF814FB0FB585B0002005
:104180008DF80800059800909DF818008DF80A0039
:1041900000208DF809009DF80A200DF119010DF19C
:1041A0000B00F4F712F8684603F01CFA09B000BDE2
:1041B00010B50648007840B9012004490870FAF7A4
:1041C00093FDF7F719FDF7F741FE10BDE00C002055
:1041D00010B53C48C2793C4801683C48F3F7F5FF0C
:1041E000384802783AA139486B38F3F7EEFF354882
:1041F00042783BA135485D38F3F7E7FF31488278D4
:104200003AA132485138F3F7E0FF2E4802793AA13B
:104210002E482B38F3F7D9FF2A48C27839A12B480A
:104220004538F3F7D2FF2748427933A12748213890
:10423000F3F7CBFF2348827939A124481738F3F7E5
:10424000C4FF2048827A38A120485F30F3F7BDFFD1
:104250001C48017A1D480A30F3F7D0FF00201B49A3
:104260006B3981F8E800002118486B3880F8E910B4
:104270008C2016496B3981F8EC00A02113486B386B
:1042800080F8ED10142011496B3981F8F0005021AD
:104290000E486B3880F8F11013200C496B3981F807
:1042A000F400882109486B3880F8F5101920074977
:1042B0006B3981F8F800192104486B3880F8F9103F
:1042C00010BD00000AC00108D40C0020F737002000
:1042D000323130393134302D535A30310000000042
:1042E0003839323620202020202000004443552039
:1042F000202020202020000048573A432E312E3025
:104300000000000053573A312E30302E435F3234D4
:10431000303431315F383932365F303000000000E0
:10432000413430553436000052325830303030315C
:104330000000000010B59F48007820F00100401CEC
:104340009C4908709C4948689C49F3F7E0FF044683
:10435000F4F709FA974948729948007C087200BF3F
:104360009848808F01129348817200BF954890F859
:104370003C00C1B28F48C1728F488089010A8D48C4
:1043800001738D48017B8B4841738F480078072863
:1043900003D10121874881730BE08C49086980476C
:1043A000022803D102218348817302E00021814861
:1043B00081738748C078012803D100217D480174AA
:1043C0000DE08348C07818B901217A48017406E0ED
:1043D0000420F8F73DF910B10221764801747C48B9
:1043E0000079012803D101217248C1730DE078489A
:1043F000007918B900216F48C17306E00320F8F76F
:1044000027F910B102216B48C173704908687149DE
:10441000F3F77DFF0446F4F7A6F9010A65484174F5
:104420006A4908686B49F3F772FF0446F4F79BF991
:10443000C1B2604881746248807B08B9012100E004
:1044400000215C48C1740120F8F702F9C043C04361
:104450005849097860F3041156480170007820F03B
:104460002000544908703320F8F7F2F8C043C043E5
:104470005049097860F386114E4801703420F8F7EE
:10448000E7F8C043C0434B49097860F3C711494876
:1044900001703020F8F7DCF8C043C0434549497843
:1044A00060F30001434841703120F8F7D1F8C04370
:1044B000C0434049497860F341013E4841700320C0
:1044C000F8F7C6F8C043C0433A49497860F382011F
:1044D000384841700320F8F7BBF8C043C043354962
:1044E000497860F3C301334841700420F8F7B0F80D
:1044F000C043C0432F49497860F304112D484170EF
:104500000420F8F7A5F8C043C0432A49497860F36E
:104510004511284841702E48407810B92C488078C1
:1045200008B1012000E000202249497860F386119B
:10453000204841703520F8F78BF8C043C0431D492F
:10454000497860F3C7111B4841703620F8F780F8AE
:10455000184988701848808988801D4800788871BB
:104560001A49486880471349C8711B4800780228D7
:1045700006DA0846007820F00200801C087005E08A
:104580000C48007820F002000A49087012480078B0
:10459000022807DD0748007820F00400001D0549C7
:1045A000087005E00348007820F004000149087015
:1045B00010BD000088380020880D00200000204138
:1045C00048090020D8070020042600206C000020A5
:1045D000C425002000401C46D80C00200E4890F84E
:1045E000EC000E49C8700C4890F8ED0008710A48BC
:1045F00090F8F100084991F8F01000EB012007490C
:10460000C880054890F8F500034991F8F41000EBD4
:1046100001200249088170478C370020500C00208F
:1046200030B585B01648006816490968884224D01C
:104630001348144909680160002500240FE004EBC9
:10464000C401114810F81100092806D1601CC2B23B
:104650002846691CCDB20DF80020601CC4B2122C93
:10466000EDDB0A48857212210B30F3F7C7FD2A46AD
:10467000694606480B30F3F7A8FD05B030BD0000D1
:10468000840C0020740C0020A8380020500C00205E
:1046900010B52D48007830B9FFF79AFDFEF7C0FC41
:1046A00001202949087029480078F0B1274890F87E
:1046B000200038B1254890F82000401E234981F899
:1046C000200011E000202149087000BF2048006848
:1046D00000F4E0601F490843001D1D490860BFF356
:1046E0004F8F00BF00BFFEE710BD1B480088401C75
:1046F00080B21949088002280DDB00200880FEF7EF
:1047000079FC01201149C8710020C87600F06CF8CE
:1047100000201249088012480088401C80B21049CD
:104720000880012805DB00200880FEF74BFCF9F724
:104730003DFAFEF7F1F9F9F7EFF8F6F7BFFEFEF7ED
:104740006DFC00BFD0E70000FE0C00206847002091
:104750000CED00E00000FA05F80C0020FC0C002035
:10476000FA0C00201FB540F2DF710098884204D097
:1047700040F23471009888422FD11A4800883228BC
:1047800002DB00201749088016480288001D00EB54
:104790000210009901609DF8041012480288001D63
:1047A00000EB021001719DF80D100E480288001DEB
:1047B00000EB021041730B480188001D00EB011053
:1047C000DDF8051040F8051FDDF8091041600548C7
:1047D0000088401C0349088003E0009988B200F07B
:1047E00031F81FBDFC43002010B51DE01248408881
:1047F000322802DB0020104948800F4880780F499A
:1048000008700D484188001D00EB011494E80F006A
:10481000FAF7C4FE08484088401C07494880084809
:104820000068401C0649086003480088024949881E
:104830008842DBD110BD0000FC430020E90C0020C1
:10484000F40C00201249097801F0010101B9704708
:10485000B0F5827F03D0A0F21111A1B909E00D4992
:10486000096821F001010B4A116000210A4A1180F8
:104870000AE00849096821F00201064A1160002196
:10488000064A118000BF00BF00BF00BFDFE7000085
:10489000500C0020740C00207E0C0020800C0020A6
:1048A0002DE9F74F84B00C4617460026F9F7B8FCFF
:1048B0000498002856D12079D3490870607948704F
:1048C000A0790006E17940EA0140217A40EA01201E
:1048D000617A0843CC494860A07AE17A40EA012035
:1048E000C9490881E07B0006A17B40EA0140617B69
:1048F00040EA0120217B0843C349C860207C617CD9
:1049000040EA0120C0490882701E88610020C86109
:1049100048624FF6FF7008840020BC490870BA480E
:10492000008AB949C968B84A1289CDE900210290C4
:10493000B548436842780178B5A000F01FFCB24842
:10494000008AB149C968B04A1289CDE900210290B4
:10495000AD48436842780178BC4800F00FFCF4F79A
:1049600097FC4EE104980128FBD1A848007810B1CB
:1049700007B0BDE8F08FE0780006A17840EA01407A
:10498000617840EA0120217808439F494861F4F7A3
:104990003FFCF9F745FC9C483A464169ACA000F061
:1049A000EDFB9948806998494969884272D09648D8
:1049B0004069954988610846C169A7F10D0008441E
:1049C0009149C8610846C369808BC0F30A02084652
:1049D000C069C10AA4A000F0D1FBF7F71BFF8A4809
:1049E000008C8949C969B0EBD12F14D08648C069C1
:1049F000C0F3CF20844908840846C069A64908440A
:104A00004FEAD0284FEAC8284146A4A000F0B6FBE0
:104A10004046F7F75BFE04F1040AA7F10D00C11749
:104A200000EB9171C1F3870BC11700EB91718910F5
:104A3000A0EB810169B1A0A000F0A0FBA7F10901E2
:104A400008190322FF21F3F7D2FB0BF1010000F05C
:104A5000FF0B6D48406A904900EB01086A48C06945
:104A600069494862002540E0002614E05AF8251004
:104A70004046F7F797FE042800D10DE0701CC6B23F
:104A8000032E08DB414692A000F078FB01205F492D
:104A900008706DE7B3E0E9E700BFD8F80090012D9A
:104AA00003DBABF10100A84206DC5AF825204B4697
:104AB000414690A000F062FB5AF8250048450DD011
:104AC00094A000F05BFB5AF825204B46414689A094
:104AD00000F054FB01204D49087049E708F1040833
:104AE000032E00DB03E0681CC5B25D45BCDB00BFE4
:104AF000F9F796FBA7F10D0081B28F480288201DBF
:104B0000F4F768FC8C4908803F4801898A4802888C
:104B10008AA000F033FBF9F783FB3B4840693A4930
:104B2000C968884269D13848008983490988884220
:104B300003D08BA000F022FB1AE700263248C168A0
:104B400091A000F01BFB9948F7F7C0FD0FE09849D2
:104B50009648F7F727FE042800D109E0701CC6B27A
:104B6000032E04DB914993A000F008FB00E0EEE780
:104B700000BF8E48D0F800904B468D4A01465DA09C
:104B800000F0FCFA8A48814503D001201F490870D3
:104B9000EEE6002612E01C4841688448001DF7F745
:104BA00001FE042800D10AE0701CC6B2032E05DB0A
:104BB0007E49091D88A000F0E1FA00E0EBE700BFA4
:104BC0007A48001DD0F800900F484B467749091DE0
:104BD00042688BA000F0D2FA0B484068484503D0E9
:104BE00001200A490870C3E6F9F71AFBF4F710FB35
:104BF0008CA000F0C3FAFAF753F8F7F7A7FDF9F71E
:104C00000FFB00BFB4E60000981B00206A050020DF
:104C10000D0A3636365570642D2D747970653A2537
:104C200064202C7665723A25642C54627974653A56
:104C300025642C204372633A25642C5061673A2521
:104C4000642C506C656E3A25640D0A009CC0010806
:104C50000A0D43757272204261673A25642C206CFC
:104C6000656E2025640A0D0057726974652D6164B4
:104C700064723A20736563746F722025642C2C6F04
:104C80006666736574202564202C7265636C656E9E
:104C9000202530640D0A000000600208343443759A
:104CA00072722045726173652D2D616464723A20C1
:104CB0002530780D0A0000000A0D6C6173742D2DEB
:104CC0002D2D2D626167212121212121210A0D0035
:104CD0002132322121212121212121215772697480
:104CE000652D4661696C2D616464723A20253078C7
:104CF0000D0A000061646472202530782C2C5772F4
:104D0000697465202530782C2C726561642025300B
:104D1000780D0A000A0D207265616476616C2021AD
:104D20003D20557064646174615B695D29212121B6
:104D300021210A0D000000006805002031323255A3
:104D40007064486561642E46696C654372633D25F5
:104D500030782C544372633D2530780D0A000000F2
:104D6000557064486561642E46696C6543726320C2
:104D7000213D2054437263202121212072657475E6
:104D8000726E210D0A0000002121217570642D69C9
:104D90006E666F21212057726974652D746F74706F
:104DA0006167202564200D0A0000000000580208F9
:104DB0004433221155706444617461466C6167210B
:104DC0002057726974652D4661696C2D6164647247
:104DD0003A202530780D0A002121217570642D6953
:104DE0006E666F21212057726974652D4661696C6A
:104DF0002D616464723A202530780D0A00000000AD
:104E00003161646472202530782C2C577269746586
:104E1000202530782C2C72656164202530780D0AAD
:104E20000000000032327570642D616C6C20777266
:104E3000697465204F4F4B4B212172657374617209
:104E40007421212121212121212121210D0A00006C
:104E500070B5C2B005460C46002641F20D00084967
:104E6000A1F80500224629460548C01DF3F7ADF913
:104E70000348448001AA02A9F6F74EFF42B070BD74
:104E8000DE1F002000BFFEE710B502240E4A106F9F
:104E9000126F916A884760B905210C48FBF746FC00
:104EA00078B12620F7F7EEFB0848FBF752FC012407
:104EB00007E0054A106F126F916A8847012800D1F8
:104EC0000024204610BD0000D8070020083700202D
:104ED0002DE9F04104460E461546601BF3F70FFC22
:104EE00080463146F3F745FA0746F3F73CFC80B2BB
:104EF000BDE8F0812DE9FC4781460C4692463148D9
:104F000000EB04100078C0B32E4800EB041040689A
:104F100048B32C4800EB041040681421B0FBF1F0BA
:104F2000284901EB04114860264901EB0411486847
:104F3000F3F7F3FB07464FF06632234BF3F7FEFA25
:104F400005460022214BF3F76BFBCDE90001F3F797
:104F50007BFC1C4901EB0411C8601A4800EB0410EB
:104F6000C068CAF800000020164901EB041148602F
:104F7000144901EB0411087022E0FFE7114800EB2F
:104F80000410007A401C0F4901EB041108720D480F
:104F900000EB0410406848440A4901EB04114860E2
:104FA000084800EB0410007A142809D101200549B3
:104FB00001EB041108700020024901EB0411087292
:104FC000BDE8FC87980D002066660A400000B040EE
:104FD00010B50121C802FBF733F800214FF400603F
:104FE000FBF72EF810BD00000020084908600848B3
:104FF0000078401C06490870084600781E2803DC2B
:105000007F2002490839086070470000082C0040E2
:10501000E901002044E032213EE000BF00BF00BFB4
:1050200000BF00BF00BF00BF00BF00BF00BF00BF88
:1050300000BF00BF00BF00BF00BF00BF00BF00BF78
:1050400000BF00BF00BF00BF00BF00BF00BF00BF68
:1050500000BF00BF00BF00BF00BF00BF00BF00BF58
:1050600000BF00BF00BF00BF00BF00BF00BF00BF48
:1050700000BF00BF00BF00BF00BF00BF00BF00BF38
:1050800000BF00BF00BF00BF00BF00BF00BF00BF28
:1050900000BF00BF4A1ED1B20029BEDC421ED0B202
:1050A0000028B8DC7047000010B51E4890F82200B8
:1050B000012817D11C4801780078401C1A4A10704A
:1050C00005290FDDF9F7ACF80020164981F8220018
:1050D0001222164801F072FE00201349087014A035
:1050E00000F04CF80F4890F82300012818D10E4822
:1050F00001780078401C0C4A1070052910DDF9F782
:105100008FF80020074981F823001022123111483E
:1051100001F054FE0020044908700FA000F02EF8A2
:1051200010BD0000A02600203A09002000F0010870
:105130004F726465725F436F64652057726974656E
:10514000207375636365737366756C6C79210D0AE2
:105150000000000000F8010850726F647563745F0E
:10516000436F646520577269746520737563636566
:10517000737366756C6C79210D0A00000FB4054BD2
:1051800010B503A9044A029800F044F910BC5DF878
:1051900014FB0000357B0108080200200FB4084B07
:1051A00010B504A902AA039800F034F9044602A934
:1051B000002000F0B2FC204610BC5DF814FB00009B
:1051C0001B5B010830B528B1144C031F0020216877
:1051D0000A4605E0084630BD9A4203D81046526898
:1051E000002AF9D1002800D041680BD00468A3EB55
:1051F0000005A54204D11B681C440346046002E07C
:10520000436000E023603AB11C68D51AA54203D17F
:1052100015682C441C6052685A6030BD600D002037
:105220002DE9F04782460F4C10480D4E0E4F001BE3
:105230004FF0000820F007054FF001090022114649
:10524000504603F037FA002802D1306810B1002030
:10525000BDE8F0873C60C4E90058C6F80090EDE76F
:10526000640D00204C4A0020600D0020486A002098
:1052700002E008C8121F08C1002AFAD1704770471F
:10528000002001E001C1121F002AFBD1704700007D
:105290002DE9FF5F82B00021DDE90430020DDDF869
:1052A00040B0034318D044F61050A2F2FF324243FC
:1052B0001514119801281FD0A5EB0B00401C5FEAC4
:1052C000000A4FF000064E4FDFF83891B0465046C6
:1052D00015D5CAF1000413E0119801244AA301284E
:1052E00001D16FEA0B010298119AC0E90031C0E9BF
:1052F000024206B0BDE8F09FCBF10000DFE70446B4
:105300000021404A491842EB0450CDE9001012E058
:10531000E00707D032463B4640464946F3F70EF9D0
:105320008046894632463B4610461946F3F706F951
:1053300006460F466410002CEAD1DDE90401DDE9E0
:105340000023BAF1000F06DAF3F7F8F842464B46AD
:10535000F3F7F4F805E0F3F763F942464B46F3F749
:105360005FF904460E460022284BF3F755FA03D89E
:105370004FF0FF30014607E00022254B2046314622
:10538000F3F735F8F3F77DFB102409E0002C0ADB76
:105390000A220023F3F79EFA039B30321A55641E4B
:1053A00050EA0102F2D1641C039AC4F111031444BF
:1053B000119A012A03D0012208430DD10AE00843C3
:1053C00004D000204FF0110B119072E7A3EB0B05F6
:1053D0006D1E0DE05B4504DD4FF0000205F1010597
:1053E00004E003DA4FF00002A5F10105002AECD039
:1053F00002981199C0E90231C0E9004579E700003F
:10540000000014400000F03F300000000000F043B6
:105410000000E03F2DE9FF4F95B09A4688460646CA
:105420000025EEE1252877D100242746F94A0121FD
:10543000039400E0044316F8013F203B01FA03F017
:105440001042F7D130782A2811D06FF02F0330782E
:10545000A0F13002092A16D8039A44F0020402EBA4
:10546000820203EB42021044761C0390EFE758F8E7
:10547000042B0392002A03DA504244F400540390B0
:1054800044F00204761C30782E2816D116F8010F4D
:1054900044F004042A280DD06FF02F023078A0F1D8
:1054A0003003092B09D807EB870302EB4303C71826
:1054B000761CF3E758F8047B761C30786C280FD004
:1054C00006DC4C2817D068280DD06A2814D104E0D7
:1054D000742810D07A280FD10DE044F400140AE0AB
:1054E00044F4801401E044F440147278824202D102
:1054F00004F58014761C761C307866280BD013DCFB
:10550000582877D009DC002875D04528F6D04628E1
:10551000F4D047281AD193E118E0632835D06428E5
:1055200079D0652812D18BE1702873D008DC672808
:10553000F1D069286FD06E280DD06F2806D1ACE06D
:1055400073282CD0752874D0782853D052461799D8
:1055500090476D1C54E1C4F30250022809D003287F
:105560000DD0D8F8001004280DD00D6008F1040803
:1055700046E1D8F80010EA17C1E90052F6E7D8F87A
:1055800000100D80F2E70D70F0E718F8041B8DF89D
:10559000001000208DF80100EB46012003E058F8D0
:1055A00004BB4FF0FF3061074FF0000102D40DE063
:1055B00009F101018946B9420FDA8145F8DB1BF890
:1055C00009100029F4D108E009F10101894681425E
:1055D000FADB1BF809100029F6D103985346A0EB1B
:1055E000090721463846179A00F080FA284400EB54
:1055F000090507E044E008E10DE01BF8010B524605
:1056000017999047B9F10109F7D253462146384618
:10561000179AF2E039E00A21C4F302524FF0000B6E
:105620000091022A06D058F8040BC117032A09D0AA
:105630000AE023E008F1070020F00702F2E8020187
:10564000904605E000B2C117042A01D140B2C1174B
:10565000002906DA0A460021404261EB02012D22B0
:1056600002E0220504D52B228DF80420012203E05C
:10567000E20701D02022F7E7914657E00A2100E037
:1056800010214FF0000B00910BE010214FF0000BA8
:1056900044F004040827009103E008204FF0000BB9
:1056A0000090C4F30252022A05D058F8040B0021DE
:1056B000032A08D008E008F1070020F00702F2E80A
:1056C0000201904603E080B2042A00D1C0B24FF03C
:1056D000000922072AD53278702A07D0DDF800C0E9
:1056E0008CF0100C5CEA0B0C05D00EE040228DF81B
:1056F0000420012208E050EA010306D030238DF88F
:1057000004308DF8052002229146009B83F00803A7
:1057100053EA0B030AD150EA010201D1620705D511
:1057200030228DF804204FF001097F1E3278582A6C
:1057300004D039A20C920CAA02920BE03BA2F9E72A
:105740005B46009AF3F7C6F80C9B9B5C029A521ECC
:105750000292137050EA0102F2D1029804A9081AC9
:1057600000F1200B600702D524F4803400E001270B
:105770005F4502DDA7EB0B0000E0002000EB0B0112
:10578000009003984944401A0390E00306D453461E
:105790002146179A039800F0A9F90544002706E06E
:1057A00001A85246C05D179990476D1C7F1C4F455C
:1057B000F6DBE0030CD553462146179A039800F018
:1057C00095F9054404E030205246179990476D1C26
:1057D0000099481E00900029F5DC08E00298029923
:1057E00052460078491C0291179990476D1CBBF1F5
:1057F0000001ABF1010BF1DC5BE100F065F9054460
:10580000761C307800287FF40DAE19B02846BDE82C
:10581000F08F00000928010030313233343536373B
:1058200038396162636465660000000030313233EC
:10583000343536373839414243444546000000008C
:10584000600700D4062708F1070020F00700F0E801
:105850000223804603F0004C5FEA0C0001D097A0C1
:1058600009E0200501D596A005E0E00701D095A04C
:1058700001E0AFF24C001390307823F0004365282C
:105880000CD006DC452809D046281DD047287FD1FA
:105890003BE0662818D067287AD136E00021112F26
:1058A00001DB112000E0781CCDE9000104A90CA85F
:1058B000FFF7EEFCDDE90D010C9A4FF0000B07F14C
:1058C0000109109200914EE04FF000400097CDE9A1
:1058D000011004A90CA8FFF7DBFCDDE90D020C9B0D
:1058E0000F994FF0000B91461093009211B9791C5B
:1058F00000EB0109B7EB090003D4C0F1FF3B07F14E
:105900000109A9EB0700019042E0012F00DA01270D
:105910000021112F01DD112000E03846CDE9000102
:1059200004A90CA8FFF7B4FCDDE90D010C9A009165
:105930004FF0000BB946109221070FD4009A4A4548
:1059400003DA914601E0A9F10109B9F1010F05DD82
:10595000109AA9F10101515C3029F4D0B84202DA61
:1059600010F1040F03DA0121CDE9011010E0002845
:1059700003DC8344A9EB000102E0411C494500DD42
:105980008946A0EB0B00401C01904FF000400290B4
:10599000200705D40198484502DB4FF0FF30019005
:1059A00000208DF84B0002980DF14B07B0F1004F2D
:1059B00025D002200C902B200D90029800280CDAA4
:1059C000404202902D200D9007E00A210298F2F744
:1059D0006BFF3031029007F8011D0C99481E0C90A6
:1059E0000029F2DC02980028EFD1791E0D9808708A
:1059F000307800F0200040F0450007F8020D11A8B3
:105A0000C01BC01D02901398007800B1012000EB6C
:105A10000901019801EBE071029801440398401AD2
:105A2000401E0390E00306D453462146179A03987C
:105A300000F05CF805441398007818B152461799A5
:105A400090476D1CE00323D553462146179A0398CF
:105A500000F04CF805441BE0BBF1000F07DB009899
:105A6000584504DD1098179910F80B0001E01799BC
:105A700030205246904701980BF1010B401E05F172
:105A80000105019004D12E205246179990476D1CB4
:105A9000B9F10001A9F10109DEDC05E017F8010BFD
:105AA0005246179990476D1C0299481E0290002992
:105AB000F4DC53462146179A03989EE62D00000019
:105AC0002B000000200000002DE9F04104460025D5
:105AD0001E461746880404D405E039462020B04706
:105AE0006D1C641EF9D52846BDE8F0812DE9F04112
:105AF000044600251E469046C80301D5302700E025
:105B00002027880404D505E041463846B0476D1C7F
:105B1000641EF9D52846BDE8F0810A68531C0B6065
:105B2000107070470749084A126888540649096886
:105B3000491C0A2291FBF2F302FB1311024A116085
:105B400070470000D42600204009002010B504460C
:105B500002F0F4FD18B10AA0FFF710FB10BD0E48CB
:105B60000E49096844540D480068401C052190FB0B
:105B7000F1F201FB12000949086000BFEEE70000E6
:105B80004576656E7420717565756520697320664C
:105B9000756C6C0A00000000240C0020200C002012
:105BA00010B58CB001F0DAFB26E09DF80C3004AAA9
:105BB00007A80699F4F763FA00208DF82F0001205A
:105BC000294908700B98009007A80FC800F002FA46
:105BD00001280FD1142207A92448F2F7F6FA224827
:105BE0000021CDE901102148006900901F480FC82D
:105BF00000F08CF9F8F714FB1D48406840B11C48D0
:105C000003AB04AA06A944680020A0470128CCD011
:105C10001AE09DF80C3004AA07A80699F4F72FFAA9
:105C200000208DF82F00FEF76BFA28B10B9800903A
:105C300007A80FC800F042F90B98009007A80FC8FA
:105C4000FEF784FAF8F7ECFA0948C06940B1084851
:105C500003AB04AA06A9C4690120A0470128D8D033
:105C600001F054FA0CB010BDE8010020D416002059
:105C70008416002010B520211A48F2F7BFFA30210F
:105C80001948F2F7BBFA01F063FBF8F7EBFBF8F702
:105C900015FC154A15490020F8F7FEFC10B114A0B8
:105CA000FFF76CFA104A183217490120F8F7F4FC94
:105CB00010B116A0FFF762FA0B48C06830B10A486D
:105CC00000231A461946C4681846A0470648406A89
:105CD00030B1054800231A461946446A0120A047FE
:105CE00010BD0000B416002084160020B001002072
:105CF00063616E3120D0ADD2E9B3F5CABCBBAFB39E
:105D0000C9B9A60D0A0000007C01002063616E3253
:105D100020D0ADD2E9B3F5CABCBBAFB3C9B9A60DAB
:105D20000A00000010B5A2B0002441F20B000D499A
:105D3000A1F8050000BF01E0601C84B2282CFBDB49
:105D40005020084948800848007C401C06490874D7
:105D500006A0FFF713FA01AA02A90248F5F7DCFF33
:105D600022B010BDDE1F00206421002053656E6448
:105D70002063656C6C2074656D70200A0D00000056
:105D800010B5A2B0002441F20C001049A1F80500A2
:105D900000BF06E00E48015D0C48C01D0155601CA7
:105DA00084B2082CF6DB0820084948800948007CAA
:105DB000401C0849087408A0FFF7E0F901AA02A9ED
:105DC0000248F5F7A9FF22B010BD0000DE1F002039
:105DD0002D2400206421002073656E6420626D73A1
:105DE0005F73746174655F696E666F0A0D00000011
:105DF00010B5A2B0002441F20A001149A1F8050033
:105E000000BF09E004EB44010E48084481780C48C7
:105E1000C01D0155601C84B2282CF3DB28200849E2
:105E200048800948007C401C0749087407A0FFF718
:105E3000A5F901AA02A90248F5F76EFF22B010BD2C
:105E4000DE1F0020B52300206421002053656E640E
:105E50002063656C6C2074656D70200A0D00000075
:105E600070B50546002400BF1FE0114951F83410F9
:105E70002868884217D10E4800EBC400406828B15A
:105E80000B4800EBC40041682846884740F2274190
:105E90002868884205D10748FAF75BFC01200649CB
:105EA000087300202860601C44B2112CDDD370BD43
:105EB0000C06002050370020480900200FB410B510
:105EC000142202A90D48F2F780F90C480468142244
:105ED00001460B48F2F779F980210A48F6F78EF867
:105EE000094801680548884714210448F2F786F9F3
:105EF00000200249086010BC5DF814FB0811002066
:105F0000CC10002000100140080600200FB470B52E
:105F1000DDE9095429484078142810DA27494978DE
:105F200001EB81022549091D01EB8200142204A91D
:105F3000F2F74BF921484078401C204948700598F9
:105F40006FF30F001E49884218D19DF81B001028DE
:105F500003D09DF81B00132804D19DF81E00194999
:105F6000087007E09DF81B00112803D19DF81C0064
:105F7000144908700A201449086015E005986FF369
:105F80000F00124988420FD19DF81B000D49097876
:105F9000884206D114200C49086000200949087085
:105FA00002E032200849086000210948FCF798FC0B
:105FB0000020207070BC5DF814FB0000000F002072
:105FC0000000EC1C08010020F00000200000EB1C89
:105FD000EC0000200FB410B5142202A93848F2F7E3
:105FE000F4F837484068374908603548808880B2FF
:105FF0004FF25641884204D04FF0FF3010BC5DF89C
:1060000014FB2F4840686FF30F002F49884207D1D7
:1060100014222B492D48F2F7D8F84FF0FF30EDE766
:10602000274840686FF30F002949884207D114229E
:1060300023492648F2F7C9F84FF0FF30DEE7214840
:106040000068244988422CD01E48006822498842B2
:1060500027D01C4800682149884222D0194800688E
:106060001F4988421DD0174800681E49884218D031
:10607000144800681C49884213D0124800681B4924
:1060800088420ED00F4800681949884209D00D484F
:1060900000681849884204D00A48006816498842B6
:1060A0000BD1142206491548F2F78FF804498A7A71
:1060B000002348680B3100F04FFD00209EE70000F0
:1060C000F4100020040100200000EC1CB00E0020A1
:1060D0000000EB1C56F4261856F4011856F4071865
:1060E00056F4081856F40A1056F4121856F41D18EF
:1060F00056F41F0856F41A1056F41A18EC0E002025
:106100002DE9F05F002029490860294848600420F3
:1061100008720020487205208872FF220821234857
:106120000B30F2F764F83320F6F792FA18B93420FE
:10613000F6F78EFAB8B11F48B0F841A00146B1F8A1
:106140004300F2F7EAFA80461B4A1C4BF2F7F6F9D5
:10615000064600221A4BF2F7EEF90446F2F717FB57
:106160001FFA80FB08E01348B0F841A0B0F84300E4
:10617000C0F57A601FFA80FB0C4981F80BA04FEA4A
:106180001A210A48017380F80DB04FEA1B21817370
:10619000084890F8450008B1022100E001210348B9
:1061A000C17301F0F7F9BDE8F09F0000C40E0020B4
:1061B000F4561018D80700209A9999999999E93FAF
:1061C0000040AF4010B50446012C25D100204B49BA
:1061D00008604B484860042008720020487208207C
:1061E0008872FF22082145480B30F2F700F8102092
:1061F0004249C8720D2141480173002141730221B7
:106200008173FF21C17300210174062141740021B3
:10621000817401F0BFF970E0022C6ED10020374983
:10622000086038484860042008720020487208203E
:106230008872FF22082131480B30F1F7D8FF012086
:106240002E49C872304890F833102C4801732E48FC
:10625000B0F83300010A294841732B48B0F83500E3
:10626000C0F57A60C1B2254881732748B0F835007F
:10627000C0F57A60010A2148C173234890F83710AD
:106280001E4801742048B0F83700010A1B484174C9
:106290001D4890F839101948817401F07BF90320EA
:1062A000F5F72BFE02201549C8721748B0F83900DF
:1062B000010A12480173144890F83B000A30C1B239
:1062C0000E48417300BF104890F83C00C1B20B4823
:1062D000817300BF0C48808F010A0848C1730A48C7
:1062E00090F83E10054801740748C08F010A034822
:1062F00041740021817401F04DF910BDC40E0020DD
:10630000F456EC1CF456EB1CD807002010B50446DC
:10631000012C25D100203E4908603E4848600420F9
:1063200008720020487208208872FF22082138482D
:106330000B30F1F75CFF10203549C8720921344851
:1063400001730021417302218173FF21C173002178
:106350000174112141740021817401F01BF956E090
:10636000022C54D100202A4908602B4848600420A0
:1063700008720020487208208872FF2208212448F1
:106380000B30F1F734FF01202149C872234890F8FF
:1063900046101F4801732148B0F84600010A1C4806
:1063A00041731E4890F84810194881731B48B0F893
:1063B0004800010A1648C173184890F84A1014485A
:1063C00001741648B0F84A00010A11484174134894
:1063D00090F86C100E48817401F0DCF80320F5F79A
:1063E0008CFD02200A49C8720C4890F84D100848EC
:1063F00001730A48B0F84D00010A054841730021B5
:106400008173C17301744174817401F0C3F810BDCC
:10641000C40E0020F456EC1CF456EB1CD8070020E8
:1064200010B5044600200C4908600C484860042060
:1064300008720020487202208872FF220821064854
:106440000B30F1F7D4FE0449CC72210A02480173E3
:1064500001F0A0F810BD0000C40E0020F45627186B
:1064600010B586B00446142101A8F1F7C7FE012C2F
:1064700025D10020924908609248486004200872A3
:106480000020487208208872FF2208218C480B30B7
:10649000F1F7ADFE10208A49C87231218848017396
:1064A0000021417307218173FF21C1730021017411
:1064B000022141740021817401F06CF8FEE0022C8D
:1064C000FCD100207E4908607F48486004200872A3
:1064D0000020487208208872FF22082178480B307B
:1064E000F1F785FE01207649C87200BF77488078B1
:1064F000087300BF7548C078487300BF73480079BF
:10650000887300BF71484079C87300BF6F488079B5
:10651000C1B26B48017400BF6C48C088010A68486A
:10652000417400BF6948007AC1B26548817401F0C6
:1065300031F80320F5F7E1FC02206149C87200BF81
:1065400062480089010A5E4801736048817A5C48AC
:1065500041735E48C17A5A4881735C48017B584850
:10656000C1735A48417B56480174002141748174BB
:1065700001F010F80320F5F7C0FC03205049C87261
:1065800001214F480173022141735048817C4C48DE
:1065900081734E48C17C4A48C1734C48017D4848CC
:1065A00001744A48417D464841744848817D4448C9
:1065B000817400F0EFFF0320F5F79FFC00204449B1
:1065C00081F88701084690F88701012806D1122238
:1065D0003E491A3101A8F1F7F8FD04E0FF2211212C
:1065E00001A8F1F704FE04203549C8723748C17D7F
:1065F000334801733548017E31484173002181736E
:106600009DF80410C1739DF8051001749DF80610E3
:1066100041749DF80710817400F0BCFF0320F5F76A
:106620006CFC05202649C8729DF8081024480173A7
:106630009DF8091041739DF80A1081739DF80B10A5
:10664000C1739DF80C1001749DF80D1041749DF8F4
:106650000E10817400F09EFF0320F5F74EFC06201B
:106660001749C8729DF80F10154801739DF8101056
:1066700041739DF8111081739DF81210C1739DF83C
:10668000131001749DF8141041741021817400F0EE
:1066900081FF0320F5F731FC07200949C8720A2160
:1066A000074801730B21417307218173E021C173F6
:1066B000FF2101744174817400F06CFF06B010BDBD
:1066C000C40E0020F456EC1CF456EB1CD807002036
:1066D000F816002010B5044600200A4908600A4850
:1066E0004860042008720020487201208872FF224E
:1066F000082104480B30F1F77AFD0248C47200F01B
:1067000049FF10BDC40E0020F456091010B5044610
:1067100000202049086020484860042008720020BA
:10672000487207208872FF2208211A480B30F1F7BF
:106730005EFD1A4890F86C001649C87200BF1748F1
:1067400090F86600C1B21348017300BF1348B0F857
:106750006600010A0F48417300BF104890F86800B6
:10676000C1B20C48817300BF0C48B0F86800010A40
:106770000848C17300BF094890F86A0005490874C9
:1067800000BF064890F86B004874084600F002FF0E
:1067900010BD0000C40E0020F4561C18D8070020BD
:1067A0002DE9F04781460024002500260027A04659
:1067B00000207E4908607E4848600420087200205E
:1067C000487207208872FF22082178480B30F1F7C1
:1067D0000EFD784890F89701012806D105244B2535
:1067E00004264A274FF0030805E005244B2504261C
:1067F0004A274FF003082B20F5F72AFF18B92C2061
:10680000F5F726FF48B16C4890F85B0020F00300D4
:10681000401C694981F85B0007E0674890F85B001D
:1068200020F00301644880F85B102D20F5F710FF7D
:1068300018B90C20F5F70CFF48B15F4890F85B00E1
:1068400020F00C00001D5C4981F85B0007E05A480D
:1068500090F85B0020F00C01574880F85B102E2068
:10686000F5F7F6FE48B1544890F85B0020F0300090
:106870001030514981F85B0007E04F4890F85B0009
:1068800020F030014C4880F85B100B20F5F7E0FE5B
:1068900048B1494890F85B0020F0C00040304649BC
:1068A00081F85B0007E0444890F85B0020F0C001ED
:1068B000414880F85B100E20F5F7CAFE18B91A207F
:1068C000F5F7C6FE48B13C4890F85C0020F00301A3
:1068D000491C394880F85C1007E0374890F85C00A4
:1068E00020F00301344880F85C1000BF324890F873
:1068F0005900012809D1304890F85C0020F00C01C3
:10690000091D2D4880F85C1007E02B4890F85C00CA
:1069100020F00C01284880F85C1000BF264890F851
:106920005A00012809D1244890F85C0020F0300179
:106930001031214880F85C1007E01F4890F85C0097
:1069400020F030011C4880F85C1000BF1A4890F815
:106950004F001649C87200BF174890F850000A301F
:10696000C1B21248017300BF134890F851000F499B
:10697000487300BF104890F852000A30C1B20B486B
:10698000817300BF0C4890F853000849C8730A4847
:1069900090F85B1005480174074890F85C100348B4
:1069A000417400F0F7FDBDE8F0870000C40E002040
:1069B000F4561318F8160020D807002010B5044626
:1069C0000020624908606248486004200872002084
:1069D0004872042088725F4890F86C00642809D1DE
:1069E0005C4890F8610020F00300401C594981F890
:1069F000610007E0574890F8610020F00301554816
:106A000080F861102F20F5F723FE48B1514890F827
:106A1000610020F0C00040304E4981F8610007E07D
:106A20004C4890F8610020F0C0014A4880F861109D
:106A30001A20F5F70DFE18B90E20F5F709FE48B13A
:106A4000444890F8620020F00301491C414880F856
:106A5000621007E03F4890F8620020F003013D48D3
:106A600080F862100B20F5F7F3FD48B1394890F833
:106A7000630020F00301491C364880F8631007E0EA
:106A8000344890F8630020F00301324880F8631026
:106A90000320F5F7DDFD18B90420F5F7D9FD48B15D
:106AA0002C4890F8630020F00C01091D294880F85B
:106AB000631007E0274890F8630020F00C01254898
:106AC00080F863102E20F5F7C3FD48B1214890F8F7
:106AD000640020F00301491C1E4880F8641007E0A0
:106AE0001C4890F8640020F003011A4880F86410F4
:106AF0000120F5F7ADFD48B1164890F8640020F08C
:106B00000C01091D134880F8641007E0114890F843
:106B1000640020F00C010F4880F864100D4890F8D4
:106B200061000A49C8720B4890F862100748017367
:106B3000084890F8631005484173064890F86410BF
:106B40000248817300F026FD10BD0000C40E002035
:106B5000F4561910D80700202DE9F04105460E46DD
:106B6000174698460024F4F7B9FA5649681A8D4238
:106B70004CD015DC5449A5EB01008D4273D008DCE4
:106B80005248284400286CD051490844002869D153
:106B90004AE050490844E8B1B0F5C02FF7D127E0EA
:106BA000B0F5202F4ED0B0F5901F5DD0B0F5A81FE6
:106BB00068D0B0F5F01FEAD1424639463046F4F7C6
:106BC000A7F804462CB14448806B40F48040424909
:106BD000886374E0424639463046F4F7DDF80446EF
:106BE0002CB13D48806B40F001003B49886366E072
:106BF000424639463046F4F71FF904462CB1364870
:106C0000806B40F002003449886358E042463946C0
:106C10003046F4F78DF804462CB12F48806B40F0D5
:106C200004002D4988634AE0424639463046F4F76D
:106C3000D1F804462CB12848806B40F00800264962
:106C400088633CE0424639463046F4F70FF8044684
:106C50002CB12148806B40F010001F4988632EE062
:106C600001E01DE02AE000BF424639463046F4F715
:106C7000CFF804462CB11848806B40F0200016492C
:106C800088631CE0424639463046F4F7ADF80446C6
:106C90002CB11148806B40F040000F4988630EE032
:106CA000424639463046F4F71FF804462CB10A48EC
:106CB000806B40F080000849886300E000BF00BF9F
:106CC000BDE8F08156F4081856F41A10AA0BE0F744
:106CD000000015F8000019F8200E0020F0B503465A
:106CE00098180F4FB84201D90320F0BD0AB900200F
:106CF000FBE7012600240BE01D780878A84204D0A9
:106D0000FF2D01D00220F0E700265B1C491C641C0B
:106D10009442F1D3012E01D10020E6E70120E4E7FF
:106D20000000020801460020C80AC00270470000A7
:106D300008B501210820F9F793F903208DF8020026
:106D400014208DF803004FF48060ADF80000694610
:106D50000D48F5F75DFF03208DF802004FF4006049
:106D6000ADF8000014208DF8030069460648F5F7D9
:106D70004FFF4FF480610448F5F740F94FF400618C
:106D80000148F5F73BF908BD000C014030B503465A
:106D90009818094DA84201D9012030BD0AB9012037
:106DA000FBE7002404E013F8010B01F8010B641C5D
:106DB0009442F8D30020F0E7000002082DE9F84FD4
:106DC00006460F4614464FF0040B30192A498842F4
:106DD00002D90120BDE8F88F0CB90020FAE704F0D1
:106DE000010000B1641C224639463046FFF776FFA9
:106DF0008046B8F1000F01D10020EBE7012080F3BD
:106E0000108800BFF5F706FD3520F5F759FC304630
:106E1000FFF788FF0090F5F759FC83464FF47A7A24
:106E200000BFBAF10000AAF101011FFA81FAF8D1FE
:106E3000002511E017F815906800401C385C49EAFD
:106E4000002949463046F5F78BFC8346BBF1040F19
:106E500000D004E0B61C6D1CB5EB540FEAD300BFA4
:106E6000F5F774FC002080F3108800BFBBF1040F1D
:106E700000D1AFE70220ADE70000020810B50446DC
:106E80003CB900210748F3F7BFFC0648F3F7B4F814
:106E900006E000210448F3F7B7FC0348F3F7ACF829
:106EA000012010BD006400400068004070B5054638
:106EB0000C46022D00DB70BD05EB85000D4901EB92
:106EC0008000006988B1A37A207A042801D1606823
:106ED00000E02068014605EB8500064A02EB8000D1
:106EE00004F10B0206692846B047284600F0DCF999
:106EF00000BFE0E71C11002070B505460E460DB935
:106F0000064900E0064908463146F3F761FD0446AC
:106F1000042C00D1FF24204670BD00000064004016
:106F20000068004070B504460D461646022C00DB92
:106F300070BD04EBC400144901EB8000C06801215E
:106F4000A9400840F0B104EBC4000F4901EB8000F8
:106F5000C0680121A940884304EBC4010A4A02EB3E
:106F60008101C860204600F09FF904EB84000749C6
:106F700051F8200030B104EB840051F8202029465C
:106F80002046904700BFD3E7441100201C11002089
:106F900070B504460D4614B9F3F77AFB01E0F2F739
:106FA00049FE012070BD000010B50446832C00D0BE
:106FB00010BD0A48007C01280ED00948C06A18B1EB
:106FC0000748C16A0120884701200449087400214C
:106FD00002481430FBF784FC00BFE9E7B416002038
:106FE000841600202DE9F04105460E4626BB2F46AB
:106FF00000240FE0124800EB04100068B84207D1EB
:107000000F4901EB041101F10C000021FBF768FCB2
:10701000601C84B2022CEDD300BF0A48807F002898
:107020000BDD0848007C022807D100210548817744
:107030001830FBF755FC00E000BFBDE8F081000010
:107040005C010020B416002010B50446002004EBBB
:10705000C401044A02EB810188602046FFF70EFF5D
:1070600010BD00004411002010B50446022C00DBC6
:1070700010BD04EB84000D4901EB8000806890B1E5
:1070800004EBC4000A4B03EB8000C06808B1012088
:1070900000E00020014604EB8400044B03EB800079
:1070A00082682046904700BFE2E700001C110020E4
:1070B0004411002010B50446022C00DB10BDF9F786
:1070C000B6FA04EB84000F4901EB8000C06838B1C8
:1070D00004EB84000A4602EB8000C1682046884722
:1070E000F9F7A7FA04EBC400074901EB8000C06878
:1070F00030B1002004EBC401034A02EB8101C860F7
:1071000000BFDBE71C110020441100207CB50020EB
:107110000090019000246CE0374800EB04100078E8
:1071200001284CD1344800EB04108089062807D28E
:10713000314800EB04108089304931F8105001E0EB
:107140002E4845892C4901EB0411081D2946FBF7FF
:10715000C7FB00284BD0F9F76AFA274800EB041068
:107160008089401C244901EB0411888104EB440010
:10717000234901EBC000C06848B104EB440001EBB7
:10718000C00000231A461946C6682046B0470220B0
:10719000194901EB0411087001208DF80000F9F77E
:1071A00048FA154901EB041101F108000021FBF731
:1071B00097FB0120104901EB0411887317E00E487A
:1071C00000EB04100078022811D10B4901EB0411E7
:1071D00001F108006721FBF783FB40B1002006495D
:1071E00001EB04118881044901EB04110870601C53
:1071F000C4B2022C90DB7CBDB416002094BA010806
:10720000841600202DE9F04104460D4616461F461F
:10721000022C02DB0020BDE8F081012004EBC40158
:10722000204A02EB81018860002004EBC40102EBDC
:107230008101487104EBC400114601EB8000077125
:1072400004EBC40001EB8000C67004EBC40021F81D
:107250002050002004EBC40102EB8101C86004EB64
:10726000C40002EB80012046FFF792FE38B10220F5
:1072700004EBC4010B4A02EB8101886006E00020A8
:1072800004EBC401074A02EB8101886004EBC400EF
:10729000044901EB80008068022801D10120BAE78F
:1072A0000020B8E744110020022800DB704700BF2F
:1072B000FCE700002DE9F04104460E4617469846CB
:1072C000022C07DA04EBC400194901EB8000806846
:1072D000022802D00020BDE8F08104EBC401144A6A
:1072E00002EB810101F1100043463A463146F2F7C4
:1072F0009FFE04EBC4000E4A02EB800000F1100177
:107300002046FFF7F9FD0546FF2D0ED004EBC40023
:10731000074901EB8000C1680120A840014304EB4C
:10732000C400034A02EB8000C1602846D3E7000096
:1073300044110020FEB504460D4616460094019502
:1073400002966946014803F0E6FEFEBD0C140020DB
:1073500010B500F0A9F800F047F810BD10B500F026
:1073600055F800F0ABF810BD10B502460B4612B947
:107370004FF0FF3010BD002114E01A4850F83100E2
:1073800090420ED1174800EBC1004360154800EB56
:10739000C100406818B90020124C44F831000020A8
:1073A000E8E7491C1429E8D313B94FF0FF30E1E7AF
:1073B000002111E00B4850F8310020B1094800EBE2
:1073C000C100406838B9074840F8312000EBC100DF
:1073D00043600020CEE7491C1429EBD34FF0FF3067
:1073E000C8E700008C11002010B54FF42671064844
:1073F000F0F704FF28230C220349A03101F5F070B7
:1074000003F05EFE002010BD8C1100203EB518E098
:1074100069460F4803F062FE00240FE00D4850F863
:1074200034000099884208D10A4800EBC40045683E
:1074300015B19DE80700A84702E0641C142CEDD3A9
:1074400000BF034803F02AFE0028E1D000203EBD23
:107450000C1400208C11002010B502460AB900203F
:1074600010BD002119E001EB41000E4B03EB800041
:10747000806880B901EB410003EB8000826000204E
:1074800001EB4103074C44F8230001EB4100234684
:1074900003EB8000E4E7481C81B21429E3D3002009
:1074A000DEE700002414002010B5F0210248F0F7B8
:1074B000A5FE002010BD000024140020F8B5002710
:1074C00000216846FBF70CFA0098B84203D0781CFC
:1074D0000099814201D10020F8BD009F00243BE0CB
:1074E00004EB44001E4901EB8000866804EB440075
:1074F00051F820507DB376B304EB4401184A02EBF7
:107500008101081D2946FBF7EBF9012823D104EB83
:107510004400134901EB80008068A8B104EB4400EB
:1075200001EB800040680099081AB0FBF5F004EB0D
:1075300044010B4A02EB8101496800FB051004EB92
:10754000440102EB810148602EB104EB4401044A7E
:1075500002EB8100B047641C142CC1D30020BBE7B0
:107560002414002070B504460E46254605B970BDAA
:107570002E600021281DFBF7B3F900BFF7E7014695
:107580000A460AB900207047106808B10120FAE7DE
:107590000020F8E77CB50446002611480068E0B1F9
:1075A0000021207A042801D1606800E02068CDE93C
:1075B0000001607A08B9A07A00E000200346207A32
:1075C000042801D1606800E020680146044804F105
:1075D0000B0205680020A8477CBD0020FCE70000E6
:1075E000841600202DE9FC4104460027FCF792FD9B
:1075F00060B9217A042901D1616800E02168084658
:10760000FCF79CFD10B90120BDE8FC812048806991
:1076100000283AD00021207A042801D1606800E0D7
:107620002068CDE90001607A08B9A07A00E0002066
:107630000346207A042801D1606800E020680146F2
:10764000134804F10B0285690120A847E8B1207AAC
:10765000042801D1606800E02068064600250FE09C
:107660000C4800EB05100068B04207D1094901EB56
:10767000051101F108000021FBF732F9681C85B201
:10768000022DEDD300BF0020BEE70020BCE70000C4
:10769000841600205C01002010B50C48008850B909
:1076A00001200A49088000BF0948F7F79BF909A0A3
:1076B000FDF764FD09E000200449088000BF04488C
:1076C000F7F7BBF908A0FDF759FD10BD50050020E4
:1076D000E80A0020B9D8B1D54443CEC2B6C8BCCC64
:1076E000B5E7C6F70D0A0000BFAAC6F44443CEC2F0
:1076F000B6C8BCCCB5E7C6F70D0A000010B50A48FD
:10770000008840B9012008490880F3F789FD07A0E7
:10771000FDF734FD07E0002003490880F7F704FB7C
:1077200007A0FDF72BFD10BD48050020B9D8B1D545
:10773000BDBBC1F7BCCCB5E7C6F70D0A0000000021
:10774000BFAAC6F4BDBBC1F7BCCCB5E7C6F70D0AEE
:10775000000000007047000010B50F48008868B9AD
:1077600001200D49088000BF00200C49C8710C4859
:10777000F7F738F90BA0FDF701FD0CE000200649F2
:10778000088000BF01200549C8710548F7F755F981
:1077900007A0FDF7F3FC10BD4C050020C425002018
:1077A000AC0A0020B9D8B1D543433143500D0A008B
:1077B000BFAAC6F443433143500D0A0010B50F4829
:1077C000008868B901200D49088000BF00200C49DD
:1077D00008720C48F7F706F90BA0FDF7CFFC0CE098
:1077E00000200649088000BF0120054908720548AD
:1077F000F7F723F908A0FDF7C1FC10BD4E050020E6
:10780000C4250020D40A0020B9D8B1D54343325F43
:1078100043430D0A00000000BFAAC6F44343325F91
:1078200043430D0A00000000F7F73AFA10B512487A
:10783000008880B901201049088000BF00200F494E
:1078400088710FA0FDF79AFC1148F7F7CBF811A04B
:10785000FDF794FC0FE000200749088000BF0120DD
:107860000649887110A0FDF789FC0948F7F7E5F88B
:1078700011A0FDF783FC10BD46050020C4250020A3
:10788000434C4F53455F44435265616C790D0A0088
:10789000840A0020B9D8B1D5D6B1C1F7BCCCB5E7C0
:1078A000C6F70D0A000000004F50454E5F4443529A
:1078B00065616C790D0A0000BFAAC6F4D6B1C1F7A4
:1078C000BCCCB5E7C6F70D0A000000007047704752
:1078D0007047000010B50C48008850B901200A49D3
:1078E000088000BF0948F7F77DF809A0FDF746FCBE
:1078F00009E000200449088000BF0448F7F79DF81C
:1079000007A0FDF73BFC10BD4A050020C00A00207F
:10791000B9D8B1D5C9FDD1B9C4A3BFE90D0A0000DA
:10792000BFAAC6F4C9FDD1B9C4A3BFE90D0A0000BE
:10793000704770477047000010B51048008870B954
:1079400001200E49088000BF0D48F7F74BF800BF33
:107950000C48F7F747F80CA0FDF710FC0DE00020ED
:107960000649088000BF0648F7F767F800BF0548DA
:10797000F7F763F808A0FDF701FC10BD44050020EF
:10798000C00A0020980A0020B9D8B1D5B8DFD1B913
:10799000C4A3BFE90D0A0000BFAAC6F4B8DFD1B97D
:1079A000C4A3BFE90D0A00002DE9F04705460E46C5
:1079B0000D20FBF7E7F80A20FBF7E4F82C46002738
:1079C00010E02078F6F795F880462078F6F784F8EE
:1079D00081464046FBF7D6F84846FBF7D3F8641CCF
:1079E000781C87B2B742ECDB0D20FBF7CBF80A20FE
:1079F000FBF7C8F8BDE8F08710B5FFF799F910BD9F
:107A00002DE9F04107460C461646F6F77FFBA0200D
:107A1000F6F74EFBF6F7A8FB00B130E0A046E11701
:107A200004EB1161C1F30720F6F742FBF6F79CFB6C
:107A300000B124E0E0B2F6F73BFBF6F795FB00B1AE
:107A40001DE0F6F763FBA120F6F732FBF6F78CFB9F
:107A500000B114E000250BE0711EA94201D0012104
:107A600000E000210846F6F7F9FA7855681C85B25F
:107A7000B542F1DBF6F764FB0120BDE8F081F6F7D3
:107A80005FFB0020F9E72DE9F04706460F469046D8
:107A90003C46002534E035B1E11704EBD1614911D2
:107AA000A4EB411109BB25B1F6F74AFB0620F4F718
:107AB00024FAF6F72BFBA020F6F7FAFAF6F754FBB8
:107AC00000B124E0A146E11704EB1161C1F30720E6
:107AD000F6F7EEFAF6F748FB00B118E0E0B2F6F779
:107AE000E7FAF6F741FB00B111E0705DF6F7E0FA56
:107AF000F6F73AFB00B10AE0601C84B2681C85B25C
:107B00004545C8DBF6F71CFB0120BDE8F087F6F71A
:107B100017FB0020F9E710B506E000F03BFA044639
:107B2000204601F0DDF800BF00F0FAFD0028F4D097
:107B300010BD000070B504460D46E1B21948FCF7CF
:107B400080FA00BF1748008800F080000028F9D0B4
:107B5000154890F8A800012822D1144880780228FE
:107B60001AD113480078962808DA1148027800786C
:107B7000401C0F4B18700F48845411E00C480178DA
:107B80000C48FDF765F90948007C401C074908745A
:107B900000200749087003E00020034981F8A8008D
:107BA000204670BD004C0040F816002064210020E3
:107BB0003A0500203524002038B5124A106F126FA4
:107BC000116B8847009069460F48F4F7A1FE044600
:107BD000012C0ED102210D48F8F7A8FD48B10C4840
:107BE000C07B401C0A49C8730848F8F7B2FD012061
:107BF00038BD2CB900200649C8730448F8F7A9FD20
:107C00000020F5E7D8070020942600202837002020
:107C10000426002010B5184890F8380000F0010044
:107C200040B116484079012804D115A0FDF7A6FA05
:107C3000012010BD104890F8380000F0010038B164
:107C400002200E49487114A0FDF798FA0120F0E7D0
:107C5000174908698047022801D00220E9E70A2174
:107C60001448F8F763FD20B11248F8F772FD0320BD
:107C7000DFE70020DDE70000200E0020AC2500201B
:107C8000424D535F50524F544F43414C5F47423235
:107C90003031350A0D000000424D535F50524F54B1
:107CA0004F43414C5F4742323031310A0D000000F2
:107CB0006C000020E836002010B5114908698047A3
:107CC0000446022C0ED100200E49C8730E4A106FD4
:107CD000126F116A884704280FD10CA0FDF74EFAE5
:107CE000012010BD012C08D1A0210D48F0F786FA23
:107CF0000CA0FDF743FA0220F3E70020F1E70000B3
:107D00006C00002004260020D8070020BDF8C8EB36
:107D1000D6B1C1F7B3E4B5E7C1F7B3CC0D0A0000A3
:107D2000E0360020BDF8C8EBBDBBC1F7B3E4B5E752
:107D3000C1F7B3CC0D0A000010B51048008F00F455
:107D4000804028B90D4890F8380000F0010058B183
:107D5000F4F724FC3D210948F0F750FAA021084827
:107D6000F0F74CFA012010BD064908698047022847
:107D700001D00220F7E70020F5E70000200E0020E8
:107D8000E03600206C00002010B50D48C078AA280D
:107D900004D10CA0FDF7F2F9012010BDF8F76EFA3E
:107DA00020B90FA0FDF7EAF90220F6E71A490869A1
:107DB0008047022801D00320EFE70020EDE7000014
:107DC000200E002052455620445F43445A5F4841EC
:107DD0004E44494E475F43524D2041410A0D000039
:107DE00052656164792D53746174652052656365D1
:107DF0006976656420546865204368617267696EBE
:107E0000672050696C652041626F7274204D657304
:107E1000736167650A0D00006C00002010B5F8F76B
:107E20002DFA20B909A0FDF7A9F9032010BDF9F733
:107E300043F908B90120F9E7134908698047022886
:107E400001D00320F2E70020F0E7000052756E6ECB
:107E5000696E672D53746174652052656365697638
:107E6000656420546865204368617267696E6720A5
:107E700050696C652041626F7274204D6573736147
:107E800067650A0D000000006C00002010B5214855
:107E9000807EAA2804D120A0FDF770F9012010BD32
:107EA000F8F7ECF920B923A0FDF768F90320F6E70D
:107EB0002820F4F7CDFBB8B90620F4F7C9FB98B930
:107EC0001C20F4F7C5FB78B92120F4F7C1FB58B9A1
:107ED0000920F4F7BDFB38B90A20F4F7B9FB18B94B
:107EE0002620F4F7B5FB08B10320D8E71F4908693D
:107EF0008047022801D00520D1E73C211C48F8F733
:107F000015FC20B11A48F8F724FC0420C7E700202C
:107F1000C5E70000200E002043445A5F5F43524FE4
:107F200020414120746F204368617267696E670A5F
:107F30000D00000053746172742D537461746520D8
:107F4000526563656976656420546865204368619D
:107F50007267696E672050696C652041626F727448
:107F6000204D6573736167650A0D00006C00002089
:107F70000037002010B505210548F8F7D7FB20B1E0
:107F80000348F8F7E6FB012010BD0020FCE70000E5
:107F90001837002010B500F0C3FB08B1002010BD59
:107FA000074808490968445C06480068401C0521E8
:107FB00090FBF1F201FB1200024908602046EEE757
:107FC000240C00201C0C002070B504460D46002631
:107FD00029462046F0F7F6FEF8F71CFA064630462A
:107FE00070BD014607207047704701460220704768
:107FF00010B51248008F00F4804078B100200F497E
:10800000886301200E49487100BF0E48008804466D
:10801000FEF706FA0CA0FDF7B1F80EE040F6B83115
:1080200007480830FAF75CFC38B10CA0FDF7A6F859
:10803000002103480830FAF753FC10BD200E002041
:10804000AC250020D8070020445F43445A5F4841D4
:108050004E44494E475F43484D0D0A004E4F20485D
:10806000616E647368616B65205369676E616C0A49
:108070000D000000014600207047704701460120B6
:1080800070477047014603207047000010B50B4849
:10809000007920B1012807D002280DD108E0022183
:1080A0000748F4F717FD07E00548F4F745FD03E03E
:1080B0000220F4F751FD00BF00BF10BDAC25002029
:1080C0006164010801460520704710B5F3F7AAF96D
:1080D00010BD01460420704770B500264048C07CA2
:1080E000012813D1F3F78AF980B1FCF7CDFE68B906
:1080F000F0F7F4FF50B1F8F733FB38B9394800799D
:10810000012803D1F1F74CF9064600E00026354678
:108110002C46354890F8380000F0040038B9304853
:10812000C07C012825D13048807EAA2821D0204655
:10813000FEF7D0FA2D4A106F126F916A8847012816
:108140000DD12848007950B900BF01202549887118
:1081500027A0FDF713F82A48F6F76FFC00BF0120AF
:108160001F49C8742048806B20F004001E498863B2
:1081700018E01B48C07CA8B92248007920B101282A
:1081800007D002280DD108E006211F48F4F7A2FC11
:1081900007E01D48F4F7D0FC03E00620F4F7DCFC10
:1081A00000BF00BF104890F8380000F0020030B166
:1081B0000D48806B20F002000B4988630EE00A48EE
:1081C00090F8380000F0080040B110A0FCF7D6FF8E
:1081D0000548806B20F008000349886370BD0000EB
:1081E00004260020C4250020200E0020D8070020EF
:1081F0004F50454E5F44435265616C790D0A000053
:10820000840A0020AC250020C561010843445A5F60
:1082100048414E44494E475F43524D2041410A0D6B
:1082200000000000014606207047000038B51C49D8
:10823000096FB1F90200002801DB014600E041426C
:1082400089B2009169461748F4F762FB08B1012032
:1082500000E00020044614480079012803D1012CD5
:1082600001D1F3F703F832211048FAF739FB01285E
:1082700006D10020FEF7A2FB00210C48FAF730FBE4
:10828000FA210A481030FAF72BFB012807D1002009
:10829000FEF73CFA002105481030FAF721FB38BD03
:1082A000D807002088260020C4250020E8250020CB
:1082B00070B505460E463046F5F7BEF8044604B9DB
:1082C00070BD812D26D004DC042D07D0802D4DD12A
:1082D00016E0822D0AD0832D48D128E094F854006E
:1082E000032802DB2046F5F7FFFC40E094F8540039
:1082F000032804DBE06C10B18220E16C884736E093
:1083000094F85400032804DBE06C10B18020E16C89
:1083100088472CE094F85400032807DB2046F5F743
:1083200083FDE06C10B18120E16C88471FE094F878
:108330005400032819DB9120005D022806D1042196
:108340009120015522780120FEF7F4FFE06C18B16E
:108350008320E16C884708E0207800F061FB2078FA
:1083600000231A46194600F0CDFB00E000BF00BF15
:1083700000BFA5E770B506460D463046F5F75CF838
:1083800004461CB394F85400022805DCE068E8B108
:108390003046E168884719E094F85400812808D1F4
:1083A0003DB184F85400324681210120FEF7C2FF1E
:1083B0000CE094F85400812808D03DB9802084F85E
:1083C0005400324680210120FEF7B4FF70BD70B525
:1083D00004460D4629462046FFF7CCFF70BD70B518
:1083E00005462846F5F728F804468CB194F8540061
:1083F000022805DCE06858B12846E168884707E0B4
:10840000832084F854002A4683210120FEF792FF3E
:1084100070BD00002DE9F04107460D4690461E460E
:108420003846F5F709F80446002C39D094F8540082
:10843000032835DB94F85400802802D1032084F807
:10844000540094F8400000F0010038B1A06C38B33B
:10845000324641462846A36C984721E01248056001
:1084600006710079002809DD0F480079082805DC2D
:108470000D4802794146401DEFF7A7FE0A4904F175
:10848000580002F048FE04F1580002F010FE38B126
:10849000822084F854003A4682210120FEF74AFFE8
:1084A0000120BDE8F08100007416002070B506467A
:1084B0000C463046F4F7C0FF05461DB1E1B2284630
:1084C000F5F7CBFC70BD002001E0411C88B23C28D0
:1084D000FBDB704710B514206C4981F86C0041F249
:1084E000883008800120887001216848C17000210F
:1084F0000171032141714FF47A71C18041F2680129
:108500000181422181725921C17244210173542198
:10851000417300218173C1730121017402214174EF
:10852000192181740B21C1740A2101750021417543
:1085300081751021C175002101764176112254A167
:108540001A30EFF742FE51482B3056A10A680260FC
:10855000496841604FF4D2704C49A1F833004FF4A0
:10856000FA714A48A0F8351041F22431A0F83910C8
:108570006E2180F83B10C82181874FF47A61C18752
:108580000020424981F840004FF47A60A1F8410090
:108590004FF416713D48A0F84310022180F84510B1
:1085A00000203A49A1F8460000213848A0F84810B8
:1085B000B0F84A006FF30B0000F5A2703349A1F840
:1085C0004A00084690F84B0020F0F00110312F4887
:1085D00080F84B103C21A0F84D1001202B4981F868
:1085E0004F006FF0310232490A20FCF771FCC1B232
:1085F000264880F85010032180F851106FF03102A6
:108600002B490520FCF764FCC1B2204880F85210C9
:10861000042180F85310002180F8541080F8551080
:1086200080F8561080F8571080F8581080F85910CC
:1086300080F85A100120154981F85D000021134887
:10864000A0F85E1080F860106420104981F8650081
:1086500040F259110D48A0F8661040F26311A0F8DD
:1086600068106FF0310212491920FCF731FCC1B2D9
:10867000064880F86A106FF031020D491C20FCF7A3
:1086800027FCC1B2014880F86B1010BDD80700204C
:108690004C56504335323739584E443031333831E7
:1086A00038000000533030314830303100000000D5
:1086B000CDCCCC3D2DE9F0410B3020F00706104D1C
:1086C00019E02068B04215D3B0420AD9871B201D9B
:1086D000D4F80480EFF779FDA019C0E9007828608C
:1086E00004E060682860201DEFF76FFD201D266004
:1086F000BDE8F081251D2C68002CE2D10020F7E7B1
:10870000600D00200448006804490968884201D1CE
:10871000012070470020FCE73C09002040090020B0
:108720000448006804490968884201D10120704763
:108730000020FCE71C0C0020200C002007480068EB
:10874000401C052190FBF1F201FB1200044909686D
:10875000884201D1012070470020FCE7200C002056
:108760001C0C002070B504460D4618480078B0B9BE
:1087700029462046FFF728FC154909680844144992
:108780000860144801780078401C124A10700929CA
:1087900002DB01200D4908700F48008870BD0020E1
:1087A0000A4908700A4800680C4908600020084916
:1087B000086008490870094800680A21B0FBF1F018
:1087C0000549088008460088E8E70000E10000202D
:1087D000D8000020E0000020D4000020DC000020B1
:1087E00086B0F8F71DFD62B64FF400410803F6F7B6
:1087F0004DFAF8F7D3FC01A8F7F748FCF6F7F1F9C2
:10880000F5F782FEF5F750FDFFF7F6F8F0F7D8FD23
:10881000F0F73CFBF0F7FAFA4FF47A3002F0D6FCAE
:108820004FF4E13002F02CFD40F2CF2140F2F31082
:10883000F8F76CFDF4F7FAF8FFF74CFEFBF710FCC5
:10884000F5F7FAFCFDF716FA544955A0FCF796FC2B
:10885000F7F786FDF2F750FCF4F722F801205349B0
:10886000887300BF5248F6F7E8F8F6F75DFA00BFE4
:108870000020504908725048F6F7B4F800BF0020B5
:108880004C49C8714D48F6F7ADF886E0FAF76CF838
:10889000FDF786F94A480078012828D10020484988
:1088A00008704248807B48B10320F3F7D1FE28B915
:1088B0000420F3F7CDFE08B9F0F798FBF0F72CFE93
:1088C000FBF7C9FB3F49086880473E49C8688047B5
:1088D0003C49486880473B4988688047F8F79AFADE
:1088E000F3F77AFAF0F770F9F5F79AFC55E03448A7
:1088F0004078012805D1002031494870F7F7D6FEAD
:108900004BE02F48807801280ED100202C49887038
:108910000220F4F7B7FD0446EFF70CFF00B22A4936
:108920008881FBF792FB38E02548C078012807D101
:1089300000202349C870F2F7DFFEF3F78DF82CE032
:108940001F48007901280BD100201D490871F7F755
:10895000F5FDF4F73DFAF2F703FDF6F7C9F81CE070
:1089600017484079012807D1002015494871F0F7D0
:10897000E1F8FFF7D0F810E01148C07901280CD1D8
:1089800000200F49C871F6F7D9FFF0F72BFEF7F773
:108990003DFAFCF789FBFBF70BFC77E7A0BA01086F
:1089A000B0E6B1BEBAC52025730D0A00AC25002083
:1089B000140C0020C4250020D40A0020AC0A00209A
:1089C000E816002080000020880D00202DE9F047E7
:1089D00004460F46154699463DB161190E4881423D
:1089E00003D8A0F50070844203D24FF0FF30BDE8F9
:1089F000F08737B1002602E0B85DA055761CAE4284
:108A0000FAD30648A4EB0008AAB21FFA88F1204660
:108A1000FBF742FB0020EAE7C8490020C8470020D6
:108A200070B505462846F4F707FD04461CB194F8D6
:108A30005400022801DC002070BD022084F854009C
:108A4000E06810B12846E16888479120005D002861
:108A500034D0D4F8A800B0B19120005D052804D12D
:108A60000021D4E92902904728E09120005D0428E4
:108A700004D10121D4E9290290471FE00321D4E960
:108A8000290290471AE0206DC0B19120005D0528B1
:108A900005D10021226DD4F8A40090470EE091206A
:108AA000005D042805D10121226DD4F8A40090476F
:108AB00004E00321226DD4F8A400904715E004F1EE
:108AC000940104F1700002F009FB70B1D4F8A80021
:108AD00020B10321D4E92902904706E0206D20B19E
:108AE0000321226DD4F8A400904704F1700002F035
:108AF000D5FA0028E3D0202104F19000EFF77EFBA7
:108B0000012099E72DE9F04105460E4617469846A3
:108B10002846F4F791FC04461CB194F8540001284F
:108B200002DC0020BDE8F081606848B343463A4665
:108B300031462846D4F804C0E04708B3D4F88C0086
:108B400040B194F84530182204F17000D4F88C102C
:108B500002F0B6FA94F8400000F0010058B9D4F8D9
:108B6000880040B194F84530102204F15800D4F840
:108B7000881002F0A5FA032084F854000120D1E700
:108B80000020CFE770B5054600242846F4F754FCD2
:108B9000044614B194F8540070BD0020FCE72DE9A0
:108BA000FF4180460E4615461F464046F4F744FCFA
:108BB00004464CB194F85400022805DD25B194F820
:108BC000400000F0010018B1002004B0BDE8F081C1
:108BD00004F1580002F062FA08B10020F5E7694696
:108BE00004F1580002F07AFA08B90020EDE7009885
:108BF00030609DF8040038709DF8040000280ADDFC
:108C00009DF80400082806DC9DF804200DF10501FC
:108C10002846EFF7DAFA94F85400822802D10320AC
:108C200084F854000120D0E72DE9F04786B0804653
:108C30000F4615461E46DDE90E9A00244046F4F71D
:108C4000FBFB044654B194F85400022806DD082EBC
:108C500004DC04F1700002F02AFA18B1002006B01A
:108C6000BDE8F087F7F7E3FC94F85400832803D0BD
:108C700094F85400032803DAF7F7DBFC0020EEE752
:108C8000CDF814A000978DF80560CDF8109015B9B7
:108C900000208DF805009DF8050000280ADD9DF8EC
:108CA0000500082806DC9DF8052029460DF1060080
:108CB000EFF78BFAFF208DF80400694604F170008D
:108CC00002F029FA9120005D10B92046F5F70CF862
:108CD000F7F7AFFC0120C2E7034600207047000011
:108CE00010B50446062C13D2DFE804F0120306097F
:108CF0000C0FF3F7C3FB0FE0F3F7FEFB0CE0F3F709
:108D000007FC09E0F3F7C6FB06E0F3F70DFC03E010
:108D100002A0FCF733FA00BF00BF10BD556E6B6EAA
:108D20006F776E206576656E742069732069676E53
:108D30006F7265640A000000F0B54FF480541B4A5E
:108D40000023072702EA070600256E406D402E43E8
:108D500007D0D21D6FF0070602EA0602134D551B1D
:108D6000641B1146124D29604FF00005104E7560CE
:108D70000A19083A6FF0070602EA06020D4D2A604A
:108D80004FF000050B4E366875600A4E3668356048
:108D90000846151A4560074D2D680560064E456862
:108DA0003560064E45683560F0BD0000DE260020C7
:108DB0002C0C0020340C00203C0C0020380C00202F
:108DC00010B50146184800E0006803688B42FBD3E9
:108DD0000246436813448B4205D143684C682344E0
:108DE0004360014600E000BF0A464B681344046834
:108DF000A34211D10D4C03682468A34208D04B68EC
:108E00000468646823444B6003681B680B6005E0DA
:108E1000064B1B680B6001E003680B60884201D0C1
:108E2000016000E000BF10BD2C0C0020340C0020BD
:108E30002DE9F04705464FF000093848006810B9A1
:108E4000FFF77AFF00E000BF7DB105F00700C0F139
:108E50001008C8F1FF30A84201D2012000E0002034
:108E600008B9454402E0002500E000BF012000EB06
:108E7000E57000284CD0002D48D029480068854274
:108E800044D8284E3046046801E0264624686068CD
:108E9000A84202D220680028F7D120480068844206
:108EA00032D0306800F10809206830606068401BEB
:108EB00010280AD9671900BF00BF6068401B78609E
:108EC00065603846FFF77CFF00E000BF144960682A
:108ED0000968081A124908600846006812490968BA
:108EE000884204D20E4800680F49086000E000BFC5
:108EF000606840F000406060002020600B4800681F
:108F0000401C0A49086004E000BF02E000BF00E026
:108F100000BF00BF00BF4846BDE8F087340C00200A
:108F2000380C00202C0C00203C0C0020400C0020B1
:108F30002DE9F04F99B0834600201890402106A8F3
:108F4000EFF75CF9002005904FF6FF7004905C4647
:108F50000020F1490874B4F8050048F22001884265
:108F600004D0B4F80500491C884243D1CDF80CB0B8
:108F7000B4F802A0B4F8050002906088B0F5967FBE
:108F800004DC6288E11DE548EFF71FF95146E3482C
:108F9000FEF70AFDAAF1020003990A5C401C085C76
:108FA00042EA00201690AAF1020081B20398F0F77D
:108FB0002FFA1790DAA0DDE91612FCF7DFF8DDE9E9
:108FC0001601884205D0DCA0FCF7D8F819B0BDE83E
:108FD000F08F0020D04948740299E031C8B252465F
:108FE000CE49FBF75DFC6420DB4908800420CA49B8
:108FF0008870EBE7B4F80500B0F5004F5FD034DCC3
:10900000B0F5D06F01F0C38714DCB0F5607F72D08B
:1090100009DC802854D0B0F5C07F79D0B0F5207F2E
:1090200041F0E68783E0B0F5906F66D0B0F5B06FA1
:10903000F6D1AAE0B0F5286F01F0D2870CDCB0F5CC
:10904000F06F01F0B787B0F5086F01F0B887B0F5A1
:10905000186FE5D101F0B8BFB0F5025F01F0C58728
:10906000B0F5065FDCD101F0C2BF48F20702811AF9
:10907000904201F09E870DDC6FF400410844062801
:1090800081F0B687DFE810F043005200610066000F
:109090008000820F062901F09C8709DC012901F07C
:1090A0008D87022901F08F870329B9D101F090BF84
:1090B000192901F099871A29B2D101F097BF00BF91
:1090C000E07901281ED194498870A44981F876007E
:1090D00008460021C1660167A0F874100146A26825
:1090E000CA66E068086701208B4988709C4908704F
:1090F0009A496C3102E029E00AE02CE099A0FCF7E3
:109100003DF802E09FA0FCF739F801F072BF00BF04
:10911000E079012806D102207F4988709EA0FCF7E3
:109120002DF802E0A1A0FCF729F8EEE700BFE179F5
:10913000A2A0FCF723F8A649D4F809200A60B4F8E5
:109140000D208A80E07B8871DFE700BFA1A0FCF7DB
:1091500015F8DAE700BFA5A0FCF710F8207A01287F
:1091600001D1A8A000E0A9A00146AAA0FCF706F83A
:10917000207A40B90120AA490870AA48007810B99D
:109180000420A8490870C0E700BF0120A649087064
:10919000E07918B9A5A0FBF7F1FF02E0A7A0FBF763
:1091A000EDFFE079012841F07786267A3146A7A0C5
:1091B000FBF7E4FF012E14D1607A40B901209849F1
:1091C00008709848007810B9042096490870607AB1
:1091D000012801D1A1A000E0A2A00146A3A0FBF7B5
:1091E000CDFF022E09D1607A012803D1A3A0FBF79D
:1091F000C5FF02E0A5A0FBF7C1FF042E1BD104F1BF
:109200000900EFF718F885B2102D0FD22A4604F1A5
:10921000090152481030EEF7D8FF04F109019FA070
:10922000FBF7ACFF01204E49087004E004F109018E
:109230009FA0FBF7A3FF072E0AD1657A2946A3A0BA
:10924000FBF79CFF4548A0F869500120444908708D
:10925000062E0ED1657A2946A3A0FBF78FFF3F4863
:10926000A0F84D50A0F84F50A0F8515001203C49B3
:109270000870082E03D1657A012039490870092E3B
:109280001DD104F10900EEF7D6FF85B2102D0ED2E4
:109290002A4604F109013148EEF797FF04F109016C
:1092A00097A0FBF76BFF01202D49087004E004F143
:1092B000090199A0FBF762FF0120294908700A2ED5
:1092C00014D1657A012D07D10120244981F8870046
:1092D00098A0FBF753FF06E00020204981F88700A3
:1092E00094A0FBF74BFF01201D4908700B2E00D105
:1092F000657A0C2E0FD1657A012D07D1012017490F
:1093000081F8890091A0FBF739FF32E10020134971
:1093100081F889002AE12FE1642100206A220020DF
:109320000A0D44637263202530782C5663726320E3
:109330002530780A0D0000000A0D2028446372636E
:1093400020213D2056637263292072657475726E08
:1093500021212121210A0D0038050020F8160020C6
:10936000FC0100207265676973746572656420731F
:1093700075636365737365642C436F64652025733F
:109380000A0D000072656769737465726564206612
:1093900061696C65640A0D004C6F67696E205375D6
:1093A000636365737365640A0D0000004C6F676941
:1093B0006E204661696C65640A0D00006865617223
:1093C0007420636F756E742025640A0D0000000020
:1093D000150E00207265636569766520737461748B
:1093E000652064617461200A0D0000007265636588
:1093F00069766520636861726765206461746120C5
:109400000A0D0000456E61626C650000446973617D
:10941000626C65006368617267652025730A0D00E0
:10942000350500200C0200203605002070617261B5
:109430006D20726561640A0D000000007061726148
:109440006D2077726974650A0D00000070617261A9
:109450006D20616464722025780A0D00656E61627A
:109460006C65000064697361626C650063686172B9
:1094700067696E672025730A0D000000636C6F73C7
:10948000652072656C61790A0D0000006F70656E71
:109490002072656C61790A0D00000000626C7565D0
:1094A000746F6F7468206E616D652025730A0D00FE
:1094B000626C7565746F6F7468206E616D65206D88
:1094C000697374616B652025730A0D0048656172CC
:1094D0007420426561742054696D652025642020E4
:1094E0007365630A0D0000004F76657254656D70F8
:1094F00056616C75652025642020200A0D0000004F
:109500005379735061726150696C65442E736E3A81
:1095100025730A0D00000000537973506172615089
:10952000696C65442E736E206661756C74202573BA
:109530000A0D0000517569636B20436861726765AD
:1095400020456E61626C650A0D00000074726963EB
:109550006B6C65204368617267696E6720536F6347
:1095600020456E61626C6520310A0D00F3A0FBF7A7
:1095700005FE0120F94908700D2E14D1657A642D7D
:1095800007DAF74981F88A502946F6A0FBF7F6FD7D
:1095900006E0FAA0FBF7F2FD5A20F14981F88A00B3
:1095A0000120EE4908700E2E15D1657A0A2095FB30
:1095B000F0F100FB115001900A2095FBF0F00090B3
:1095C0000146F4A0019AFBF7D9FDE54880F88B50DD
:1095D0000120E24908700F2E0ED1657A2946F3A0CA
:1095E000FBF7CCFD05EB85004006000EDC4981F859
:1095F0008C000120D9490870102E37D1617AA07AE9
:1096000041EA00252946EFA0FBF7B8FDD448B0F8A1
:10961000590005EB8501B0EB410F0CDD05EB850032
:109620004FF6FF7101EA4000CD49A1F88300012007
:10963000CA4908701AE0CA48B0F8592005EB8500FD
:109640004100E4A0FBF79AFDC548B0F85900143872
:10965000C349A1F883000846B0F883000A2190FBB3
:10966000F1F001460190E2A0FBF788FD112E25D113
:10967000617AA07A41EA00252946E2A0FBF77EFD47
:10968000B748B0F85B0005EB8501B0EB410F0CDD8E
:1096900005EB85004FF6FF7101EA4000B049A1F8E3
:1096A00085000120AD49087008E0AD48B0F85B20A6
:1096B00005EB85004100D8A0FBF760FD122E13D109
:1096C000617AA07A41EA00252946D9A0FBF756FD28
:1096D00005EB85004FF6FF7101EA4000A049A1F8B3
:1096E000590001209D490870132E13D1617AA07A88
:1096F00041EA00252946D3A0FBF740FD05EB850094
:109700004FF6FF7101EA40009549A1F85B00012086
:1097100092490870142E19D1657A2946CEA0FBF71C
:109720002DFDD2488078202802DD2020CF49887086
:10973000CE48807800EBC001CC48C01C00EB410053
:109740008580CA488078401CC8498870162E18D178
:10975000617AA07A41EA00258148A0F863500A2086
:1097600095FBF0F100FB115001900A2095FBF0F001
:1097700000900146BEA0019AFBF700FD0120774949
:1097800008701D2E17D1657A012D01D0022D0FD141
:10979000734981F88D50012D01D1BBA000E0BBA021
:1097A0000146BBA0FBF7EAFC01206C49087002E00F
:1097B000BCA0FBF7E3FC1E2E20D1657A05EB8500EB
:1097C0004FF6FF7101EA40006549A1F853000846D1
:1097D000B0F853000A2190FBF1F201FB1200019056
:1097E0005F48B0F8530090FBF1F000900146B3A041
:1097F000019AFBF7C3FC0120584908701F2E50D175
:10980000657A5748B0F890005549B1F8531088422E
:1098100027DD5348B0F853000A2190FBF1F0019086
:109820004F48B0F8900090FBF1F000900146A9A0DD
:10983000019AFBF7A3FC4A48B0F853000A3848499C
:10984000A1F890000846B0F890000A2190FBF1F0D2
:1098500001460190AAA0FBF791FC01203F49087046
:109860001FE005EB85004FF6FF7101EA40003C491F
:10987000A1F890000846B0F890000A2190FBF1F2A0
:1098800001FB120001903648B0F8900090FBF1F017
:1098900000900146A0A0019AFBF770FC01202F491F
:1098A0000870202E1DD1657A05EB85004FF6FF71FB
:1098B00001EA40002A49A1F8B3000846B0F8B30015
:1098C000642190FBF1F201FB120001902448B0F8F2
:1098D000B30090FBF1F00090014696A0019AFBF7CF
:1098E0004DFC212E20D1657A05EB85004FF6FF71E6
:1098F00001EA40001A49A1F8B1000846B0F8B100E9
:10990000642190FBF1F201FB120001901448B0F8C1
:10991000B10090FBF1F0009001468DA0019AFBF799
:109920002DFC01200D490870222E06D1657A0C48C5
:10993000A0F8B750B0F8B71018E11DE17472696370
:109940006B6C65204368617267696E6720536F6353
:1099500020456E61626C6520300A0D00FC0100201C
:10996000F8160020747269636B6C654368617267F6
:10997000696E67536F6325640A0D00007472696332
:109980006B6C654368617267696E67536F632039FA
:10999000300A0D00747269636B6C6520706F7765B7
:1099A000722025642E25646B770A0D00747269633A
:1099B0006B6C652063757272656E742564410A0D67
:1099C00000000000426D734D6178566F6C74256421
:1099D000200A0D00256420426D734D6178566F6C2E
:1099E00074202564206661696C640A0D0000000023
:1099F000426D52657175697265566F6C742025648D
:109A0000200A0D00426D734D617843757272656E68
:109A100074202564200A0D00726571202564206F72
:109A2000766572206D6178202564200A0D000000A3
:109A3000426D734D6178566F6C74202564200A0D59
:109A400000000000426D734D617843757272656E5F
:109A5000742564200A0D000073657474696E6720B4
:109A6000736F63282564290A0D0000005419002033
:109A7000754261744D6178456E6572677920256421
:109A80002E25640A0D0000004343000043560000E9
:109A90004368617267696E674D6F64653A2573202C
:109AA0000A0D00004368617267696E674D6F6465F7
:109AB000204661756C740A0D000000004F766572D7
:109AC000506F776572203A25642E25646B77680A9B
:109AD0000D00000052657175697265506F7765728F
:109AE000202564206B77204F766572506F77657202
:109AF000203A25646B772C6661756C740A0D000042
:109B000052657175697265506F77657220256420A2
:109B10006B77200A0D0000005265717569726550FF
:109B20006F776572203A25642E25646B77680A0D7D
:109B3000000000004261745261746564566F6C7479
:109B4000616765203A25642E2564560A0D000000E1
:109B50004261744D6178436861726765566F6C202D
:109B60003A25642E2564560A0D000000EDA0FBF78F
:109B700005FB0120EF490870232E1CD1617AA07AE1
:109B800041EA0025EC48A0F85F50B0F85F000A21D8
:109B900090FBF1F201FB12000190E748B0F85F0082
:109BA00090FBF1F000900146E4A0019AFBF7E6FA81
:109BB0000120E0490870242E1CD1617AA07A41EA84
:109BC0000025DD48A0F85950B0F859000A2190FB53
:109BD000F1F201FB12000190D748B0F8590090FB58
:109BE000F1F000900146DCA0019AFBF7C7FA0120D2
:109BF000D0490870252E0CD1657A2946DBA0FBF7E9
